
sharp_lcd_l4.elf:     file format elf32-littlearm

Sections:
Idx Name          Size      VMA       LMA       File off  Algn
  0 .isr_vector   00000188  08000000  08000000  00010000  2**0
                  CONTENTS, ALLOC, LOAD, READONLY, DATA
  1 .text         000067d0  08000188  08000188  00010188  2**3
                  CONTENTS, ALLOC, LOAD, READONLY, CODE
  2 .rodata       000056f4  08006958  08006958  00016958  2**2
                  CONTENTS, ALLOC, LOAD, READONLY, DATA
  3 .ARM.extab    00000000  0800c04c  0800c04c  0002001c  2**0
                  CONTENTS
  4 .ARM          00000000  0800c04c  0800c04c  0002001c  2**0
                  CONTENTS
  5 .preinit_array 00000000  0800c04c  0800c04c  0002001c  2**0
                  CONTENTS, ALLOC, LOAD, DATA
  6 .init_array   00000008  0800c04c  0800c04c  0001c04c  2**2
                  CONTENTS, ALLOC, LOAD, DATA
  7 .fini_array   00000004  0800c054  0800c054  0001c054  2**2
                  CONTENTS, ALLOC, LOAD, DATA
  8 .data         0000001c  20000000  0800c058  00020000  2**2
                  CONTENTS, ALLOC, LOAD, DATA
  9 .bss          00004f1c  2000001c  0800c074  0002001c  2**2
                  ALLOC
 10 ._user_heap_stack 00000600  20004f38  0800c074  00024f38  2**0
                  ALLOC
 11 .ARM.attributes 00000030  00000000  00000000  0002001c  2**0
                  CONTENTS, READONLY
 12 .debug_info   0001c98f  00000000  00000000  0002004c  2**0
                  CONTENTS, READONLY, DEBUGGING
 13 .debug_abbrev 000033e5  00000000  00000000  0003c9db  2**0
                  CONTENTS, READONLY, DEBUGGING
 14 .debug_aranges 00001460  00000000  00000000  0003fdc0  2**3
                  CONTENTS, READONLY, DEBUGGING
 15 .debug_ranges 00001338  00000000  00000000  00041220  2**3
                  CONTENTS, READONLY, DEBUGGING
 16 .debug_macro  000054b2  00000000  00000000  00042558  2**0
                  CONTENTS, READONLY, DEBUGGING
 17 .debug_line   0001045a  00000000  00000000  00047a0a  2**0
                  CONTENTS, READONLY, DEBUGGING
 18 .debug_str    000f5e77  00000000  00000000  00057e64  2**0
                  CONTENTS, READONLY, DEBUGGING
 19 .comment      0000007b  00000000  00000000  0014dcdb  2**0
                  CONTENTS, READONLY
 20 .debug_frame  00005668  00000000  00000000  0014dd58  2**2
                  CONTENTS, READONLY, DEBUGGING

Disassembly of section .text:

08000188 <__do_global_dtors_aux>:
 8000188:	b510      	push	{r4, lr}
 800018a:	4c05      	ldr	r4, [pc, #20]	; (80001a0 <__do_global_dtors_aux+0x18>)
 800018c:	7823      	ldrb	r3, [r4, #0]
 800018e:	b933      	cbnz	r3, 800019e <__do_global_dtors_aux+0x16>
 8000190:	4b04      	ldr	r3, [pc, #16]	; (80001a4 <__do_global_dtors_aux+0x1c>)
 8000192:	b113      	cbz	r3, 800019a <__do_global_dtors_aux+0x12>
 8000194:	4804      	ldr	r0, [pc, #16]	; (80001a8 <__do_global_dtors_aux+0x20>)
 8000196:	f3af 8000 	nop.w
 800019a:	2301      	movs	r3, #1
 800019c:	7023      	strb	r3, [r4, #0]
 800019e:	bd10      	pop	{r4, pc}
 80001a0:	2000001c 	.word	0x2000001c
 80001a4:	00000000 	.word	0x00000000
 80001a8:	08006940 	.word	0x08006940

080001ac <frame_dummy>:
 80001ac:	b508      	push	{r3, lr}
 80001ae:	4b03      	ldr	r3, [pc, #12]	; (80001bc <frame_dummy+0x10>)
 80001b0:	b11b      	cbz	r3, 80001ba <frame_dummy+0xe>
 80001b2:	4903      	ldr	r1, [pc, #12]	; (80001c0 <frame_dummy+0x14>)
 80001b4:	4803      	ldr	r0, [pc, #12]	; (80001c4 <frame_dummy+0x18>)
 80001b6:	f3af 8000 	nop.w
 80001ba:	bd08      	pop	{r3, pc}
 80001bc:	00000000 	.word	0x00000000
 80001c0:	20000020 	.word	0x20000020
 80001c4:	08006940 	.word	0x08006940

080001c8 <__aeabi_drsub>:
 80001c8:	f081 4100 	eor.w	r1, r1, #2147483648	; 0x80000000
 80001cc:	e002      	b.n	80001d4 <__adddf3>
 80001ce:	bf00      	nop

080001d0 <__aeabi_dsub>:
 80001d0:	f083 4300 	eor.w	r3, r3, #2147483648	; 0x80000000

080001d4 <__adddf3>:
 80001d4:	b530      	push	{r4, r5, lr}
 80001d6:	ea4f 0441 	mov.w	r4, r1, lsl #1
 80001da:	ea4f 0543 	mov.w	r5, r3, lsl #1
 80001de:	ea94 0f05 	teq	r4, r5
 80001e2:	bf08      	it	eq
 80001e4:	ea90 0f02 	teqeq	r0, r2
 80001e8:	bf1f      	itttt	ne
 80001ea:	ea54 0c00 	orrsne.w	ip, r4, r0
 80001ee:	ea55 0c02 	orrsne.w	ip, r5, r2
 80001f2:	ea7f 5c64 	mvnsne.w	ip, r4, asr #21
 80001f6:	ea7f 5c65 	mvnsne.w	ip, r5, asr #21
 80001fa:	f000 80e2 	beq.w	80003c2 <__adddf3+0x1ee>
 80001fe:	ea4f 5454 	mov.w	r4, r4, lsr #21
 8000202:	ebd4 5555 	rsbs	r5, r4, r5, lsr #21
 8000206:	bfb8      	it	lt
 8000208:	426d      	neglt	r5, r5
 800020a:	dd0c      	ble.n	8000226 <__adddf3+0x52>
 800020c:	442c      	add	r4, r5
 800020e:	ea80 0202 	eor.w	r2, r0, r2
 8000212:	ea81 0303 	eor.w	r3, r1, r3
 8000216:	ea82 0000 	eor.w	r0, r2, r0
 800021a:	ea83 0101 	eor.w	r1, r3, r1
 800021e:	ea80 0202 	eor.w	r2, r0, r2
 8000222:	ea81 0303 	eor.w	r3, r1, r3
 8000226:	2d36      	cmp	r5, #54	; 0x36
 8000228:	bf88      	it	hi
 800022a:	bd30      	pophi	{r4, r5, pc}
 800022c:	f011 4f00 	tst.w	r1, #2147483648	; 0x80000000
 8000230:	ea4f 3101 	mov.w	r1, r1, lsl #12
 8000234:	f44f 1c80 	mov.w	ip, #1048576	; 0x100000
 8000238:	ea4c 3111 	orr.w	r1, ip, r1, lsr #12
 800023c:	d002      	beq.n	8000244 <__adddf3+0x70>
 800023e:	4240      	negs	r0, r0
 8000240:	eb61 0141 	sbc.w	r1, r1, r1, lsl #1
 8000244:	f013 4f00 	tst.w	r3, #2147483648	; 0x80000000
 8000248:	ea4f 3303 	mov.w	r3, r3, lsl #12
 800024c:	ea4c 3313 	orr.w	r3, ip, r3, lsr #12
 8000250:	d002      	beq.n	8000258 <__adddf3+0x84>
 8000252:	4252      	negs	r2, r2
 8000254:	eb63 0343 	sbc.w	r3, r3, r3, lsl #1
 8000258:	ea94 0f05 	teq	r4, r5
 800025c:	f000 80a7 	beq.w	80003ae <__adddf3+0x1da>
 8000260:	f1a4 0401 	sub.w	r4, r4, #1
 8000264:	f1d5 0e20 	rsbs	lr, r5, #32
 8000268:	db0d      	blt.n	8000286 <__adddf3+0xb2>
 800026a:	fa02 fc0e 	lsl.w	ip, r2, lr
 800026e:	fa22 f205 	lsr.w	r2, r2, r5
 8000272:	1880      	adds	r0, r0, r2
 8000274:	f141 0100 	adc.w	r1, r1, #0
 8000278:	fa03 f20e 	lsl.w	r2, r3, lr
 800027c:	1880      	adds	r0, r0, r2
 800027e:	fa43 f305 	asr.w	r3, r3, r5
 8000282:	4159      	adcs	r1, r3
 8000284:	e00e      	b.n	80002a4 <__adddf3+0xd0>
 8000286:	f1a5 0520 	sub.w	r5, r5, #32
 800028a:	f10e 0e20 	add.w	lr, lr, #32
 800028e:	2a01      	cmp	r2, #1
 8000290:	fa03 fc0e 	lsl.w	ip, r3, lr
 8000294:	bf28      	it	cs
 8000296:	f04c 0c02 	orrcs.w	ip, ip, #2
 800029a:	fa43 f305 	asr.w	r3, r3, r5
 800029e:	18c0      	adds	r0, r0, r3
 80002a0:	eb51 71e3 	adcs.w	r1, r1, r3, asr #31
 80002a4:	f001 4500 	and.w	r5, r1, #2147483648	; 0x80000000
 80002a8:	d507      	bpl.n	80002ba <__adddf3+0xe6>
 80002aa:	f04f 0e00 	mov.w	lr, #0
 80002ae:	f1dc 0c00 	rsbs	ip, ip, #0
 80002b2:	eb7e 0000 	sbcs.w	r0, lr, r0
 80002b6:	eb6e 0101 	sbc.w	r1, lr, r1
 80002ba:	f5b1 1f80 	cmp.w	r1, #1048576	; 0x100000
 80002be:	d31b      	bcc.n	80002f8 <__adddf3+0x124>
 80002c0:	f5b1 1f00 	cmp.w	r1, #2097152	; 0x200000
 80002c4:	d30c      	bcc.n	80002e0 <__adddf3+0x10c>
 80002c6:	0849      	lsrs	r1, r1, #1
 80002c8:	ea5f 0030 	movs.w	r0, r0, rrx
 80002cc:	ea4f 0c3c 	mov.w	ip, ip, rrx
 80002d0:	f104 0401 	add.w	r4, r4, #1
 80002d4:	ea4f 5244 	mov.w	r2, r4, lsl #21
 80002d8:	f512 0f80 	cmn.w	r2, #4194304	; 0x400000
 80002dc:	f080 809a 	bcs.w	8000414 <__adddf3+0x240>
 80002e0:	f1bc 4f00 	cmp.w	ip, #2147483648	; 0x80000000
 80002e4:	bf08      	it	eq
 80002e6:	ea5f 0c50 	movseq.w	ip, r0, lsr #1
 80002ea:	f150 0000 	adcs.w	r0, r0, #0
 80002ee:	eb41 5104 	adc.w	r1, r1, r4, lsl #20
 80002f2:	ea41 0105 	orr.w	r1, r1, r5
 80002f6:	bd30      	pop	{r4, r5, pc}
 80002f8:	ea5f 0c4c 	movs.w	ip, ip, lsl #1
 80002fc:	4140      	adcs	r0, r0
 80002fe:	eb41 0101 	adc.w	r1, r1, r1
 8000302:	f411 1f80 	tst.w	r1, #1048576	; 0x100000
 8000306:	f1a4 0401 	sub.w	r4, r4, #1
 800030a:	d1e9      	bne.n	80002e0 <__adddf3+0x10c>
 800030c:	f091 0f00 	teq	r1, #0
 8000310:	bf04      	itt	eq
 8000312:	4601      	moveq	r1, r0
 8000314:	2000      	moveq	r0, #0
 8000316:	fab1 f381 	clz	r3, r1
 800031a:	bf08      	it	eq
 800031c:	3320      	addeq	r3, #32
 800031e:	f1a3 030b 	sub.w	r3, r3, #11
 8000322:	f1b3 0220 	subs.w	r2, r3, #32
 8000326:	da0c      	bge.n	8000342 <__adddf3+0x16e>
 8000328:	320c      	adds	r2, #12
 800032a:	dd08      	ble.n	800033e <__adddf3+0x16a>
 800032c:	f102 0c14 	add.w	ip, r2, #20
 8000330:	f1c2 020c 	rsb	r2, r2, #12
 8000334:	fa01 f00c 	lsl.w	r0, r1, ip
 8000338:	fa21 f102 	lsr.w	r1, r1, r2
 800033c:	e00c      	b.n	8000358 <__adddf3+0x184>
 800033e:	f102 0214 	add.w	r2, r2, #20
 8000342:	bfd8      	it	le
 8000344:	f1c2 0c20 	rsble	ip, r2, #32
 8000348:	fa01 f102 	lsl.w	r1, r1, r2
 800034c:	fa20 fc0c 	lsr.w	ip, r0, ip
 8000350:	bfdc      	itt	le
 8000352:	ea41 010c 	orrle.w	r1, r1, ip
 8000356:	4090      	lslle	r0, r2
 8000358:	1ae4      	subs	r4, r4, r3
 800035a:	bfa2      	ittt	ge
 800035c:	eb01 5104 	addge.w	r1, r1, r4, lsl #20
 8000360:	4329      	orrge	r1, r5
 8000362:	bd30      	popge	{r4, r5, pc}
 8000364:	ea6f 0404 	mvn.w	r4, r4
 8000368:	3c1f      	subs	r4, #31
 800036a:	da1c      	bge.n	80003a6 <__adddf3+0x1d2>
 800036c:	340c      	adds	r4, #12
 800036e:	dc0e      	bgt.n	800038e <__adddf3+0x1ba>
 8000370:	f104 0414 	add.w	r4, r4, #20
 8000374:	f1c4 0220 	rsb	r2, r4, #32
 8000378:	fa20 f004 	lsr.w	r0, r0, r4
 800037c:	fa01 f302 	lsl.w	r3, r1, r2
 8000380:	ea40 0003 	orr.w	r0, r0, r3
 8000384:	fa21 f304 	lsr.w	r3, r1, r4
 8000388:	ea45 0103 	orr.w	r1, r5, r3
 800038c:	bd30      	pop	{r4, r5, pc}
 800038e:	f1c4 040c 	rsb	r4, r4, #12
 8000392:	f1c4 0220 	rsb	r2, r4, #32
 8000396:	fa20 f002 	lsr.w	r0, r0, r2
 800039a:	fa01 f304 	lsl.w	r3, r1, r4
 800039e:	ea40 0003 	orr.w	r0, r0, r3
 80003a2:	4629      	mov	r1, r5
 80003a4:	bd30      	pop	{r4, r5, pc}
 80003a6:	fa21 f004 	lsr.w	r0, r1, r4
 80003aa:	4629      	mov	r1, r5
 80003ac:	bd30      	pop	{r4, r5, pc}
 80003ae:	f094 0f00 	teq	r4, #0
 80003b2:	f483 1380 	eor.w	r3, r3, #1048576	; 0x100000
 80003b6:	bf06      	itte	eq
 80003b8:	f481 1180 	eoreq.w	r1, r1, #1048576	; 0x100000
 80003bc:	3401      	addeq	r4, #1
 80003be:	3d01      	subne	r5, #1
 80003c0:	e74e      	b.n	8000260 <__adddf3+0x8c>
 80003c2:	ea7f 5c64 	mvns.w	ip, r4, asr #21
 80003c6:	bf18      	it	ne
 80003c8:	ea7f 5c65 	mvnsne.w	ip, r5, asr #21
 80003cc:	d029      	beq.n	8000422 <__adddf3+0x24e>
 80003ce:	ea94 0f05 	teq	r4, r5
 80003d2:	bf08      	it	eq
 80003d4:	ea90 0f02 	teqeq	r0, r2
 80003d8:	d005      	beq.n	80003e6 <__adddf3+0x212>
 80003da:	ea54 0c00 	orrs.w	ip, r4, r0
 80003de:	bf04      	itt	eq
 80003e0:	4619      	moveq	r1, r3
 80003e2:	4610      	moveq	r0, r2
 80003e4:	bd30      	pop	{r4, r5, pc}
 80003e6:	ea91 0f03 	teq	r1, r3
 80003ea:	bf1e      	ittt	ne
 80003ec:	2100      	movne	r1, #0
 80003ee:	2000      	movne	r0, #0
 80003f0:	bd30      	popne	{r4, r5, pc}
 80003f2:	ea5f 5c54 	movs.w	ip, r4, lsr #21
 80003f6:	d105      	bne.n	8000404 <__adddf3+0x230>
 80003f8:	0040      	lsls	r0, r0, #1
 80003fa:	4149      	adcs	r1, r1
 80003fc:	bf28      	it	cs
 80003fe:	f041 4100 	orrcs.w	r1, r1, #2147483648	; 0x80000000
 8000402:	bd30      	pop	{r4, r5, pc}
 8000404:	f514 0480 	adds.w	r4, r4, #4194304	; 0x400000
 8000408:	bf3c      	itt	cc
 800040a:	f501 1180 	addcc.w	r1, r1, #1048576	; 0x100000
 800040e:	bd30      	popcc	{r4, r5, pc}
 8000410:	f001 4500 	and.w	r5, r1, #2147483648	; 0x80000000
 8000414:	f045 41fe 	orr.w	r1, r5, #2130706432	; 0x7f000000
 8000418:	f441 0170 	orr.w	r1, r1, #15728640	; 0xf00000
 800041c:	f04f 0000 	mov.w	r0, #0
 8000420:	bd30      	pop	{r4, r5, pc}
 8000422:	ea7f 5c64 	mvns.w	ip, r4, asr #21
 8000426:	bf1a      	itte	ne
 8000428:	4619      	movne	r1, r3
 800042a:	4610      	movne	r0, r2
 800042c:	ea7f 5c65 	mvnseq.w	ip, r5, asr #21
 8000430:	bf1c      	itt	ne
 8000432:	460b      	movne	r3, r1
 8000434:	4602      	movne	r2, r0
 8000436:	ea50 3401 	orrs.w	r4, r0, r1, lsl #12
 800043a:	bf06      	itte	eq
 800043c:	ea52 3503 	orrseq.w	r5, r2, r3, lsl #12
 8000440:	ea91 0f03 	teqeq	r1, r3
 8000444:	f441 2100 	orrne.w	r1, r1, #524288	; 0x80000
 8000448:	bd30      	pop	{r4, r5, pc}
 800044a:	bf00      	nop

0800044c <__aeabi_ui2d>:
 800044c:	f090 0f00 	teq	r0, #0
 8000450:	bf04      	itt	eq
 8000452:	2100      	moveq	r1, #0
 8000454:	4770      	bxeq	lr
 8000456:	b530      	push	{r4, r5, lr}
 8000458:	f44f 6480 	mov.w	r4, #1024	; 0x400
 800045c:	f104 0432 	add.w	r4, r4, #50	; 0x32
 8000460:	f04f 0500 	mov.w	r5, #0
 8000464:	f04f 0100 	mov.w	r1, #0
 8000468:	e750      	b.n	800030c <__adddf3+0x138>
 800046a:	bf00      	nop

0800046c <__aeabi_i2d>:
 800046c:	f090 0f00 	teq	r0, #0
 8000470:	bf04      	itt	eq
 8000472:	2100      	moveq	r1, #0
 8000474:	4770      	bxeq	lr
 8000476:	b530      	push	{r4, r5, lr}
 8000478:	f44f 6480 	mov.w	r4, #1024	; 0x400
 800047c:	f104 0432 	add.w	r4, r4, #50	; 0x32
 8000480:	f010 4500 	ands.w	r5, r0, #2147483648	; 0x80000000
 8000484:	bf48      	it	mi
 8000486:	4240      	negmi	r0, r0
 8000488:	f04f 0100 	mov.w	r1, #0
 800048c:	e73e      	b.n	800030c <__adddf3+0x138>
 800048e:	bf00      	nop

08000490 <__aeabi_f2d>:
 8000490:	0042      	lsls	r2, r0, #1
 8000492:	ea4f 01e2 	mov.w	r1, r2, asr #3
 8000496:	ea4f 0131 	mov.w	r1, r1, rrx
 800049a:	ea4f 7002 	mov.w	r0, r2, lsl #28
 800049e:	bf1f      	itttt	ne
 80004a0:	f012 437f 	andsne.w	r3, r2, #4278190080	; 0xff000000
 80004a4:	f093 4f7f 	teqne	r3, #4278190080	; 0xff000000
 80004a8:	f081 5160 	eorne.w	r1, r1, #939524096	; 0x38000000
 80004ac:	4770      	bxne	lr
 80004ae:	f032 427f 	bics.w	r2, r2, #4278190080	; 0xff000000
 80004b2:	bf08      	it	eq
 80004b4:	4770      	bxeq	lr
 80004b6:	f093 4f7f 	teq	r3, #4278190080	; 0xff000000
 80004ba:	bf04      	itt	eq
 80004bc:	f441 2100 	orreq.w	r1, r1, #524288	; 0x80000
 80004c0:	4770      	bxeq	lr
 80004c2:	b530      	push	{r4, r5, lr}
 80004c4:	f44f 7460 	mov.w	r4, #896	; 0x380
 80004c8:	f001 4500 	and.w	r5, r1, #2147483648	; 0x80000000
 80004cc:	f021 4100 	bic.w	r1, r1, #2147483648	; 0x80000000
 80004d0:	e71c      	b.n	800030c <__adddf3+0x138>
 80004d2:	bf00      	nop

080004d4 <__aeabi_ul2d>:
 80004d4:	ea50 0201 	orrs.w	r2, r0, r1
 80004d8:	bf08      	it	eq
 80004da:	4770      	bxeq	lr
 80004dc:	b530      	push	{r4, r5, lr}
 80004de:	f04f 0500 	mov.w	r5, #0
 80004e2:	e00a      	b.n	80004fa <__aeabi_l2d+0x16>

080004e4 <__aeabi_l2d>:
 80004e4:	ea50 0201 	orrs.w	r2, r0, r1
 80004e8:	bf08      	it	eq
 80004ea:	4770      	bxeq	lr
 80004ec:	b530      	push	{r4, r5, lr}
 80004ee:	f011 4500 	ands.w	r5, r1, #2147483648	; 0x80000000
 80004f2:	d502      	bpl.n	80004fa <__aeabi_l2d+0x16>
 80004f4:	4240      	negs	r0, r0
 80004f6:	eb61 0141 	sbc.w	r1, r1, r1, lsl #1
 80004fa:	f44f 6480 	mov.w	r4, #1024	; 0x400
 80004fe:	f104 0432 	add.w	r4, r4, #50	; 0x32
 8000502:	ea5f 5c91 	movs.w	ip, r1, lsr #22
 8000506:	f43f aed8 	beq.w	80002ba <__adddf3+0xe6>
 800050a:	f04f 0203 	mov.w	r2, #3
 800050e:	ea5f 0cdc 	movs.w	ip, ip, lsr #3
 8000512:	bf18      	it	ne
 8000514:	3203      	addne	r2, #3
 8000516:	ea5f 0cdc 	movs.w	ip, ip, lsr #3
 800051a:	bf18      	it	ne
 800051c:	3203      	addne	r2, #3
 800051e:	eb02 02dc 	add.w	r2, r2, ip, lsr #3
 8000522:	f1c2 0320 	rsb	r3, r2, #32
 8000526:	fa00 fc03 	lsl.w	ip, r0, r3
 800052a:	fa20 f002 	lsr.w	r0, r0, r2
 800052e:	fa01 fe03 	lsl.w	lr, r1, r3
 8000532:	ea40 000e 	orr.w	r0, r0, lr
 8000536:	fa21 f102 	lsr.w	r1, r1, r2
 800053a:	4414      	add	r4, r2
 800053c:	e6bd      	b.n	80002ba <__adddf3+0xe6>
 800053e:	bf00      	nop

08000540 <__aeabi_dmul>:
 8000540:	b570      	push	{r4, r5, r6, lr}
 8000542:	f04f 0cff 	mov.w	ip, #255	; 0xff
 8000546:	f44c 6ce0 	orr.w	ip, ip, #1792	; 0x700
 800054a:	ea1c 5411 	ands.w	r4, ip, r1, lsr #20
 800054e:	bf1d      	ittte	ne
 8000550:	ea1c 5513 	andsne.w	r5, ip, r3, lsr #20
 8000554:	ea94 0f0c 	teqne	r4, ip
 8000558:	ea95 0f0c 	teqne	r5, ip
 800055c:	f000 f8de 	bleq	800071c <__aeabi_dmul+0x1dc>
 8000560:	442c      	add	r4, r5
 8000562:	ea81 0603 	eor.w	r6, r1, r3
 8000566:	ea21 514c 	bic.w	r1, r1, ip, lsl #21
 800056a:	ea23 534c 	bic.w	r3, r3, ip, lsl #21
 800056e:	ea50 3501 	orrs.w	r5, r0, r1, lsl #12
 8000572:	bf18      	it	ne
 8000574:	ea52 3503 	orrsne.w	r5, r2, r3, lsl #12
 8000578:	f441 1180 	orr.w	r1, r1, #1048576	; 0x100000
 800057c:	f443 1380 	orr.w	r3, r3, #1048576	; 0x100000
 8000580:	d038      	beq.n	80005f4 <__aeabi_dmul+0xb4>
 8000582:	fba0 ce02 	umull	ip, lr, r0, r2
 8000586:	f04f 0500 	mov.w	r5, #0
 800058a:	fbe1 e502 	umlal	lr, r5, r1, r2
 800058e:	f006 4200 	and.w	r2, r6, #2147483648	; 0x80000000
 8000592:	fbe0 e503 	umlal	lr, r5, r0, r3
 8000596:	f04f 0600 	mov.w	r6, #0
 800059a:	fbe1 5603 	umlal	r5, r6, r1, r3
 800059e:	f09c 0f00 	teq	ip, #0
 80005a2:	bf18      	it	ne
 80005a4:	f04e 0e01 	orrne.w	lr, lr, #1
 80005a8:	f1a4 04ff 	sub.w	r4, r4, #255	; 0xff
 80005ac:	f5b6 7f00 	cmp.w	r6, #512	; 0x200
 80005b0:	f564 7440 	sbc.w	r4, r4, #768	; 0x300
 80005b4:	d204      	bcs.n	80005c0 <__aeabi_dmul+0x80>
 80005b6:	ea5f 0e4e 	movs.w	lr, lr, lsl #1
 80005ba:	416d      	adcs	r5, r5
 80005bc:	eb46 0606 	adc.w	r6, r6, r6
 80005c0:	ea42 21c6 	orr.w	r1, r2, r6, lsl #11
 80005c4:	ea41 5155 	orr.w	r1, r1, r5, lsr #21
 80005c8:	ea4f 20c5 	mov.w	r0, r5, lsl #11
 80005cc:	ea40 505e 	orr.w	r0, r0, lr, lsr #21
 80005d0:	ea4f 2ece 	mov.w	lr, lr, lsl #11
 80005d4:	f1b4 0cfd 	subs.w	ip, r4, #253	; 0xfd
 80005d8:	bf88      	it	hi
 80005da:	f5bc 6fe0 	cmphi.w	ip, #1792	; 0x700
 80005de:	d81e      	bhi.n	800061e <__aeabi_dmul+0xde>
 80005e0:	f1be 4f00 	cmp.w	lr, #2147483648	; 0x80000000
 80005e4:	bf08      	it	eq
 80005e6:	ea5f 0e50 	movseq.w	lr, r0, lsr #1
 80005ea:	f150 0000 	adcs.w	r0, r0, #0
 80005ee:	eb41 5104 	adc.w	r1, r1, r4, lsl #20
 80005f2:	bd70      	pop	{r4, r5, r6, pc}
 80005f4:	f006 4600 	and.w	r6, r6, #2147483648	; 0x80000000
 80005f8:	ea46 0101 	orr.w	r1, r6, r1
 80005fc:	ea40 0002 	orr.w	r0, r0, r2
 8000600:	ea81 0103 	eor.w	r1, r1, r3
 8000604:	ebb4 045c 	subs.w	r4, r4, ip, lsr #1
 8000608:	bfc2      	ittt	gt
 800060a:	ebd4 050c 	rsbsgt	r5, r4, ip
 800060e:	ea41 5104 	orrgt.w	r1, r1, r4, lsl #20
 8000612:	bd70      	popgt	{r4, r5, r6, pc}
 8000614:	f441 1180 	orr.w	r1, r1, #1048576	; 0x100000
 8000618:	f04f 0e00 	mov.w	lr, #0
 800061c:	3c01      	subs	r4, #1
 800061e:	f300 80ab 	bgt.w	8000778 <__aeabi_dmul+0x238>
 8000622:	f114 0f36 	cmn.w	r4, #54	; 0x36
 8000626:	bfde      	ittt	le
 8000628:	2000      	movle	r0, #0
 800062a:	f001 4100 	andle.w	r1, r1, #2147483648	; 0x80000000
 800062e:	bd70      	pople	{r4, r5, r6, pc}
 8000630:	f1c4 0400 	rsb	r4, r4, #0
 8000634:	3c20      	subs	r4, #32
 8000636:	da35      	bge.n	80006a4 <__aeabi_dmul+0x164>
 8000638:	340c      	adds	r4, #12
 800063a:	dc1b      	bgt.n	8000674 <__aeabi_dmul+0x134>
 800063c:	f104 0414 	add.w	r4, r4, #20
 8000640:	f1c4 0520 	rsb	r5, r4, #32
 8000644:	fa00 f305 	lsl.w	r3, r0, r5
 8000648:	fa20 f004 	lsr.w	r0, r0, r4
 800064c:	fa01 f205 	lsl.w	r2, r1, r5
 8000650:	ea40 0002 	orr.w	r0, r0, r2
 8000654:	f001 4200 	and.w	r2, r1, #2147483648	; 0x80000000
 8000658:	f021 4100 	bic.w	r1, r1, #2147483648	; 0x80000000
 800065c:	eb10 70d3 	adds.w	r0, r0, r3, lsr #31
 8000660:	fa21 f604 	lsr.w	r6, r1, r4
 8000664:	eb42 0106 	adc.w	r1, r2, r6
 8000668:	ea5e 0e43 	orrs.w	lr, lr, r3, lsl #1
 800066c:	bf08      	it	eq
 800066e:	ea20 70d3 	biceq.w	r0, r0, r3, lsr #31
 8000672:	bd70      	pop	{r4, r5, r6, pc}
 8000674:	f1c4 040c 	rsb	r4, r4, #12
 8000678:	f1c4 0520 	rsb	r5, r4, #32
 800067c:	fa00 f304 	lsl.w	r3, r0, r4
 8000680:	fa20 f005 	lsr.w	r0, r0, r5
 8000684:	fa01 f204 	lsl.w	r2, r1, r4
 8000688:	ea40 0002 	orr.w	r0, r0, r2
 800068c:	f001 4100 	and.w	r1, r1, #2147483648	; 0x80000000
 8000690:	eb10 70d3 	adds.w	r0, r0, r3, lsr #31
 8000694:	f141 0100 	adc.w	r1, r1, #0
 8000698:	ea5e 0e43 	orrs.w	lr, lr, r3, lsl #1
 800069c:	bf08      	it	eq
 800069e:	ea20 70d3 	biceq.w	r0, r0, r3, lsr #31
 80006a2:	bd70      	pop	{r4, r5, r6, pc}
 80006a4:	f1c4 0520 	rsb	r5, r4, #32
 80006a8:	fa00 f205 	lsl.w	r2, r0, r5
 80006ac:	ea4e 0e02 	orr.w	lr, lr, r2
 80006b0:	fa20 f304 	lsr.w	r3, r0, r4
 80006b4:	fa01 f205 	lsl.w	r2, r1, r5
 80006b8:	ea43 0302 	orr.w	r3, r3, r2
 80006bc:	fa21 f004 	lsr.w	r0, r1, r4
 80006c0:	f001 4100 	and.w	r1, r1, #2147483648	; 0x80000000
 80006c4:	fa21 f204 	lsr.w	r2, r1, r4
 80006c8:	ea20 0002 	bic.w	r0, r0, r2
 80006cc:	eb00 70d3 	add.w	r0, r0, r3, lsr #31
 80006d0:	ea5e 0e43 	orrs.w	lr, lr, r3, lsl #1
 80006d4:	bf08      	it	eq
 80006d6:	ea20 70d3 	biceq.w	r0, r0, r3, lsr #31
 80006da:	bd70      	pop	{r4, r5, r6, pc}
 80006dc:	f094 0f00 	teq	r4, #0
 80006e0:	d10f      	bne.n	8000702 <__aeabi_dmul+0x1c2>
 80006e2:	f001 4600 	and.w	r6, r1, #2147483648	; 0x80000000
 80006e6:	0040      	lsls	r0, r0, #1
 80006e8:	eb41 0101 	adc.w	r1, r1, r1
 80006ec:	f411 1f80 	tst.w	r1, #1048576	; 0x100000
 80006f0:	bf08      	it	eq
 80006f2:	3c01      	subeq	r4, #1
 80006f4:	d0f7      	beq.n	80006e6 <__aeabi_dmul+0x1a6>
 80006f6:	ea41 0106 	orr.w	r1, r1, r6
 80006fa:	f095 0f00 	teq	r5, #0
 80006fe:	bf18      	it	ne
 8000700:	4770      	bxne	lr
 8000702:	f003 4600 	and.w	r6, r3, #2147483648	; 0x80000000
 8000706:	0052      	lsls	r2, r2, #1
 8000708:	eb43 0303 	adc.w	r3, r3, r3
 800070c:	f413 1f80 	tst.w	r3, #1048576	; 0x100000
 8000710:	bf08      	it	eq
 8000712:	3d01      	subeq	r5, #1
 8000714:	d0f7      	beq.n	8000706 <__aeabi_dmul+0x1c6>
 8000716:	ea43 0306 	orr.w	r3, r3, r6
 800071a:	4770      	bx	lr
 800071c:	ea94 0f0c 	teq	r4, ip
 8000720:	ea0c 5513 	and.w	r5, ip, r3, lsr #20
 8000724:	bf18      	it	ne
 8000726:	ea95 0f0c 	teqne	r5, ip
 800072a:	d00c      	beq.n	8000746 <__aeabi_dmul+0x206>
 800072c:	ea50 0641 	orrs.w	r6, r0, r1, lsl #1
 8000730:	bf18      	it	ne
 8000732:	ea52 0643 	orrsne.w	r6, r2, r3, lsl #1
 8000736:	d1d1      	bne.n	80006dc <__aeabi_dmul+0x19c>
 8000738:	ea81 0103 	eor.w	r1, r1, r3
 800073c:	f001 4100 	and.w	r1, r1, #2147483648	; 0x80000000
 8000740:	f04f 0000 	mov.w	r0, #0
 8000744:	bd70      	pop	{r4, r5, r6, pc}
 8000746:	ea50 0641 	orrs.w	r6, r0, r1, lsl #1
 800074a:	bf06      	itte	eq
 800074c:	4610      	moveq	r0, r2
 800074e:	4619      	moveq	r1, r3
 8000750:	ea52 0643 	orrsne.w	r6, r2, r3, lsl #1
 8000754:	d019      	beq.n	800078a <__aeabi_dmul+0x24a>
 8000756:	ea94 0f0c 	teq	r4, ip
 800075a:	d102      	bne.n	8000762 <__aeabi_dmul+0x222>
 800075c:	ea50 3601 	orrs.w	r6, r0, r1, lsl #12
 8000760:	d113      	bne.n	800078a <__aeabi_dmul+0x24a>
 8000762:	ea95 0f0c 	teq	r5, ip
 8000766:	d105      	bne.n	8000774 <__aeabi_dmul+0x234>
 8000768:	ea52 3603 	orrs.w	r6, r2, r3, lsl #12
 800076c:	bf1c      	itt	ne
 800076e:	4610      	movne	r0, r2
 8000770:	4619      	movne	r1, r3
 8000772:	d10a      	bne.n	800078a <__aeabi_dmul+0x24a>
 8000774:	ea81 0103 	eor.w	r1, r1, r3
 8000778:	f001 4100 	and.w	r1, r1, #2147483648	; 0x80000000
 800077c:	f041 41fe 	orr.w	r1, r1, #2130706432	; 0x7f000000
 8000780:	f441 0170 	orr.w	r1, r1, #15728640	; 0xf00000
 8000784:	f04f 0000 	mov.w	r0, #0
 8000788:	bd70      	pop	{r4, r5, r6, pc}
 800078a:	f041 41fe 	orr.w	r1, r1, #2130706432	; 0x7f000000
 800078e:	f441 0178 	orr.w	r1, r1, #16252928	; 0xf80000
 8000792:	bd70      	pop	{r4, r5, r6, pc}

08000794 <__aeabi_ddiv>:
 8000794:	b570      	push	{r4, r5, r6, lr}
 8000796:	f04f 0cff 	mov.w	ip, #255	; 0xff
 800079a:	f44c 6ce0 	orr.w	ip, ip, #1792	; 0x700
 800079e:	ea1c 5411 	ands.w	r4, ip, r1, lsr #20
 80007a2:	bf1d      	ittte	ne
 80007a4:	ea1c 5513 	andsne.w	r5, ip, r3, lsr #20
 80007a8:	ea94 0f0c 	teqne	r4, ip
 80007ac:	ea95 0f0c 	teqne	r5, ip
 80007b0:	f000 f8a7 	bleq	8000902 <__aeabi_ddiv+0x16e>
 80007b4:	eba4 0405 	sub.w	r4, r4, r5
 80007b8:	ea81 0e03 	eor.w	lr, r1, r3
 80007bc:	ea52 3503 	orrs.w	r5, r2, r3, lsl #12
 80007c0:	ea4f 3101 	mov.w	r1, r1, lsl #12
 80007c4:	f000 8088 	beq.w	80008d8 <__aeabi_ddiv+0x144>
 80007c8:	ea4f 3303 	mov.w	r3, r3, lsl #12
 80007cc:	f04f 5580 	mov.w	r5, #268435456	; 0x10000000
 80007d0:	ea45 1313 	orr.w	r3, r5, r3, lsr #4
 80007d4:	ea43 6312 	orr.w	r3, r3, r2, lsr #24
 80007d8:	ea4f 2202 	mov.w	r2, r2, lsl #8
 80007dc:	ea45 1511 	orr.w	r5, r5, r1, lsr #4
 80007e0:	ea45 6510 	orr.w	r5, r5, r0, lsr #24
 80007e4:	ea4f 2600 	mov.w	r6, r0, lsl #8
 80007e8:	f00e 4100 	and.w	r1, lr, #2147483648	; 0x80000000
 80007ec:	429d      	cmp	r5, r3
 80007ee:	bf08      	it	eq
 80007f0:	4296      	cmpeq	r6, r2
 80007f2:	f144 04fd 	adc.w	r4, r4, #253	; 0xfd
 80007f6:	f504 7440 	add.w	r4, r4, #768	; 0x300
 80007fa:	d202      	bcs.n	8000802 <__aeabi_ddiv+0x6e>
 80007fc:	085b      	lsrs	r3, r3, #1
 80007fe:	ea4f 0232 	mov.w	r2, r2, rrx
 8000802:	1ab6      	subs	r6, r6, r2
 8000804:	eb65 0503 	sbc.w	r5, r5, r3
 8000808:	085b      	lsrs	r3, r3, #1
 800080a:	ea4f 0232 	mov.w	r2, r2, rrx
 800080e:	f44f 1080 	mov.w	r0, #1048576	; 0x100000
 8000812:	f44f 2c00 	mov.w	ip, #524288	; 0x80000
 8000816:	ebb6 0e02 	subs.w	lr, r6, r2
 800081a:	eb75 0e03 	sbcs.w	lr, r5, r3
 800081e:	bf22      	ittt	cs
 8000820:	1ab6      	subcs	r6, r6, r2
 8000822:	4675      	movcs	r5, lr
 8000824:	ea40 000c 	orrcs.w	r0, r0, ip
 8000828:	085b      	lsrs	r3, r3, #1
 800082a:	ea4f 0232 	mov.w	r2, r2, rrx
 800082e:	ebb6 0e02 	subs.w	lr, r6, r2
 8000832:	eb75 0e03 	sbcs.w	lr, r5, r3
 8000836:	bf22      	ittt	cs
 8000838:	1ab6      	subcs	r6, r6, r2
 800083a:	4675      	movcs	r5, lr
 800083c:	ea40 005c 	orrcs.w	r0, r0, ip, lsr #1
 8000840:	085b      	lsrs	r3, r3, #1
 8000842:	ea4f 0232 	mov.w	r2, r2, rrx
 8000846:	ebb6 0e02 	subs.w	lr, r6, r2
 800084a:	eb75 0e03 	sbcs.w	lr, r5, r3
 800084e:	bf22      	ittt	cs
 8000850:	1ab6      	subcs	r6, r6, r2
 8000852:	4675      	movcs	r5, lr
 8000854:	ea40 009c 	orrcs.w	r0, r0, ip, lsr #2
 8000858:	085b      	lsrs	r3, r3, #1
 800085a:	ea4f 0232 	mov.w	r2, r2, rrx
 800085e:	ebb6 0e02 	subs.w	lr, r6, r2
 8000862:	eb75 0e03 	sbcs.w	lr, r5, r3
 8000866:	bf22      	ittt	cs
 8000868:	1ab6      	subcs	r6, r6, r2
 800086a:	4675      	movcs	r5, lr
 800086c:	ea40 00dc 	orrcs.w	r0, r0, ip, lsr #3
 8000870:	ea55 0e06 	orrs.w	lr, r5, r6
 8000874:	d018      	beq.n	80008a8 <__aeabi_ddiv+0x114>
 8000876:	ea4f 1505 	mov.w	r5, r5, lsl #4
 800087a:	ea45 7516 	orr.w	r5, r5, r6, lsr #28
 800087e:	ea4f 1606 	mov.w	r6, r6, lsl #4
 8000882:	ea4f 03c3 	mov.w	r3, r3, lsl #3
 8000886:	ea43 7352 	orr.w	r3, r3, r2, lsr #29
 800088a:	ea4f 02c2 	mov.w	r2, r2, lsl #3
 800088e:	ea5f 1c1c 	movs.w	ip, ip, lsr #4
 8000892:	d1c0      	bne.n	8000816 <__aeabi_ddiv+0x82>
 8000894:	f411 1f80 	tst.w	r1, #1048576	; 0x100000
 8000898:	d10b      	bne.n	80008b2 <__aeabi_ddiv+0x11e>
 800089a:	ea41 0100 	orr.w	r1, r1, r0
 800089e:	f04f 0000 	mov.w	r0, #0
 80008a2:	f04f 4c00 	mov.w	ip, #2147483648	; 0x80000000
 80008a6:	e7b6      	b.n	8000816 <__aeabi_ddiv+0x82>
 80008a8:	f411 1f80 	tst.w	r1, #1048576	; 0x100000
 80008ac:	bf04      	itt	eq
 80008ae:	4301      	orreq	r1, r0
 80008b0:	2000      	moveq	r0, #0
 80008b2:	f1b4 0cfd 	subs.w	ip, r4, #253	; 0xfd
 80008b6:	bf88      	it	hi
 80008b8:	f5bc 6fe0 	cmphi.w	ip, #1792	; 0x700
 80008bc:	f63f aeaf 	bhi.w	800061e <__aeabi_dmul+0xde>
 80008c0:	ebb5 0c03 	subs.w	ip, r5, r3
 80008c4:	bf04      	itt	eq
 80008c6:	ebb6 0c02 	subseq.w	ip, r6, r2
 80008ca:	ea5f 0c50 	movseq.w	ip, r0, lsr #1
 80008ce:	f150 0000 	adcs.w	r0, r0, #0
 80008d2:	eb41 5104 	adc.w	r1, r1, r4, lsl #20
 80008d6:	bd70      	pop	{r4, r5, r6, pc}
 80008d8:	f00e 4e00 	and.w	lr, lr, #2147483648	; 0x80000000
 80008dc:	ea4e 3111 	orr.w	r1, lr, r1, lsr #12
 80008e0:	eb14 045c 	adds.w	r4, r4, ip, lsr #1
 80008e4:	bfc2      	ittt	gt
 80008e6:	ebd4 050c 	rsbsgt	r5, r4, ip
 80008ea:	ea41 5104 	orrgt.w	r1, r1, r4, lsl #20
 80008ee:	bd70      	popgt	{r4, r5, r6, pc}
 80008f0:	f441 1180 	orr.w	r1, r1, #1048576	; 0x100000
 80008f4:	f04f 0e00 	mov.w	lr, #0
 80008f8:	3c01      	subs	r4, #1
 80008fa:	e690      	b.n	800061e <__aeabi_dmul+0xde>
 80008fc:	ea45 0e06 	orr.w	lr, r5, r6
 8000900:	e68d      	b.n	800061e <__aeabi_dmul+0xde>
 8000902:	ea0c 5513 	and.w	r5, ip, r3, lsr #20
 8000906:	ea94 0f0c 	teq	r4, ip
 800090a:	bf08      	it	eq
 800090c:	ea95 0f0c 	teqeq	r5, ip
 8000910:	f43f af3b 	beq.w	800078a <__aeabi_dmul+0x24a>
 8000914:	ea94 0f0c 	teq	r4, ip
 8000918:	d10a      	bne.n	8000930 <__aeabi_ddiv+0x19c>
 800091a:	ea50 3401 	orrs.w	r4, r0, r1, lsl #12
 800091e:	f47f af34 	bne.w	800078a <__aeabi_dmul+0x24a>
 8000922:	ea95 0f0c 	teq	r5, ip
 8000926:	f47f af25 	bne.w	8000774 <__aeabi_dmul+0x234>
 800092a:	4610      	mov	r0, r2
 800092c:	4619      	mov	r1, r3
 800092e:	e72c      	b.n	800078a <__aeabi_dmul+0x24a>
 8000930:	ea95 0f0c 	teq	r5, ip
 8000934:	d106      	bne.n	8000944 <__aeabi_ddiv+0x1b0>
 8000936:	ea52 3503 	orrs.w	r5, r2, r3, lsl #12
 800093a:	f43f aefd 	beq.w	8000738 <__aeabi_dmul+0x1f8>
 800093e:	4610      	mov	r0, r2
 8000940:	4619      	mov	r1, r3
 8000942:	e722      	b.n	800078a <__aeabi_dmul+0x24a>
 8000944:	ea50 0641 	orrs.w	r6, r0, r1, lsl #1
 8000948:	bf18      	it	ne
 800094a:	ea52 0643 	orrsne.w	r6, r2, r3, lsl #1
 800094e:	f47f aec5 	bne.w	80006dc <__aeabi_dmul+0x19c>
 8000952:	ea50 0441 	orrs.w	r4, r0, r1, lsl #1
 8000956:	f47f af0d 	bne.w	8000774 <__aeabi_dmul+0x234>
 800095a:	ea52 0543 	orrs.w	r5, r2, r3, lsl #1
 800095e:	f47f aeeb 	bne.w	8000738 <__aeabi_dmul+0x1f8>
 8000962:	e712      	b.n	800078a <__aeabi_dmul+0x24a>

08000964 <__aeabi_d2f>:
 8000964:	ea4f 0241 	mov.w	r2, r1, lsl #1
 8000968:	f1b2 43e0 	subs.w	r3, r2, #1879048192	; 0x70000000
 800096c:	bf24      	itt	cs
 800096e:	f5b3 1c00 	subscs.w	ip, r3, #2097152	; 0x200000
 8000972:	f1dc 5cfe 	rsbscs	ip, ip, #532676608	; 0x1fc00000
 8000976:	d90d      	bls.n	8000994 <__aeabi_d2f+0x30>
 8000978:	f001 4c00 	and.w	ip, r1, #2147483648	; 0x80000000
 800097c:	ea4f 02c0 	mov.w	r2, r0, lsl #3
 8000980:	ea4c 7050 	orr.w	r0, ip, r0, lsr #29
 8000984:	f1b2 4f00 	cmp.w	r2, #2147483648	; 0x80000000
 8000988:	eb40 0083 	adc.w	r0, r0, r3, lsl #2
 800098c:	bf08      	it	eq
 800098e:	f020 0001 	biceq.w	r0, r0, #1
 8000992:	4770      	bx	lr
 8000994:	f011 4f80 	tst.w	r1, #1073741824	; 0x40000000
 8000998:	d121      	bne.n	80009de <__aeabi_d2f+0x7a>
 800099a:	f113 7238 	adds.w	r2, r3, #48234496	; 0x2e00000
 800099e:	bfbc      	itt	lt
 80009a0:	f001 4000 	andlt.w	r0, r1, #2147483648	; 0x80000000
 80009a4:	4770      	bxlt	lr
 80009a6:	f441 1180 	orr.w	r1, r1, #1048576	; 0x100000
 80009aa:	ea4f 5252 	mov.w	r2, r2, lsr #21
 80009ae:	f1c2 0218 	rsb	r2, r2, #24
 80009b2:	f1c2 0c20 	rsb	ip, r2, #32
 80009b6:	fa10 f30c 	lsls.w	r3, r0, ip
 80009ba:	fa20 f002 	lsr.w	r0, r0, r2
 80009be:	bf18      	it	ne
 80009c0:	f040 0001 	orrne.w	r0, r0, #1
 80009c4:	ea4f 23c1 	mov.w	r3, r1, lsl #11
 80009c8:	ea4f 23d3 	mov.w	r3, r3, lsr #11
 80009cc:	fa03 fc0c 	lsl.w	ip, r3, ip
 80009d0:	ea40 000c 	orr.w	r0, r0, ip
 80009d4:	fa23 f302 	lsr.w	r3, r3, r2
 80009d8:	ea4f 0343 	mov.w	r3, r3, lsl #1
 80009dc:	e7cc      	b.n	8000978 <__aeabi_d2f+0x14>
 80009de:	ea7f 5362 	mvns.w	r3, r2, asr #21
 80009e2:	d107      	bne.n	80009f4 <__aeabi_d2f+0x90>
 80009e4:	ea50 3301 	orrs.w	r3, r0, r1, lsl #12
 80009e8:	bf1e      	ittt	ne
 80009ea:	f04f 40fe 	movne.w	r0, #2130706432	; 0x7f000000
 80009ee:	f440 0040 	orrne.w	r0, r0, #12582912	; 0xc00000
 80009f2:	4770      	bxne	lr
 80009f4:	f001 4000 	and.w	r0, r1, #2147483648	; 0x80000000
 80009f8:	f040 40fe 	orr.w	r0, r0, #2130706432	; 0x7f000000
 80009fc:	f440 0000 	orr.w	r0, r0, #8388608	; 0x800000
 8000a00:	4770      	bx	lr
 8000a02:	bf00      	nop

08000a04 <_ZN13FastMathClassC1Ev>:
#ifdef __cplusplus
extern "C" {
#endif

/* Used to calculate the trigonometric function from a lookUp table */
class FastMathClass
 8000a04:	b580      	push	{r7, lr}
 8000a06:	b082      	sub	sp, #8
 8000a08:	af00      	add	r7, sp, #0
 8000a0a:	6078      	str	r0, [r7, #4]
 8000a0c:	687b      	ldr	r3, [r7, #4]
 8000a0e:	4a06      	ldr	r2, [pc, #24]	; (8000a28 <_ZN13FastMathClassC1Ev+0x24>)
 8000a10:	4618      	mov	r0, r3
 8000a12:	4611      	mov	r1, r2
 8000a14:	235b      	movs	r3, #91	; 0x5b
 8000a16:	461a      	mov	r2, r3
 8000a18:	f005 ff7e 	bl	8006918 <memcpy>
 8000a1c:	687b      	ldr	r3, [r7, #4]
 8000a1e:	4618      	mov	r0, r3
 8000a20:	3708      	adds	r7, #8
 8000a22:	46bd      	mov	sp, r7
 8000a24:	bd80      	pop	{r7, pc}
 8000a26:	bf00      	nop
 8000a28:	08006958 	.word	0x08006958

08000a2c <_ZN7DisplayC1Ev>:
/*!
   @brief    Constructor for Display Object
   @param    None
 */
/**************************************************************************/
Display::Display(void) { }
 8000a2c:	b580      	push	{r7, lr}
 8000a2e:	b082      	sub	sp, #8
 8000a30:	af00      	add	r7, sp, #0
 8000a32:	6078      	str	r0, [r7, #4]
 8000a34:	687b      	ldr	r3, [r7, #4]
 8000a36:	4618      	mov	r0, r3
 8000a38:	f7ff ffe4 	bl	8000a04 <_ZN13FastMathClassC1Ev>
 8000a3c:	687b      	ldr	r3, [r7, #4]
 8000a3e:	4618      	mov	r0, r3
 8000a40:	3708      	adds	r7, #8
 8000a42:	46bd      	mov	sp, r7
 8000a44:	bd80      	pop	{r7, pc}
	...

08000a48 <_ZN7Display11initDisplayEv>:
   @brief    Initialize the base parameters of the display variables here
   @param    None
 */
/**************************************************************************/
void Display::initDisplay(void)
{
 8000a48:	b580      	push	{r7, lr}
 8000a4a:	b082      	sub	sp, #8
 8000a4c:	af00      	add	r7, sp, #0
 8000a4e:	6078      	str	r0, [r7, #4]
    g_Graphics.initGraphics();
 8000a50:	4814      	ldr	r0, [pc, #80]	; (8000aa4 <_ZN7Display11initDisplayEv+0x5c>)
 8000a52:	f000 ff11 	bl	8001878 <_ZN8Graphics12initGraphicsEv>
    resolution.width = SCREENDIMENSIONSWIDTH;/* number of width bits */
 8000a56:	687b      	ldr	r3, [r7, #4]
 8000a58:	22f0      	movs	r2, #240	; 0xf0
 8000a5a:	f8a3 205c 	strh.w	r2, [r3, #92]	; 0x5c
    resolution.height = SCREENDIMENSIONSHEIGHT;/* number of height bits */
 8000a5e:	687b      	ldr	r3, [r7, #4]
 8000a60:	f240 122f 	movw	r2, #303	; 0x12f
 8000a64:	f8a3 205e 	strh.w	r2, [r3, #94]	; 0x5e
    fontWidth = g_Graphics.getFontYAdvance();/* Widest character spacing */
 8000a68:	480e      	ldr	r0, [pc, #56]	; (8000aa4 <_ZN7Display11initDisplayEv+0x5c>)
 8000a6a:	f001 f9f5 	bl	8001e58 <_ZN8Graphics15getFontYAdvanceEv>
 8000a6e:	4603      	mov	r3, r0
 8000a70:	461a      	mov	r2, r3
 8000a72:	687b      	ldr	r3, [r7, #4]
 8000a74:	f883 2068 	strb.w	r2, [r3, #104]	; 0x68
    fontHeight = g_Graphics.getFontXAdvance();/* Tallest character spacing */
 8000a78:	480a      	ldr	r0, [pc, #40]	; (8000aa4 <_ZN7Display11initDisplayEv+0x5c>)
 8000a7a:	f001 f9cb 	bl	8001e14 <_ZN8Graphics15getFontXAdvanceEv>
 8000a7e:	4603      	mov	r3, r0
 8000a80:	461a      	mov	r2, r3
 8000a82:	687b      	ldr	r3, [r7, #4]
 8000a84:	f883 2069 	strb.w	r2, [r3, #105]	; 0x69
    setCursorOffset(0,0);
 8000a88:	2200      	movs	r2, #0
 8000a8a:	2100      	movs	r1, #0
 8000a8c:	6878      	ldr	r0, [r7, #4]
 8000a8e:	f000 f80b 	bl	8000aa8 <_ZN7Display15setCursorOffsetEtt>
    setLineNum(1);
 8000a92:	2101      	movs	r1, #1
 8000a94:	6878      	ldr	r0, [r7, #4]
 8000a96:	f000 f81d 	bl	8000ad4 <_ZN7Display10setLineNumEh>
}
 8000a9a:	bf00      	nop
 8000a9c:	3708      	adds	r7, #8
 8000a9e:	46bd      	mov	sp, r7
 8000aa0:	bd80      	pop	{r7, pc}
 8000aa2:	bf00      	nop
 8000aa4:	200000a8 	.word	0x200000a8

08000aa8 <_ZN7Display15setCursorOffsetEtt>:
   NOTE: m_cursorOffsetX and m_cursorOffsetY are used right now for centerTextCust() which is set to the center, You may need to also check setCursor() in
   the graphics module and adjust that as well.
 */
/**************************************************************************/
void Display::setCursorOffset(uint16_t x, uint16_t y)
{
 8000aa8:	b480      	push	{r7}
 8000aaa:	b083      	sub	sp, #12
 8000aac:	af00      	add	r7, sp, #0
 8000aae:	6078      	str	r0, [r7, #4]
 8000ab0:	460b      	mov	r3, r1
 8000ab2:	807b      	strh	r3, [r7, #2]
 8000ab4:	4613      	mov	r3, r2
 8000ab6:	803b      	strh	r3, [r7, #0]
    m_cursorOffsetX = x;
 8000ab8:	687b      	ldr	r3, [r7, #4]
 8000aba:	887a      	ldrh	r2, [r7, #2]
 8000abc:	f8a3 206c 	strh.w	r2, [r3, #108]	; 0x6c
    m_cursorOffsetY = y;
 8000ac0:	687b      	ldr	r3, [r7, #4]
 8000ac2:	883a      	ldrh	r2, [r7, #0]
 8000ac4:	f8a3 206e 	strh.w	r2, [r3, #110]	; 0x6e
}
 8000ac8:	bf00      	nop
 8000aca:	370c      	adds	r7, #12
 8000acc:	46bd      	mov	sp, r7
 8000ace:	f85d 7b04 	ldr.w	r7, [sp], #4
 8000ad2:	4770      	bx	lr

08000ad4 <_ZN7Display10setLineNumEh>:
   NOTE: m_lineNum is used to give spacing between the text when the next text is on another line. this way they do not collide with each other if you are
   sing different font sizes.
 */
/**************************************************************************/
void Display::setLineNum(uint8_t lineNum)
{
 8000ad4:	b480      	push	{r7}
 8000ad6:	b083      	sub	sp, #12
 8000ad8:	af00      	add	r7, sp, #0
 8000ada:	6078      	str	r0, [r7, #4]
 8000adc:	460b      	mov	r3, r1
 8000ade:	70fb      	strb	r3, [r7, #3]
    m_lineNum = lineNum;
 8000ae0:	687b      	ldr	r3, [r7, #4]
 8000ae2:	78fa      	ldrb	r2, [r7, #3]
 8000ae4:	f883 206a 	strb.w	r2, [r3, #106]	; 0x6a
}
 8000ae8:	bf00      	nop
 8000aea:	370c      	adds	r7, #12
 8000aec:	46bd      	mov	sp, r7
 8000aee:	f85d 7b04 	ldr.w	r7, [sp], #4
 8000af2:	4770      	bx	lr

08000af4 <_ZN7Display11writeStreamEPKhj>:

   NOTE: ensure the setCursor(x,y) whcih is defined in the graphics module is set where you want it to be before writing
 */
/**************************************************************************/
size_t Display::writeStream(const uint8_t *buffer, size_t size)
{
 8000af4:	b580      	push	{r7, lr}
 8000af6:	b086      	sub	sp, #24
 8000af8:	af00      	add	r7, sp, #0
 8000afa:	60f8      	str	r0, [r7, #12]
 8000afc:	60b9      	str	r1, [r7, #8]
 8000afe:	607a      	str	r2, [r7, #4]
    size_t count = 0;
 8000b00:	2300      	movs	r3, #0
 8000b02:	617b      	str	r3, [r7, #20]
    while (size--)
 8000b04:	687b      	ldr	r3, [r7, #4]
 8000b06:	1e5a      	subs	r2, r3, #1
 8000b08:	607a      	str	r2, [r7, #4]
 8000b0a:	2b00      	cmp	r3, #0
 8000b0c:	bf14      	ite	ne
 8000b0e:	2301      	movne	r3, #1
 8000b10:	2300      	moveq	r3, #0
 8000b12:	b2db      	uxtb	r3, r3
 8000b14:	2b00      	cmp	r3, #0
 8000b16:	d00b      	beq.n	8000b30 <_ZN7Display11writeStreamEPKhj+0x3c>
    {
        count = count + 1;
 8000b18:	697b      	ldr	r3, [r7, #20]
 8000b1a:	3301      	adds	r3, #1
 8000b1c:	617b      	str	r3, [r7, #20]
        g_Graphics.write(*buffer++);
 8000b1e:	68bb      	ldr	r3, [r7, #8]
 8000b20:	1c5a      	adds	r2, r3, #1
 8000b22:	60ba      	str	r2, [r7, #8]
 8000b24:	781b      	ldrb	r3, [r3, #0]
 8000b26:	4619      	mov	r1, r3
 8000b28:	4804      	ldr	r0, [pc, #16]	; (8000b3c <_ZN7Display11writeStreamEPKhj+0x48>)
 8000b2a:	f000 ff81 	bl	8001a30 <_ZN8Graphics5writeEh>
    while (size--)
 8000b2e:	e7e9      	b.n	8000b04 <_ZN7Display11writeStreamEPKhj+0x10>
    }
    return count;
 8000b30:	697b      	ldr	r3, [r7, #20]
}
 8000b32:	4618      	mov	r0, r3
 8000b34:	3718      	adds	r7, #24
 8000b36:	46bd      	mov	sp, r7
 8000b38:	bd80      	pop	{r7, pc}
 8000b3a:	bf00      	nop
 8000b3c:	200000a8 	.word	0x200000a8

08000b40 <_ZN7Display9drawShapeENS_7Shape_tEtPv>:
   NOTE: argp is a void* which means it has to be typecasted to the correct Structure

 */
/**************************************************************************/
void Display::drawShape(Shape_t shape, uint16_t color, void* argp)
{
 8000b40:	b5f0      	push	{r4, r5, r6, r7, lr}
 8000b42:	b0a5      	sub	sp, #148	; 0x94
 8000b44:	af04      	add	r7, sp, #16
 8000b46:	60f8      	str	r0, [r7, #12]
 8000b48:	607b      	str	r3, [r7, #4]
 8000b4a:	460b      	mov	r3, r1
 8000b4c:	72fb      	strb	r3, [r7, #11]
 8000b4e:	4613      	mov	r3, r2
 8000b50:	813b      	strh	r3, [r7, #8]
    switch(shape)
 8000b52:	7afb      	ldrb	r3, [r7, #11]
 8000b54:	2b09      	cmp	r3, #9
 8000b56:	f200 84dc 	bhi.w	8001512 <_ZN7Display9drawShapeENS_7Shape_tEtPv+0x9d2>
 8000b5a:	a201      	add	r2, pc, #4	; (adr r2, 8000b60 <_ZN7Display9drawShapeENS_7Shape_tEtPv+0x20>)
 8000b5c:	f852 f023 	ldr.w	pc, [r2, r3, lsl #2]
 8000b60:	08000b89 	.word	0x08000b89
 8000b64:	08000ba1 	.word	0x08000ba1
 8000b68:	08000bcd 	.word	0x08000bcd
 8000b6c:	08000bef 	.word	0x08000bef
 8000b70:	08000c2d 	.word	0x08000c2d
 8000b74:	08000c59 	.word	0x08000c59
 8000b78:	08000c85 	.word	0x08000c85
 8000b7c:	08000cb9 	.word	0x08000cb9
 8000b80:	08000f35 	.word	0x08000f35
 8000b84:	080012e3 	.word	0x080012e3
    {
    case SHAPE_Point:
    {
        g_Graphics.drawPixel(((ShapePoint_t *)argp)->x,
 8000b88:	687b      	ldr	r3, [r7, #4]
 8000b8a:	f9b3 1000 	ldrsh.w	r1, [r3]
 8000b8e:	687b      	ldr	r3, [r7, #4]
 8000b90:	f9b3 2002 	ldrsh.w	r2, [r3, #2]
 8000b94:	893b      	ldrh	r3, [r7, #8]
 8000b96:	4847      	ldr	r0, [pc, #284]	; (8000cb4 <_ZN7Display9drawShapeENS_7Shape_tEtPv+0x174>)
 8000b98:	f000 fee2 	bl	8001960 <_ZN8Graphics9drawPixelEsst>
                ((ShapePoint_t *)argp)->y,
                color);
        break;
 8000b9c:	f000 bcbe 	b.w	800151c <_ZN7Display9drawShapeENS_7Shape_tEtPv+0x9dc>
    }
    case SHAPE_Line:
    {
        g_Graphics.drawLine(((ShapeLine_t *)argp)->start.x,
 8000ba0:	687b      	ldr	r3, [r7, #4]
 8000ba2:	f9b3 1000 	ldrsh.w	r1, [r3]
 8000ba6:	687b      	ldr	r3, [r7, #4]
 8000ba8:	f9b3 0002 	ldrsh.w	r0, [r3, #2]
 8000bac:	687b      	ldr	r3, [r7, #4]
 8000bae:	f9b3 4004 	ldrsh.w	r4, [r3, #4]
 8000bb2:	687b      	ldr	r3, [r7, #4]
 8000bb4:	f9b3 3006 	ldrsh.w	r3, [r3, #6]
 8000bb8:	893a      	ldrh	r2, [r7, #8]
 8000bba:	9201      	str	r2, [sp, #4]
 8000bbc:	9300      	str	r3, [sp, #0]
 8000bbe:	4623      	mov	r3, r4
 8000bc0:	4602      	mov	r2, r0
 8000bc2:	483c      	ldr	r0, [pc, #240]	; (8000cb4 <_ZN7Display9drawShapeENS_7Shape_tEtPv+0x174>)
 8000bc4:	f001 fb4a 	bl	800225c <_ZN8Graphics8drawLineEsssst>
                ((ShapeLine_t *)argp)->start.y,
                ((ShapeLine_t *)argp)->end.x,
                ((ShapeLine_t *)argp)->end.y,
                color);
        break;
 8000bc8:	f000 bca8 	b.w	800151c <_ZN7Display9drawShapeENS_7Shape_tEtPv+0x9dc>
    }
    case SHAPE_Circle:
    {
        g_Graphics.drawCircle(((ShapeCircle_t *)argp)->center.x,
 8000bcc:	687b      	ldr	r3, [r7, #4]
 8000bce:	f9b3 1000 	ldrsh.w	r1, [r3]
 8000bd2:	687b      	ldr	r3, [r7, #4]
 8000bd4:	f9b3 2002 	ldrsh.w	r2, [r3, #2]
                ((ShapeCircle_t *)argp)->center.y,
                ((ShapeCircle_t *)argp)->radius,
 8000bd8:	687b      	ldr	r3, [r7, #4]
 8000bda:	889b      	ldrh	r3, [r3, #4]
        g_Graphics.drawCircle(((ShapeCircle_t *)argp)->center.x,
 8000bdc:	b218      	sxth	r0, r3
 8000bde:	893b      	ldrh	r3, [r7, #8]
 8000be0:	9300      	str	r3, [sp, #0]
 8000be2:	4603      	mov	r3, r0
 8000be4:	4833      	ldr	r0, [pc, #204]	; (8000cb4 <_ZN7Display9drawShapeENS_7Shape_tEtPv+0x174>)
 8000be6:	f001 f95b 	bl	8001ea0 <_ZN8Graphics10drawCircleEssst>
                color);
        break;
 8000bea:	f000 bc97 	b.w	800151c <_ZN7Display9drawShapeENS_7Shape_tEtPv+0x9dc>
    }
    case SHAPE_Triangle:
    {
        g_Graphics.fillTriangle(((ShapeTriangle_t *)argp)->first.x,
 8000bee:	687b      	ldr	r3, [r7, #4]
 8000bf0:	f9b3 4000 	ldrsh.w	r4, [r3]
 8000bf4:	687b      	ldr	r3, [r7, #4]
 8000bf6:	f9b3 5002 	ldrsh.w	r5, [r3, #2]
 8000bfa:	687b      	ldr	r3, [r7, #4]
 8000bfc:	f9b3 6004 	ldrsh.w	r6, [r3, #4]
 8000c00:	687b      	ldr	r3, [r7, #4]
 8000c02:	f9b3 3006 	ldrsh.w	r3, [r3, #6]
 8000c06:	687a      	ldr	r2, [r7, #4]
 8000c08:	f9b2 2008 	ldrsh.w	r2, [r2, #8]
 8000c0c:	6879      	ldr	r1, [r7, #4]
 8000c0e:	f9b1 100a 	ldrsh.w	r1, [r1, #10]
 8000c12:	8938      	ldrh	r0, [r7, #8]
 8000c14:	9003      	str	r0, [sp, #12]
 8000c16:	9102      	str	r1, [sp, #8]
 8000c18:	9201      	str	r2, [sp, #4]
 8000c1a:	9300      	str	r3, [sp, #0]
 8000c1c:	4633      	mov	r3, r6
 8000c1e:	462a      	mov	r2, r5
 8000c20:	4621      	mov	r1, r4
 8000c22:	4824      	ldr	r0, [pc, #144]	; (8000cb4 <_ZN7Display9drawShapeENS_7Shape_tEtPv+0x174>)
 8000c24:	f001 fce9 	bl	80025fa <_ZN8Graphics12fillTriangleEsssssst>
                ((ShapeTriangle_t *)argp)->second.x,
                ((ShapeTriangle_t *)argp)->second.y,
                ((ShapeTriangle_t *)argp)->third.x,
                ((ShapeTriangle_t *)argp)->third.y,
                color);
        break;
 8000c28:	f000 bc78 	b.w	800151c <_ZN7Display9drawShapeENS_7Shape_tEtPv+0x9dc>
    }
    case SHAPE_Rectangle:
    {
        g_Graphics.drawRect(((ShapeRectangle_t *)argp)->start.x,
 8000c2c:	687b      	ldr	r3, [r7, #4]
 8000c2e:	f9b3 1000 	ldrsh.w	r1, [r3]
 8000c32:	687b      	ldr	r3, [r7, #4]
 8000c34:	f9b3 0002 	ldrsh.w	r0, [r3, #2]
                ((ShapeRectangle_t *)argp)->start.y,
                ((ShapeRectangle_t *)argp)->width,
 8000c38:	687b      	ldr	r3, [r7, #4]
 8000c3a:	889b      	ldrh	r3, [r3, #4]
        g_Graphics.drawRect(((ShapeRectangle_t *)argp)->start.x,
 8000c3c:	b21c      	sxth	r4, r3
                ((ShapeRectangle_t *)argp)->height,
 8000c3e:	687b      	ldr	r3, [r7, #4]
 8000c40:	88db      	ldrh	r3, [r3, #6]
        g_Graphics.drawRect(((ShapeRectangle_t *)argp)->start.x,
 8000c42:	b21b      	sxth	r3, r3
 8000c44:	893a      	ldrh	r2, [r7, #8]
 8000c46:	9201      	str	r2, [sp, #4]
 8000c48:	9300      	str	r3, [sp, #0]
 8000c4a:	4623      	mov	r3, r4
 8000c4c:	4602      	mov	r2, r0
 8000c4e:	4819      	ldr	r0, [pc, #100]	; (8000cb4 <_ZN7Display9drawShapeENS_7Shape_tEtPv+0x174>)
 8000c50:	f001 fba3 	bl	800239a <_ZN8Graphics8drawRectEsssst>
                color);
        break;
 8000c54:	f000 bc62 	b.w	800151c <_ZN7Display9drawShapeENS_7Shape_tEtPv+0x9dc>
    }
    case SHAPE_FillRect:
    {
        g_Graphics.fillRect(((ShapeRectangle_t *)argp)->start.x,
 8000c58:	687b      	ldr	r3, [r7, #4]
 8000c5a:	f9b3 1000 	ldrsh.w	r1, [r3]
 8000c5e:	687b      	ldr	r3, [r7, #4]
 8000c60:	f9b3 0002 	ldrsh.w	r0, [r3, #2]
                ((ShapeRectangle_t *)argp)->start.y,
                ((ShapeRectangle_t *)argp)->width,
 8000c64:	687b      	ldr	r3, [r7, #4]
 8000c66:	889b      	ldrh	r3, [r3, #4]
        g_Graphics.fillRect(((ShapeRectangle_t *)argp)->start.x,
 8000c68:	b21c      	sxth	r4, r3
                ((ShapeRectangle_t *)argp)->height,
 8000c6a:	687b      	ldr	r3, [r7, #4]
 8000c6c:	88db      	ldrh	r3, [r3, #6]
        g_Graphics.fillRect(((ShapeRectangle_t *)argp)->start.x,
 8000c6e:	b21b      	sxth	r3, r3
 8000c70:	893a      	ldrh	r2, [r7, #8]
 8000c72:	9201      	str	r2, [sp, #4]
 8000c74:	9300      	str	r3, [sp, #0]
 8000c76:	4623      	mov	r3, r4
 8000c78:	4602      	mov	r2, r0
 8000c7a:	480e      	ldr	r0, [pc, #56]	; (8000cb4 <_ZN7Display9drawShapeENS_7Shape_tEtPv+0x174>)
 8000c7c:	f001 fc23 	bl	80024c6 <_ZN8Graphics8fillRectEsssst>
                color);
        break;
 8000c80:	f000 bc4c 	b.w	800151c <_ZN7Display9drawShapeENS_7Shape_tEtPv+0x9dc>
    }
    case SHAPE_FillRoundRect:
    {
        g_Graphics.fillRoundRect(((ShapeRectangle_t *)argp)->start.x,
 8000c84:	687b      	ldr	r3, [r7, #4]
 8000c86:	f9b3 1000 	ldrsh.w	r1, [r3]
 8000c8a:	687b      	ldr	r3, [r7, #4]
 8000c8c:	f9b3 0002 	ldrsh.w	r0, [r3, #2]
                ((ShapeRectangle_t *)argp)->start.y,
                ((ShapeRectangle_t *)argp)->width,
 8000c90:	687b      	ldr	r3, [r7, #4]
 8000c92:	889b      	ldrh	r3, [r3, #4]
        g_Graphics.fillRoundRect(((ShapeRectangle_t *)argp)->start.x,
 8000c94:	b21c      	sxth	r4, r3
                ((ShapeRectangle_t *)argp)->height,6,
 8000c96:	687b      	ldr	r3, [r7, #4]
 8000c98:	88db      	ldrh	r3, [r3, #6]
        g_Graphics.fillRoundRect(((ShapeRectangle_t *)argp)->start.x,
 8000c9a:	b21b      	sxth	r3, r3
 8000c9c:	893a      	ldrh	r2, [r7, #8]
 8000c9e:	9202      	str	r2, [sp, #8]
 8000ca0:	2206      	movs	r2, #6
 8000ca2:	9201      	str	r2, [sp, #4]
 8000ca4:	9300      	str	r3, [sp, #0]
 8000ca6:	4623      	mov	r3, r4
 8000ca8:	4602      	mov	r2, r0
 8000caa:	4802      	ldr	r0, [pc, #8]	; (8000cb4 <_ZN7Display9drawShapeENS_7Shape_tEtPv+0x174>)
 8000cac:	f001 fc3a 	bl	8002524 <_ZN8Graphics13fillRoundRectEssssst>
                color);
        break;
 8000cb0:	f000 bc34 	b.w	800151c <_ZN7Display9drawShapeENS_7Shape_tEtPv+0x9dc>
 8000cb4:	200000a8 	.word	0x200000a8
    }
    case SHAPE_Arc:
    {
        uint16_t angle_trig;
        uint16_t spreadAngle = ((ShapeArc_t *)argp)->arcLength/2;
 8000cb8:	687b      	ldr	r3, [r7, #4]
 8000cba:	889b      	ldrh	r3, [r3, #4]
 8000cbc:	085b      	lsrs	r3, r3, #1
 8000cbe:	87bb      	strh	r3, [r7, #60]	; 0x3c
        uint16_t heading = ((ShapeArc_t *)argp)->heading;
 8000cc0:	687b      	ldr	r3, [r7, #4]
 8000cc2:	885b      	ldrh	r3, [r3, #2]
 8000cc4:	877b      	strh	r3, [r7, #58]	; 0x3a
        // Convert heading into trig degrees.
        angle_trig = (360 + 90 - heading) % 360;
 8000cc6:	8f7b      	ldrh	r3, [r7, #58]	; 0x3a
 8000cc8:	f5c3 73e1 	rsb	r3, r3, #450	; 0x1c2
 8000ccc:	4a97      	ldr	r2, [pc, #604]	; (8000f2c <_ZN7Display9drawShapeENS_7Shape_tEtPv+0x3ec>)
 8000cce:	fb82 1203 	smull	r1, r2, r2, r3
 8000cd2:	441a      	add	r2, r3
 8000cd4:	1211      	asrs	r1, r2, #8
 8000cd6:	17da      	asrs	r2, r3, #31
 8000cd8:	1a8a      	subs	r2, r1, r2
 8000cda:	f44f 71b4 	mov.w	r1, #360	; 0x168
 8000cde:	fb01 f202 	mul.w	r2, r1, r2
 8000ce2:	1a9a      	subs	r2, r3, r2
 8000ce4:	4613      	mov	r3, r2
 8000ce6:	873b      	strh	r3, [r7, #56]	; 0x38

        uint16_t arcRadius = ((ShapeArc_t *)argp)->radius;
 8000ce8:	687b      	ldr	r3, [r7, #4]
 8000cea:	881b      	ldrh	r3, [r3, #0]
 8000cec:	86fb      	strh	r3, [r7, #54]	; 0x36

        for (uint16_t i = 1 ; i <= spreadAngle ; i++)
 8000cee:	2301      	movs	r3, #1
 8000cf0:	f8a7 307e 	strh.w	r3, [r7, #126]	; 0x7e
 8000cf4:	f8b7 207e 	ldrh.w	r2, [r7, #126]	; 0x7e
 8000cf8:	8fbb      	ldrh	r3, [r7, #60]	; 0x3c
 8000cfa:	429a      	cmp	r2, r3
 8000cfc:	f200 840b 	bhi.w	8001516 <_ZN7Display9drawShapeENS_7Shape_tEtPv+0x9d6>
        {
            g_Graphics.drawPixel((icos(i+angle_trig)*arcRadius)+((ShapeArc_t *)argp)->x, (-isin(i+angle_trig)*arcRadius)+((ShapeArc_t *)argp)->y,0);
 8000d00:	68f8      	ldr	r0, [r7, #12]
 8000d02:	f8b7 207e 	ldrh.w	r2, [r7, #126]	; 0x7e
 8000d06:	8f3b      	ldrh	r3, [r7, #56]	; 0x38
 8000d08:	4413      	add	r3, r2
 8000d0a:	4619      	mov	r1, r3
 8000d0c:	f000 fda2 	bl	8001854 <_ZN13FastMathClass4icosEl>
 8000d10:	eeb0 7a40 	vmov.f32	s14, s0
 8000d14:	8efb      	ldrh	r3, [r7, #54]	; 0x36
 8000d16:	ee07 3a90 	vmov	s15, r3
 8000d1a:	eef8 7ae7 	vcvt.f32.s32	s15, s15
 8000d1e:	ee27 7a27 	vmul.f32	s14, s14, s15
 8000d22:	687b      	ldr	r3, [r7, #4]
 8000d24:	88db      	ldrh	r3, [r3, #6]
 8000d26:	ee07 3a90 	vmov	s15, r3
 8000d2a:	eef8 7ae7 	vcvt.f32.s32	s15, s15
 8000d2e:	ee77 7a27 	vadd.f32	s15, s14, s15
 8000d32:	eefd 7ae7 	vcvt.s32.f32	s15, s15
 8000d36:	ee17 3a90 	vmov	r3, s15
 8000d3a:	b21c      	sxth	r4, r3
 8000d3c:	68f8      	ldr	r0, [r7, #12]
 8000d3e:	f8b7 207e 	ldrh.w	r2, [r7, #126]	; 0x7e
 8000d42:	8f3b      	ldrh	r3, [r7, #56]	; 0x38
 8000d44:	4413      	add	r3, r2
 8000d46:	4619      	mov	r1, r3
 8000d48:	f000 fd0e 	bl	8001768 <_ZN13FastMathClass4isinEl>
 8000d4c:	eef0 7a40 	vmov.f32	s15, s0
 8000d50:	eeb1 7a67 	vneg.f32	s14, s15
 8000d54:	8efb      	ldrh	r3, [r7, #54]	; 0x36
 8000d56:	ee07 3a90 	vmov	s15, r3
 8000d5a:	eef8 7ae7 	vcvt.f32.s32	s15, s15
 8000d5e:	ee27 7a27 	vmul.f32	s14, s14, s15
 8000d62:	687b      	ldr	r3, [r7, #4]
 8000d64:	891b      	ldrh	r3, [r3, #8]
 8000d66:	ee07 3a90 	vmov	s15, r3
 8000d6a:	eef8 7ae7 	vcvt.f32.s32	s15, s15
 8000d6e:	ee77 7a27 	vadd.f32	s15, s14, s15
 8000d72:	eefd 7ae7 	vcvt.s32.f32	s15, s15
 8000d76:	ee17 3a90 	vmov	r3, s15
 8000d7a:	b21a      	sxth	r2, r3
 8000d7c:	2300      	movs	r3, #0
 8000d7e:	4621      	mov	r1, r4
 8000d80:	486b      	ldr	r0, [pc, #428]	; (8000f30 <_ZN7Display9drawShapeENS_7Shape_tEtPv+0x3f0>)
 8000d82:	f000 fded 	bl	8001960 <_ZN8Graphics9drawPixelEsst>
            g_Graphics.drawPixel((icos(i+angle_trig)*(arcRadius-1))+((ShapeArc_t *)argp)->x, (-isin(i+angle_trig)*(arcRadius-1))+((ShapeArc_t *)argp)->y,0);
 8000d86:	68f8      	ldr	r0, [r7, #12]
 8000d88:	f8b7 207e 	ldrh.w	r2, [r7, #126]	; 0x7e
 8000d8c:	8f3b      	ldrh	r3, [r7, #56]	; 0x38
 8000d8e:	4413      	add	r3, r2
 8000d90:	4619      	mov	r1, r3
 8000d92:	f000 fd5f 	bl	8001854 <_ZN13FastMathClass4icosEl>
 8000d96:	eeb0 7a40 	vmov.f32	s14, s0
 8000d9a:	8efb      	ldrh	r3, [r7, #54]	; 0x36
 8000d9c:	3b01      	subs	r3, #1
 8000d9e:	ee07 3a90 	vmov	s15, r3
 8000da2:	eef8 7ae7 	vcvt.f32.s32	s15, s15
 8000da6:	ee27 7a27 	vmul.f32	s14, s14, s15
 8000daa:	687b      	ldr	r3, [r7, #4]
 8000dac:	88db      	ldrh	r3, [r3, #6]
 8000dae:	ee07 3a90 	vmov	s15, r3
 8000db2:	eef8 7ae7 	vcvt.f32.s32	s15, s15
 8000db6:	ee77 7a27 	vadd.f32	s15, s14, s15
 8000dba:	eefd 7ae7 	vcvt.s32.f32	s15, s15
 8000dbe:	ee17 3a90 	vmov	r3, s15
 8000dc2:	b21c      	sxth	r4, r3
 8000dc4:	68f8      	ldr	r0, [r7, #12]
 8000dc6:	f8b7 207e 	ldrh.w	r2, [r7, #126]	; 0x7e
 8000dca:	8f3b      	ldrh	r3, [r7, #56]	; 0x38
 8000dcc:	4413      	add	r3, r2
 8000dce:	4619      	mov	r1, r3
 8000dd0:	f000 fcca 	bl	8001768 <_ZN13FastMathClass4isinEl>
 8000dd4:	eef0 7a40 	vmov.f32	s15, s0
 8000dd8:	eeb1 7a67 	vneg.f32	s14, s15
 8000ddc:	8efb      	ldrh	r3, [r7, #54]	; 0x36
 8000dde:	3b01      	subs	r3, #1
 8000de0:	ee07 3a90 	vmov	s15, r3
 8000de4:	eef8 7ae7 	vcvt.f32.s32	s15, s15
 8000de8:	ee27 7a27 	vmul.f32	s14, s14, s15
 8000dec:	687b      	ldr	r3, [r7, #4]
 8000dee:	891b      	ldrh	r3, [r3, #8]
 8000df0:	ee07 3a90 	vmov	s15, r3
 8000df4:	eef8 7ae7 	vcvt.f32.s32	s15, s15
 8000df8:	ee77 7a27 	vadd.f32	s15, s14, s15
 8000dfc:	eefd 7ae7 	vcvt.s32.f32	s15, s15
 8000e00:	ee17 3a90 	vmov	r3, s15
 8000e04:	b21a      	sxth	r2, r3
 8000e06:	2300      	movs	r3, #0
 8000e08:	4621      	mov	r1, r4
 8000e0a:	4849      	ldr	r0, [pc, #292]	; (8000f30 <_ZN7Display9drawShapeENS_7Shape_tEtPv+0x3f0>)
 8000e0c:	f000 fda8 	bl	8001960 <_ZN8Graphics9drawPixelEsst>
            g_Graphics.drawPixel((icos(angle_trig-i)*arcRadius)+((ShapeArc_t *)argp)->x, (-isin(angle_trig-i)*arcRadius)+((ShapeArc_t *)argp)->y,0);
 8000e10:	68f8      	ldr	r0, [r7, #12]
 8000e12:	8f3a      	ldrh	r2, [r7, #56]	; 0x38
 8000e14:	f8b7 307e 	ldrh.w	r3, [r7, #126]	; 0x7e
 8000e18:	1ad3      	subs	r3, r2, r3
 8000e1a:	4619      	mov	r1, r3
 8000e1c:	f000 fd1a 	bl	8001854 <_ZN13FastMathClass4icosEl>
 8000e20:	eeb0 7a40 	vmov.f32	s14, s0
 8000e24:	8efb      	ldrh	r3, [r7, #54]	; 0x36
 8000e26:	ee07 3a90 	vmov	s15, r3
 8000e2a:	eef8 7ae7 	vcvt.f32.s32	s15, s15
 8000e2e:	ee27 7a27 	vmul.f32	s14, s14, s15
 8000e32:	687b      	ldr	r3, [r7, #4]
 8000e34:	88db      	ldrh	r3, [r3, #6]
 8000e36:	ee07 3a90 	vmov	s15, r3
 8000e3a:	eef8 7ae7 	vcvt.f32.s32	s15, s15
 8000e3e:	ee77 7a27 	vadd.f32	s15, s14, s15
 8000e42:	eefd 7ae7 	vcvt.s32.f32	s15, s15
 8000e46:	ee17 3a90 	vmov	r3, s15
 8000e4a:	b21c      	sxth	r4, r3
 8000e4c:	68f8      	ldr	r0, [r7, #12]
 8000e4e:	8f3a      	ldrh	r2, [r7, #56]	; 0x38
 8000e50:	f8b7 307e 	ldrh.w	r3, [r7, #126]	; 0x7e
 8000e54:	1ad3      	subs	r3, r2, r3
 8000e56:	4619      	mov	r1, r3
 8000e58:	f000 fc86 	bl	8001768 <_ZN13FastMathClass4isinEl>
 8000e5c:	eef0 7a40 	vmov.f32	s15, s0
 8000e60:	eeb1 7a67 	vneg.f32	s14, s15
 8000e64:	8efb      	ldrh	r3, [r7, #54]	; 0x36
 8000e66:	ee07 3a90 	vmov	s15, r3
 8000e6a:	eef8 7ae7 	vcvt.f32.s32	s15, s15
 8000e6e:	ee27 7a27 	vmul.f32	s14, s14, s15
 8000e72:	687b      	ldr	r3, [r7, #4]
 8000e74:	891b      	ldrh	r3, [r3, #8]
 8000e76:	ee07 3a90 	vmov	s15, r3
 8000e7a:	eef8 7ae7 	vcvt.f32.s32	s15, s15
 8000e7e:	ee77 7a27 	vadd.f32	s15, s14, s15
 8000e82:	eefd 7ae7 	vcvt.s32.f32	s15, s15
 8000e86:	ee17 3a90 	vmov	r3, s15
 8000e8a:	b21a      	sxth	r2, r3
 8000e8c:	2300      	movs	r3, #0
 8000e8e:	4621      	mov	r1, r4
 8000e90:	4827      	ldr	r0, [pc, #156]	; (8000f30 <_ZN7Display9drawShapeENS_7Shape_tEtPv+0x3f0>)
 8000e92:	f000 fd65 	bl	8001960 <_ZN8Graphics9drawPixelEsst>
            g_Graphics.drawPixel((icos(angle_trig-i)*(arcRadius-1))+((ShapeArc_t *)argp)->x, (-isin(angle_trig-i)*(arcRadius-1))+((ShapeArc_t *)argp)->y,0);
 8000e96:	68f8      	ldr	r0, [r7, #12]
 8000e98:	8f3a      	ldrh	r2, [r7, #56]	; 0x38
 8000e9a:	f8b7 307e 	ldrh.w	r3, [r7, #126]	; 0x7e
 8000e9e:	1ad3      	subs	r3, r2, r3
 8000ea0:	4619      	mov	r1, r3
 8000ea2:	f000 fcd7 	bl	8001854 <_ZN13FastMathClass4icosEl>
 8000ea6:	eeb0 7a40 	vmov.f32	s14, s0
 8000eaa:	8efb      	ldrh	r3, [r7, #54]	; 0x36
 8000eac:	3b01      	subs	r3, #1
 8000eae:	ee07 3a90 	vmov	s15, r3
 8000eb2:	eef8 7ae7 	vcvt.f32.s32	s15, s15
 8000eb6:	ee27 7a27 	vmul.f32	s14, s14, s15
 8000eba:	687b      	ldr	r3, [r7, #4]
 8000ebc:	88db      	ldrh	r3, [r3, #6]
 8000ebe:	ee07 3a90 	vmov	s15, r3
 8000ec2:	eef8 7ae7 	vcvt.f32.s32	s15, s15
 8000ec6:	ee77 7a27 	vadd.f32	s15, s14, s15
 8000eca:	eefd 7ae7 	vcvt.s32.f32	s15, s15
 8000ece:	ee17 3a90 	vmov	r3, s15
 8000ed2:	b21c      	sxth	r4, r3
 8000ed4:	68f8      	ldr	r0, [r7, #12]
 8000ed6:	8f3a      	ldrh	r2, [r7, #56]	; 0x38
 8000ed8:	f8b7 307e 	ldrh.w	r3, [r7, #126]	; 0x7e
 8000edc:	1ad3      	subs	r3, r2, r3
 8000ede:	4619      	mov	r1, r3
 8000ee0:	f000 fc42 	bl	8001768 <_ZN13FastMathClass4isinEl>
 8000ee4:	eef0 7a40 	vmov.f32	s15, s0
 8000ee8:	eeb1 7a67 	vneg.f32	s14, s15
 8000eec:	8efb      	ldrh	r3, [r7, #54]	; 0x36
 8000eee:	3b01      	subs	r3, #1
 8000ef0:	ee07 3a90 	vmov	s15, r3
 8000ef4:	eef8 7ae7 	vcvt.f32.s32	s15, s15
 8000ef8:	ee27 7a27 	vmul.f32	s14, s14, s15
 8000efc:	687b      	ldr	r3, [r7, #4]
 8000efe:	891b      	ldrh	r3, [r3, #8]
 8000f00:	ee07 3a90 	vmov	s15, r3
 8000f04:	eef8 7ae7 	vcvt.f32.s32	s15, s15
 8000f08:	ee77 7a27 	vadd.f32	s15, s14, s15
 8000f0c:	eefd 7ae7 	vcvt.s32.f32	s15, s15
 8000f10:	ee17 3a90 	vmov	r3, s15
 8000f14:	b21a      	sxth	r2, r3
 8000f16:	2300      	movs	r3, #0
 8000f18:	4621      	mov	r1, r4
 8000f1a:	4805      	ldr	r0, [pc, #20]	; (8000f30 <_ZN7Display9drawShapeENS_7Shape_tEtPv+0x3f0>)
 8000f1c:	f000 fd20 	bl	8001960 <_ZN8Graphics9drawPixelEsst>
        for (uint16_t i = 1 ; i <= spreadAngle ; i++)
 8000f20:	f8b7 307e 	ldrh.w	r3, [r7, #126]	; 0x7e
 8000f24:	3301      	adds	r3, #1
 8000f26:	f8a7 307e 	strh.w	r3, [r7, #126]	; 0x7e
 8000f2a:	e6e3      	b.n	8000cf4 <_ZN7Display9drawShapeENS_7Shape_tEtPv+0x1b4>
 8000f2c:	b60b60b7 	.word	0xb60b60b7
 8000f30:	200000a8 	.word	0x200000a8

        break;
    }
    case SHAPE_Arrow:
    {
        int16_t x2=0;
 8000f34:	2300      	movs	r3, #0
 8000f36:	f8a7 3070 	strh.w	r3, [r7, #112]	; 0x70
        int16_t y2=0;
 8000f3a:	2300      	movs	r3, #0
 8000f3c:	f8a7 306e 	strh.w	r3, [r7, #110]	; 0x6e
        int16_t edgeLength = 55 ;
 8000f40:	2337      	movs	r3, #55	; 0x37
 8000f42:	f8a7 306c 	strh.w	r3, [r7, #108]	; 0x6c
        int16_t arrowArm = 40 ;
 8000f46:	2328      	movs	r3, #40	; 0x28
 8000f48:	f8a7 306a 	strh.w	r3, [r7, #106]	; 0x6a
        int16_t osx = X_CENTER;
 8000f4c:	2373      	movs	r3, #115	; 0x73
 8000f4e:	f8a7 3068 	strh.w	r3, [r7, #104]	; 0x68
        int16_t osy = Y_CENTER;
 8000f52:	236f      	movs	r3, #111	; 0x6f
 8000f54:	f8a7 3066 	strh.w	r3, [r7, #102]	; 0x66
        uint8_t arrowWidth = 25, rectWidth=10;
 8000f58:	2319      	movs	r3, #25
 8000f5a:	f887 3065 	strb.w	r3, [r7, #101]	; 0x65
 8000f5e:	230a      	movs	r3, #10
 8000f60:	f887 3064 	strb.w	r3, [r7, #100]	; 0x64

        int16_t headingAngle =  *((ShapeArrow_t *)argp);
 8000f64:	687b      	ldr	r3, [r7, #4]
 8000f66:	881b      	ldrh	r3, [r3, #0]
 8000f68:	f8a7 3062 	strh.w	r3, [r7, #98]	; 0x62

        x2 = -icos(headingAngle) * edgeLength;
 8000f6c:	68fb      	ldr	r3, [r7, #12]
 8000f6e:	f9b7 2062 	ldrsh.w	r2, [r7, #98]	; 0x62
 8000f72:	4611      	mov	r1, r2
 8000f74:	4618      	mov	r0, r3
 8000f76:	f000 fc6d 	bl	8001854 <_ZN13FastMathClass4icosEl>
 8000f7a:	eef0 7a40 	vmov.f32	s15, s0
 8000f7e:	eeb1 7a67 	vneg.f32	s14, s15
 8000f82:	f9b7 306c 	ldrsh.w	r3, [r7, #108]	; 0x6c
 8000f86:	ee07 3a90 	vmov	s15, r3
 8000f8a:	eef8 7ae7 	vcvt.f32.s32	s15, s15
 8000f8e:	ee67 7a27 	vmul.f32	s15, s14, s15
 8000f92:	eefd 7ae7 	vcvt.s32.f32	s15, s15
 8000f96:	ee17 3a90 	vmov	r3, s15
 8000f9a:	f8a7 3070 	strh.w	r3, [r7, #112]	; 0x70
        y2 = isin(headingAngle) * edgeLength;
 8000f9e:	68fb      	ldr	r3, [r7, #12]
 8000fa0:	f9b7 2062 	ldrsh.w	r2, [r7, #98]	; 0x62
 8000fa4:	4611      	mov	r1, r2
 8000fa6:	4618      	mov	r0, r3
 8000fa8:	f000 fbde 	bl	8001768 <_ZN13FastMathClass4isinEl>
 8000fac:	eeb0 7a40 	vmov.f32	s14, s0
 8000fb0:	f9b7 306c 	ldrsh.w	r3, [r7, #108]	; 0x6c
 8000fb4:	ee07 3a90 	vmov	s15, r3
 8000fb8:	eef8 7ae7 	vcvt.f32.s32	s15, s15
 8000fbc:	ee67 7a27 	vmul.f32	s15, s14, s15
 8000fc0:	eefd 7ae7 	vcvt.s32.f32	s15, s15
 8000fc4:	ee17 3a90 	vmov	r3, s15
 8000fc8:	f8a7 306e 	strh.w	r3, [r7, #110]	; 0x6e

        // Arrow Head Point
        int16_t xt = -x2+osx;
 8000fcc:	f8b7 2068 	ldrh.w	r2, [r7, #104]	; 0x68
 8000fd0:	f8b7 3070 	ldrh.w	r3, [r7, #112]	; 0x70
 8000fd4:	1ad3      	subs	r3, r2, r3
 8000fd6:	b29b      	uxth	r3, r3
 8000fd8:	f8a7 3060 	strh.w	r3, [r7, #96]	; 0x60
        int16_t yt = -y2+osy;
 8000fdc:	f8b7 2066 	ldrh.w	r2, [r7, #102]	; 0x66
 8000fe0:	f8b7 306e 	ldrh.w	r3, [r7, #110]	; 0x6e
 8000fe4:	1ad3      	subs	r3, r2, r3
 8000fe6:	b29b      	uxth	r3, r3
 8000fe8:	f8a7 305e 	strh.w	r3, [r7, #94]	; 0x5e

        // Arrow Arms end points
        int16_t xt1 = (icos(headingAngle+arrowWidth) * arrowArm)+osx;
 8000fec:	68f8      	ldr	r0, [r7, #12]
 8000fee:	f9b7 2062 	ldrsh.w	r2, [r7, #98]	; 0x62
 8000ff2:	f897 3065 	ldrb.w	r3, [r7, #101]	; 0x65
 8000ff6:	4413      	add	r3, r2
 8000ff8:	4619      	mov	r1, r3
 8000ffa:	f000 fc2b 	bl	8001854 <_ZN13FastMathClass4icosEl>
 8000ffe:	eeb0 7a40 	vmov.f32	s14, s0
 8001002:	f9b7 306a 	ldrsh.w	r3, [r7, #106]	; 0x6a
 8001006:	ee07 3a90 	vmov	s15, r3
 800100a:	eef8 7ae7 	vcvt.f32.s32	s15, s15
 800100e:	ee27 7a27 	vmul.f32	s14, s14, s15
 8001012:	f9b7 3068 	ldrsh.w	r3, [r7, #104]	; 0x68
 8001016:	ee07 3a90 	vmov	s15, r3
 800101a:	eef8 7ae7 	vcvt.f32.s32	s15, s15
 800101e:	ee77 7a27 	vadd.f32	s15, s14, s15
 8001022:	eefd 7ae7 	vcvt.s32.f32	s15, s15
 8001026:	ee17 3a90 	vmov	r3, s15
 800102a:	f8a7 305c 	strh.w	r3, [r7, #92]	; 0x5c
        int16_t yt1 = (-isin(headingAngle+arrowWidth) * arrowArm )+osy;
 800102e:	68f8      	ldr	r0, [r7, #12]
 8001030:	f9b7 2062 	ldrsh.w	r2, [r7, #98]	; 0x62
 8001034:	f897 3065 	ldrb.w	r3, [r7, #101]	; 0x65
 8001038:	4413      	add	r3, r2
 800103a:	4619      	mov	r1, r3
 800103c:	f000 fb94 	bl	8001768 <_ZN13FastMathClass4isinEl>
 8001040:	eef0 7a40 	vmov.f32	s15, s0
 8001044:	eeb1 7a67 	vneg.f32	s14, s15
 8001048:	f9b7 306a 	ldrsh.w	r3, [r7, #106]	; 0x6a
 800104c:	ee07 3a90 	vmov	s15, r3
 8001050:	eef8 7ae7 	vcvt.f32.s32	s15, s15
 8001054:	ee27 7a27 	vmul.f32	s14, s14, s15
 8001058:	f9b7 3066 	ldrsh.w	r3, [r7, #102]	; 0x66
 800105c:	ee07 3a90 	vmov	s15, r3
 8001060:	eef8 7ae7 	vcvt.f32.s32	s15, s15
 8001064:	ee77 7a27 	vadd.f32	s15, s14, s15
 8001068:	eefd 7ae7 	vcvt.s32.f32	s15, s15
 800106c:	ee17 3a90 	vmov	r3, s15
 8001070:	f8a7 305a 	strh.w	r3, [r7, #90]	; 0x5a
        int16_t xt2 = (icos(headingAngle-arrowWidth) * arrowArm)+osx;
 8001074:	68f8      	ldr	r0, [r7, #12]
 8001076:	f9b7 2062 	ldrsh.w	r2, [r7, #98]	; 0x62
 800107a:	f897 3065 	ldrb.w	r3, [r7, #101]	; 0x65
 800107e:	1ad3      	subs	r3, r2, r3
 8001080:	4619      	mov	r1, r3
 8001082:	f000 fbe7 	bl	8001854 <_ZN13FastMathClass4icosEl>
 8001086:	eeb0 7a40 	vmov.f32	s14, s0
 800108a:	f9b7 306a 	ldrsh.w	r3, [r7, #106]	; 0x6a
 800108e:	ee07 3a90 	vmov	s15, r3
 8001092:	eef8 7ae7 	vcvt.f32.s32	s15, s15
 8001096:	ee27 7a27 	vmul.f32	s14, s14, s15
 800109a:	f9b7 3068 	ldrsh.w	r3, [r7, #104]	; 0x68
 800109e:	ee07 3a90 	vmov	s15, r3
 80010a2:	eef8 7ae7 	vcvt.f32.s32	s15, s15
 80010a6:	ee77 7a27 	vadd.f32	s15, s14, s15
 80010aa:	eefd 7ae7 	vcvt.s32.f32	s15, s15
 80010ae:	ee17 3a90 	vmov	r3, s15
 80010b2:	f8a7 3058 	strh.w	r3, [r7, #88]	; 0x58
        int16_t yt2 = (-isin(headingAngle-arrowWidth) * arrowArm )+osy;
 80010b6:	68f8      	ldr	r0, [r7, #12]
 80010b8:	f9b7 2062 	ldrsh.w	r2, [r7, #98]	; 0x62
 80010bc:	f897 3065 	ldrb.w	r3, [r7, #101]	; 0x65
 80010c0:	1ad3      	subs	r3, r2, r3
 80010c2:	4619      	mov	r1, r3
 80010c4:	f000 fb50 	bl	8001768 <_ZN13FastMathClass4isinEl>
 80010c8:	eef0 7a40 	vmov.f32	s15, s0
 80010cc:	eeb1 7a67 	vneg.f32	s14, s15
 80010d0:	f9b7 306a 	ldrsh.w	r3, [r7, #106]	; 0x6a
 80010d4:	ee07 3a90 	vmov	s15, r3
 80010d8:	eef8 7ae7 	vcvt.f32.s32	s15, s15
 80010dc:	ee27 7a27 	vmul.f32	s14, s14, s15
 80010e0:	f9b7 3066 	ldrsh.w	r3, [r7, #102]	; 0x66
 80010e4:	ee07 3a90 	vmov	s15, r3
 80010e8:	eef8 7ae7 	vcvt.f32.s32	s15, s15
 80010ec:	ee77 7a27 	vadd.f32	s15, s14, s15
 80010f0:	eefd 7ae7 	vcvt.s32.f32	s15, s15
 80010f4:	ee17 3a90 	vmov	r3, s15
 80010f8:	f8a7 3056 	strh.w	r3, [r7, #86]	; 0x56

        int16_t xt3 = (-icos(headingAngle+rectWidth) * arrowArm);
 80010fc:	68f8      	ldr	r0, [r7, #12]
 80010fe:	f9b7 2062 	ldrsh.w	r2, [r7, #98]	; 0x62
 8001102:	f897 3064 	ldrb.w	r3, [r7, #100]	; 0x64
 8001106:	4413      	add	r3, r2
 8001108:	4619      	mov	r1, r3
 800110a:	f000 fba3 	bl	8001854 <_ZN13FastMathClass4icosEl>
 800110e:	eef0 7a40 	vmov.f32	s15, s0
 8001112:	eeb1 7a67 	vneg.f32	s14, s15
 8001116:	f9b7 306a 	ldrsh.w	r3, [r7, #106]	; 0x6a
 800111a:	ee07 3a90 	vmov	s15, r3
 800111e:	eef8 7ae7 	vcvt.f32.s32	s15, s15
 8001122:	ee67 7a27 	vmul.f32	s15, s14, s15
 8001126:	eefd 7ae7 	vcvt.s32.f32	s15, s15
 800112a:	ee17 3a90 	vmov	r3, s15
 800112e:	f8a7 3054 	strh.w	r3, [r7, #84]	; 0x54
        int16_t yt3 = (isin(headingAngle+rectWidth) * arrowArm );
 8001132:	68f8      	ldr	r0, [r7, #12]
 8001134:	f9b7 2062 	ldrsh.w	r2, [r7, #98]	; 0x62
 8001138:	f897 3064 	ldrb.w	r3, [r7, #100]	; 0x64
 800113c:	4413      	add	r3, r2
 800113e:	4619      	mov	r1, r3
 8001140:	f000 fb12 	bl	8001768 <_ZN13FastMathClass4isinEl>
 8001144:	eeb0 7a40 	vmov.f32	s14, s0
 8001148:	f9b7 306a 	ldrsh.w	r3, [r7, #106]	; 0x6a
 800114c:	ee07 3a90 	vmov	s15, r3
 8001150:	eef8 7ae7 	vcvt.f32.s32	s15, s15
 8001154:	ee67 7a27 	vmul.f32	s15, s14, s15
 8001158:	eefd 7ae7 	vcvt.s32.f32	s15, s15
 800115c:	ee17 3a90 	vmov	r3, s15
 8001160:	f8a7 3052 	strh.w	r3, [r7, #82]	; 0x52
        int16_t xt4 = (-icos(headingAngle-rectWidth) * arrowArm);
 8001164:	68f8      	ldr	r0, [r7, #12]
 8001166:	f9b7 2062 	ldrsh.w	r2, [r7, #98]	; 0x62
 800116a:	f897 3064 	ldrb.w	r3, [r7, #100]	; 0x64
 800116e:	1ad3      	subs	r3, r2, r3
 8001170:	4619      	mov	r1, r3
 8001172:	f000 fb6f 	bl	8001854 <_ZN13FastMathClass4icosEl>
 8001176:	eef0 7a40 	vmov.f32	s15, s0
 800117a:	eeb1 7a67 	vneg.f32	s14, s15
 800117e:	f9b7 306a 	ldrsh.w	r3, [r7, #106]	; 0x6a
 8001182:	ee07 3a90 	vmov	s15, r3
 8001186:	eef8 7ae7 	vcvt.f32.s32	s15, s15
 800118a:	ee67 7a27 	vmul.f32	s15, s14, s15
 800118e:	eefd 7ae7 	vcvt.s32.f32	s15, s15
 8001192:	ee17 3a90 	vmov	r3, s15
 8001196:	f8a7 3050 	strh.w	r3, [r7, #80]	; 0x50
        int16_t yt4 = (isin(headingAngle-rectWidth) * arrowArm );
 800119a:	68f8      	ldr	r0, [r7, #12]
 800119c:	f9b7 2062 	ldrsh.w	r2, [r7, #98]	; 0x62
 80011a0:	f897 3064 	ldrb.w	r3, [r7, #100]	; 0x64
 80011a4:	1ad3      	subs	r3, r2, r3
 80011a6:	4619      	mov	r1, r3
 80011a8:	f000 fade 	bl	8001768 <_ZN13FastMathClass4isinEl>
 80011ac:	eeb0 7a40 	vmov.f32	s14, s0
 80011b0:	f9b7 306a 	ldrsh.w	r3, [r7, #106]	; 0x6a
 80011b4:	ee07 3a90 	vmov	s15, r3
 80011b8:	eef8 7ae7 	vcvt.f32.s32	s15, s15
 80011bc:	ee67 7a27 	vmul.f32	s15, s14, s15
 80011c0:	eefd 7ae7 	vcvt.s32.f32	s15, s15
 80011c4:	ee17 3a90 	vmov	r3, s15
 80011c8:	f8a7 304e 	strh.w	r3, [r7, #78]	; 0x4e

        int16_t xrect1 = -xt3+osx;
 80011cc:	f8b7 2068 	ldrh.w	r2, [r7, #104]	; 0x68
 80011d0:	f8b7 3054 	ldrh.w	r3, [r7, #84]	; 0x54
 80011d4:	1ad3      	subs	r3, r2, r3
 80011d6:	b29b      	uxth	r3, r3
 80011d8:	f8a7 304c 	strh.w	r3, [r7, #76]	; 0x4c
        int16_t yrect1 = -yt3+osy;
 80011dc:	f8b7 2066 	ldrh.w	r2, [r7, #102]	; 0x66
 80011e0:	f8b7 3052 	ldrh.w	r3, [r7, #82]	; 0x52
 80011e4:	1ad3      	subs	r3, r2, r3
 80011e6:	b29b      	uxth	r3, r3
 80011e8:	f8a7 304a 	strh.w	r3, [r7, #74]	; 0x4a
        int16_t xrect2 = xt3+osx;
 80011ec:	f8b7 2054 	ldrh.w	r2, [r7, #84]	; 0x54
 80011f0:	f8b7 3068 	ldrh.w	r3, [r7, #104]	; 0x68
 80011f4:	4413      	add	r3, r2
 80011f6:	b29b      	uxth	r3, r3
 80011f8:	f8a7 3048 	strh.w	r3, [r7, #72]	; 0x48
        int16_t yrect2 = yt3+osy;
 80011fc:	f8b7 2052 	ldrh.w	r2, [r7, #82]	; 0x52
 8001200:	f8b7 3066 	ldrh.w	r3, [r7, #102]	; 0x66
 8001204:	4413      	add	r3, r2
 8001206:	b29b      	uxth	r3, r3
 8001208:	f8a7 3046 	strh.w	r3, [r7, #70]	; 0x46

        int16_t xrect3 = -xt4+osx;
 800120c:	f8b7 2068 	ldrh.w	r2, [r7, #104]	; 0x68
 8001210:	f8b7 3050 	ldrh.w	r3, [r7, #80]	; 0x50
 8001214:	1ad3      	subs	r3, r2, r3
 8001216:	b29b      	uxth	r3, r3
 8001218:	f8a7 3044 	strh.w	r3, [r7, #68]	; 0x44
        int16_t yrect3 = -yt4+osy;
 800121c:	f8b7 2066 	ldrh.w	r2, [r7, #102]	; 0x66
 8001220:	f8b7 304e 	ldrh.w	r3, [r7, #78]	; 0x4e
 8001224:	1ad3      	subs	r3, r2, r3
 8001226:	b29b      	uxth	r3, r3
 8001228:	f8a7 3042 	strh.w	r3, [r7, #66]	; 0x42
        int16_t xrect4 = xt4+osx;
 800122c:	f8b7 2050 	ldrh.w	r2, [r7, #80]	; 0x50
 8001230:	f8b7 3068 	ldrh.w	r3, [r7, #104]	; 0x68
 8001234:	4413      	add	r3, r2
 8001236:	b29b      	uxth	r3, r3
 8001238:	f8a7 3040 	strh.w	r3, [r7, #64]	; 0x40
        int16_t yrect4 = yt4+osy;
 800123c:	f8b7 204e 	ldrh.w	r2, [r7, #78]	; 0x4e
 8001240:	f8b7 3066 	ldrh.w	r3, [r7, #102]	; 0x66
 8001244:	4413      	add	r3, r2
 8001246:	b29b      	uxth	r3, r3
 8001248:	87fb      	strh	r3, [r7, #62]	; 0x3e

        ShapeTriangle_t tri = {{xt,yt},{xt1,yt1},{xt2,yt2}};
 800124a:	f8b7 3060 	ldrh.w	r3, [r7, #96]	; 0x60
 800124e:	853b      	strh	r3, [r7, #40]	; 0x28
 8001250:	f8b7 305e 	ldrh.w	r3, [r7, #94]	; 0x5e
 8001254:	857b      	strh	r3, [r7, #42]	; 0x2a
 8001256:	f8b7 305c 	ldrh.w	r3, [r7, #92]	; 0x5c
 800125a:	85bb      	strh	r3, [r7, #44]	; 0x2c
 800125c:	f8b7 305a 	ldrh.w	r3, [r7, #90]	; 0x5a
 8001260:	85fb      	strh	r3, [r7, #46]	; 0x2e
 8001262:	f8b7 3058 	ldrh.w	r3, [r7, #88]	; 0x58
 8001266:	863b      	strh	r3, [r7, #48]	; 0x30
 8001268:	f8b7 3056 	ldrh.w	r3, [r7, #86]	; 0x56
 800126c:	867b      	strh	r3, [r7, #50]	; 0x32
        ShapeTriangle_t tri2 = {{xrect1,yrect1},{xrect2,yrect2},{xrect4,yrect4}};
 800126e:	f8b7 304c 	ldrh.w	r3, [r7, #76]	; 0x4c
 8001272:	83bb      	strh	r3, [r7, #28]
 8001274:	f8b7 304a 	ldrh.w	r3, [r7, #74]	; 0x4a
 8001278:	83fb      	strh	r3, [r7, #30]
 800127a:	f8b7 3048 	ldrh.w	r3, [r7, #72]	; 0x48
 800127e:	843b      	strh	r3, [r7, #32]
 8001280:	f8b7 3046 	ldrh.w	r3, [r7, #70]	; 0x46
 8001284:	847b      	strh	r3, [r7, #34]	; 0x22
 8001286:	f8b7 3040 	ldrh.w	r3, [r7, #64]	; 0x40
 800128a:	84bb      	strh	r3, [r7, #36]	; 0x24
 800128c:	8ffb      	ldrh	r3, [r7, #62]	; 0x3e
 800128e:	84fb      	strh	r3, [r7, #38]	; 0x26
        ShapeTriangle_t tri3 = {{xrect1,yrect1},{xrect3,yrect3},{xrect2,yrect2}};
 8001290:	f8b7 304c 	ldrh.w	r3, [r7, #76]	; 0x4c
 8001294:	823b      	strh	r3, [r7, #16]
 8001296:	f8b7 304a 	ldrh.w	r3, [r7, #74]	; 0x4a
 800129a:	827b      	strh	r3, [r7, #18]
 800129c:	f8b7 3044 	ldrh.w	r3, [r7, #68]	; 0x44
 80012a0:	82bb      	strh	r3, [r7, #20]
 80012a2:	f8b7 3042 	ldrh.w	r3, [r7, #66]	; 0x42
 80012a6:	82fb      	strh	r3, [r7, #22]
 80012a8:	f8b7 3048 	ldrh.w	r3, [r7, #72]	; 0x48
 80012ac:	833b      	strh	r3, [r7, #24]
 80012ae:	f8b7 3046 	ldrh.w	r3, [r7, #70]	; 0x46
 80012b2:	837b      	strh	r3, [r7, #26]

        //The arrow consists of three triangles
        drawShape(SHAPE_Triangle, color, &tri);			//Arrowpoint
 80012b4:	f107 0328 	add.w	r3, r7, #40	; 0x28
 80012b8:	893a      	ldrh	r2, [r7, #8]
 80012ba:	2103      	movs	r1, #3
 80012bc:	68f8      	ldr	r0, [r7, #12]
 80012be:	f7ff fc3f 	bl	8000b40 <_ZN7Display9drawShapeENS_7Shape_tEtPv>
        drawShape(SHAPE_Triangle, color, &tri2);		//triangle left arm
 80012c2:	f107 031c 	add.w	r3, r7, #28
 80012c6:	893a      	ldrh	r2, [r7, #8]
 80012c8:	2103      	movs	r1, #3
 80012ca:	68f8      	ldr	r0, [r7, #12]
 80012cc:	f7ff fc38 	bl	8000b40 <_ZN7Display9drawShapeENS_7Shape_tEtPv>
        drawShape(SHAPE_Triangle, color, &tri3);		//triangle right arm
 80012d0:	f107 0310 	add.w	r3, r7, #16
 80012d4:	893a      	ldrh	r2, [r7, #8]
 80012d6:	2103      	movs	r1, #3
 80012d8:	68f8      	ldr	r0, [r7, #12]
 80012da:	f7ff fc31 	bl	8000b40 <_ZN7Display9drawShapeENS_7Shape_tEtPv>

        break;
 80012de:	bf00      	nop
 80012e0:	e11c      	b.n	800151c <_ZN7Display9drawShapeENS_7Shape_tEtPv+0x9dc>
    }
    case SHAPE_BoldArc:
    {
        uint16_t angle_trig;
        uint16_t spreadAngle = ((ShapeArc_t *)argp)->arcLength/2;
 80012e2:	687b      	ldr	r3, [r7, #4]
 80012e4:	889b      	ldrh	r3, [r3, #4]
 80012e6:	085b      	lsrs	r3, r3, #1
 80012e8:	f8a7 307a 	strh.w	r3, [r7, #122]	; 0x7a
        uint16_t heading = ((ShapeArc_t *)argp)->heading;
 80012ec:	687b      	ldr	r3, [r7, #4]
 80012ee:	885b      	ldrh	r3, [r3, #2]
 80012f0:	f8a7 3078 	strh.w	r3, [r7, #120]	; 0x78
        // Convert heading into trig degrees.
        angle_trig = (360 + 90 - heading) % 360;
 80012f4:	f8b7 3078 	ldrh.w	r3, [r7, #120]	; 0x78
 80012f8:	f5c3 73e1 	rsb	r3, r3, #450	; 0x1c2
 80012fc:	4a89      	ldr	r2, [pc, #548]	; (8001524 <_ZN7Display9drawShapeENS_7Shape_tEtPv+0x9e4>)
 80012fe:	fb82 1203 	smull	r1, r2, r2, r3
 8001302:	441a      	add	r2, r3
 8001304:	1211      	asrs	r1, r2, #8
 8001306:	17da      	asrs	r2, r3, #31
 8001308:	1a8a      	subs	r2, r1, r2
 800130a:	f44f 71b4 	mov.w	r1, #360	; 0x168
 800130e:	fb01 f202 	mul.w	r2, r1, r2
 8001312:	1a9a      	subs	r2, r3, r2
 8001314:	4613      	mov	r3, r2
 8001316:	f8a7 3076 	strh.w	r3, [r7, #118]	; 0x76

        uint16_t arcRadius = ((ShapeArc_t *)argp)->radius;
 800131a:	687b      	ldr	r3, [r7, #4]
 800131c:	881b      	ldrh	r3, [r3, #0]
 800131e:	f8a7 3074 	strh.w	r3, [r7, #116]	; 0x74

        uint8_t cirRadius = CIRCLE_RADIUS;
 8001322:	2305      	movs	r3, #5
 8001324:	f887 3073 	strb.w	r3, [r7, #115]	; 0x73

        if(spreadAngle == 0)
 8001328:	f8b7 307a 	ldrh.w	r3, [r7, #122]	; 0x7a
 800132c:	2b00      	cmp	r3, #0
 800132e:	d148      	bne.n	80013c2 <_ZN7Display9drawShapeENS_7Shape_tEtPv+0x882>
        {
            g_Graphics.fillCircle((icos(angle_trig)*arcRadius)+((ShapeArc_t *)argp)->x, (-isin(angle_trig)*arcRadius)+((ShapeArc_t *)argp)->y,cirRadius,0);
 8001330:	68fb      	ldr	r3, [r7, #12]
 8001332:	f8b7 2076 	ldrh.w	r2, [r7, #118]	; 0x76
 8001336:	4611      	mov	r1, r2
 8001338:	4618      	mov	r0, r3
 800133a:	f000 fa8b 	bl	8001854 <_ZN13FastMathClass4icosEl>
 800133e:	eeb0 7a40 	vmov.f32	s14, s0
 8001342:	f8b7 3074 	ldrh.w	r3, [r7, #116]	; 0x74
 8001346:	ee07 3a90 	vmov	s15, r3
 800134a:	eef8 7ae7 	vcvt.f32.s32	s15, s15
 800134e:	ee27 7a27 	vmul.f32	s14, s14, s15
 8001352:	687b      	ldr	r3, [r7, #4]
 8001354:	88db      	ldrh	r3, [r3, #6]
 8001356:	ee07 3a90 	vmov	s15, r3
 800135a:	eef8 7ae7 	vcvt.f32.s32	s15, s15
 800135e:	ee77 7a27 	vadd.f32	s15, s14, s15
 8001362:	eefd 7ae7 	vcvt.s32.f32	s15, s15
 8001366:	ee17 3a90 	vmov	r3, s15
 800136a:	b21c      	sxth	r4, r3
 800136c:	68fb      	ldr	r3, [r7, #12]
 800136e:	f8b7 2076 	ldrh.w	r2, [r7, #118]	; 0x76
 8001372:	4611      	mov	r1, r2
 8001374:	4618      	mov	r0, r3
 8001376:	f000 f9f7 	bl	8001768 <_ZN13FastMathClass4isinEl>
 800137a:	eef0 7a40 	vmov.f32	s15, s0
 800137e:	eeb1 7a67 	vneg.f32	s14, s15
 8001382:	f8b7 3074 	ldrh.w	r3, [r7, #116]	; 0x74
 8001386:	ee07 3a90 	vmov	s15, r3
 800138a:	eef8 7ae7 	vcvt.f32.s32	s15, s15
 800138e:	ee27 7a27 	vmul.f32	s14, s14, s15
 8001392:	687b      	ldr	r3, [r7, #4]
 8001394:	891b      	ldrh	r3, [r3, #8]
 8001396:	ee07 3a90 	vmov	s15, r3
 800139a:	eef8 7ae7 	vcvt.f32.s32	s15, s15
 800139e:	ee77 7a27 	vadd.f32	s15, s14, s15
 80013a2:	eefd 7ae7 	vcvt.s32.f32	s15, s15
 80013a6:	ee17 3a90 	vmov	r3, s15
 80013aa:	b21a      	sxth	r2, r3
 80013ac:	f897 3073 	ldrb.w	r3, [r7, #115]	; 0x73
 80013b0:	b219      	sxth	r1, r3
 80013b2:	2300      	movs	r3, #0
 80013b4:	9300      	str	r3, [sp, #0]
 80013b6:	460b      	mov	r3, r1
 80013b8:	4621      	mov	r1, r4
 80013ba:	485b      	ldr	r0, [pc, #364]	; (8001528 <_ZN7Display9drawShapeENS_7Shape_tEtPv+0x9e8>)
 80013bc:	f000 fe59 	bl	8002072 <_ZN8Graphics10fillCircleEssst>
            {
                g_Graphics.fillCircle((icos(i+angle_trig)*arcRadius)+((ShapeArc_t *)argp)->x, (-isin(i+angle_trig)*arcRadius)+((ShapeArc_t *)argp)->y,cirRadius,0);
                g_Graphics.fillCircle((icos(angle_trig-i)*arcRadius)+((ShapeArc_t *)argp)->x, (-isin(angle_trig-i)*arcRadius)+((ShapeArc_t *)argp)->y,cirRadius,0);
            }
        }
        break;
 80013c0:	e0ab      	b.n	800151a <_ZN7Display9drawShapeENS_7Shape_tEtPv+0x9da>
            for (uint16_t i = 1 ; i <= spreadAngle ; i++)
 80013c2:	2301      	movs	r3, #1
 80013c4:	f8a7 307c 	strh.w	r3, [r7, #124]	; 0x7c
 80013c8:	f8b7 207c 	ldrh.w	r2, [r7, #124]	; 0x7c
 80013cc:	f8b7 307a 	ldrh.w	r3, [r7, #122]	; 0x7a
 80013d0:	429a      	cmp	r2, r3
 80013d2:	f200 80a2 	bhi.w	800151a <_ZN7Display9drawShapeENS_7Shape_tEtPv+0x9da>
                g_Graphics.fillCircle((icos(i+angle_trig)*arcRadius)+((ShapeArc_t *)argp)->x, (-isin(i+angle_trig)*arcRadius)+((ShapeArc_t *)argp)->y,cirRadius,0);
 80013d6:	68f8      	ldr	r0, [r7, #12]
 80013d8:	f8b7 207c 	ldrh.w	r2, [r7, #124]	; 0x7c
 80013dc:	f8b7 3076 	ldrh.w	r3, [r7, #118]	; 0x76
 80013e0:	4413      	add	r3, r2
 80013e2:	4619      	mov	r1, r3
 80013e4:	f000 fa36 	bl	8001854 <_ZN13FastMathClass4icosEl>
 80013e8:	eeb0 7a40 	vmov.f32	s14, s0
 80013ec:	f8b7 3074 	ldrh.w	r3, [r7, #116]	; 0x74
 80013f0:	ee07 3a90 	vmov	s15, r3
 80013f4:	eef8 7ae7 	vcvt.f32.s32	s15, s15
 80013f8:	ee27 7a27 	vmul.f32	s14, s14, s15
 80013fc:	687b      	ldr	r3, [r7, #4]
 80013fe:	88db      	ldrh	r3, [r3, #6]
 8001400:	ee07 3a90 	vmov	s15, r3
 8001404:	eef8 7ae7 	vcvt.f32.s32	s15, s15
 8001408:	ee77 7a27 	vadd.f32	s15, s14, s15
 800140c:	eefd 7ae7 	vcvt.s32.f32	s15, s15
 8001410:	ee17 3a90 	vmov	r3, s15
 8001414:	b21c      	sxth	r4, r3
 8001416:	68f8      	ldr	r0, [r7, #12]
 8001418:	f8b7 207c 	ldrh.w	r2, [r7, #124]	; 0x7c
 800141c:	f8b7 3076 	ldrh.w	r3, [r7, #118]	; 0x76
 8001420:	4413      	add	r3, r2
 8001422:	4619      	mov	r1, r3
 8001424:	f000 f9a0 	bl	8001768 <_ZN13FastMathClass4isinEl>
 8001428:	eef0 7a40 	vmov.f32	s15, s0
 800142c:	eeb1 7a67 	vneg.f32	s14, s15
 8001430:	f8b7 3074 	ldrh.w	r3, [r7, #116]	; 0x74
 8001434:	ee07 3a90 	vmov	s15, r3
 8001438:	eef8 7ae7 	vcvt.f32.s32	s15, s15
 800143c:	ee27 7a27 	vmul.f32	s14, s14, s15
 8001440:	687b      	ldr	r3, [r7, #4]
 8001442:	891b      	ldrh	r3, [r3, #8]
 8001444:	ee07 3a90 	vmov	s15, r3
 8001448:	eef8 7ae7 	vcvt.f32.s32	s15, s15
 800144c:	ee77 7a27 	vadd.f32	s15, s14, s15
 8001450:	eefd 7ae7 	vcvt.s32.f32	s15, s15
 8001454:	ee17 3a90 	vmov	r3, s15
 8001458:	b21a      	sxth	r2, r3
 800145a:	f897 3073 	ldrb.w	r3, [r7, #115]	; 0x73
 800145e:	b219      	sxth	r1, r3
 8001460:	2300      	movs	r3, #0
 8001462:	9300      	str	r3, [sp, #0]
 8001464:	460b      	mov	r3, r1
 8001466:	4621      	mov	r1, r4
 8001468:	482f      	ldr	r0, [pc, #188]	; (8001528 <_ZN7Display9drawShapeENS_7Shape_tEtPv+0x9e8>)
 800146a:	f000 fe02 	bl	8002072 <_ZN8Graphics10fillCircleEssst>
                g_Graphics.fillCircle((icos(angle_trig-i)*arcRadius)+((ShapeArc_t *)argp)->x, (-isin(angle_trig-i)*arcRadius)+((ShapeArc_t *)argp)->y,cirRadius,0);
 800146e:	68f8      	ldr	r0, [r7, #12]
 8001470:	f8b7 2076 	ldrh.w	r2, [r7, #118]	; 0x76
 8001474:	f8b7 307c 	ldrh.w	r3, [r7, #124]	; 0x7c
 8001478:	1ad3      	subs	r3, r2, r3
 800147a:	4619      	mov	r1, r3
 800147c:	f000 f9ea 	bl	8001854 <_ZN13FastMathClass4icosEl>
 8001480:	eeb0 7a40 	vmov.f32	s14, s0
 8001484:	f8b7 3074 	ldrh.w	r3, [r7, #116]	; 0x74
 8001488:	ee07 3a90 	vmov	s15, r3
 800148c:	eef8 7ae7 	vcvt.f32.s32	s15, s15
 8001490:	ee27 7a27 	vmul.f32	s14, s14, s15
 8001494:	687b      	ldr	r3, [r7, #4]
 8001496:	88db      	ldrh	r3, [r3, #6]
 8001498:	ee07 3a90 	vmov	s15, r3
 800149c:	eef8 7ae7 	vcvt.f32.s32	s15, s15
 80014a0:	ee77 7a27 	vadd.f32	s15, s14, s15
 80014a4:	eefd 7ae7 	vcvt.s32.f32	s15, s15
 80014a8:	ee17 3a90 	vmov	r3, s15
 80014ac:	b21c      	sxth	r4, r3
 80014ae:	68f8      	ldr	r0, [r7, #12]
 80014b0:	f8b7 2076 	ldrh.w	r2, [r7, #118]	; 0x76
 80014b4:	f8b7 307c 	ldrh.w	r3, [r7, #124]	; 0x7c
 80014b8:	1ad3      	subs	r3, r2, r3
 80014ba:	4619      	mov	r1, r3
 80014bc:	f000 f954 	bl	8001768 <_ZN13FastMathClass4isinEl>
 80014c0:	eef0 7a40 	vmov.f32	s15, s0
 80014c4:	eeb1 7a67 	vneg.f32	s14, s15
 80014c8:	f8b7 3074 	ldrh.w	r3, [r7, #116]	; 0x74
 80014cc:	ee07 3a90 	vmov	s15, r3
 80014d0:	eef8 7ae7 	vcvt.f32.s32	s15, s15
 80014d4:	ee27 7a27 	vmul.f32	s14, s14, s15
 80014d8:	687b      	ldr	r3, [r7, #4]
 80014da:	891b      	ldrh	r3, [r3, #8]
 80014dc:	ee07 3a90 	vmov	s15, r3
 80014e0:	eef8 7ae7 	vcvt.f32.s32	s15, s15
 80014e4:	ee77 7a27 	vadd.f32	s15, s14, s15
 80014e8:	eefd 7ae7 	vcvt.s32.f32	s15, s15
 80014ec:	ee17 3a90 	vmov	r3, s15
 80014f0:	b21a      	sxth	r2, r3
 80014f2:	f897 3073 	ldrb.w	r3, [r7, #115]	; 0x73
 80014f6:	b219      	sxth	r1, r3
 80014f8:	2300      	movs	r3, #0
 80014fa:	9300      	str	r3, [sp, #0]
 80014fc:	460b      	mov	r3, r1
 80014fe:	4621      	mov	r1, r4
 8001500:	4809      	ldr	r0, [pc, #36]	; (8001528 <_ZN7Display9drawShapeENS_7Shape_tEtPv+0x9e8>)
 8001502:	f000 fdb6 	bl	8002072 <_ZN8Graphics10fillCircleEssst>
            for (uint16_t i = 1 ; i <= spreadAngle ; i++)
 8001506:	f8b7 307c 	ldrh.w	r3, [r7, #124]	; 0x7c
 800150a:	3301      	adds	r3, #1
 800150c:	f8a7 307c 	strh.w	r3, [r7, #124]	; 0x7c
 8001510:	e75a      	b.n	80013c8 <_ZN7Display9drawShapeENS_7Shape_tEtPv+0x888>
    }
    default:
    {
        break;
 8001512:	bf00      	nop
 8001514:	e002      	b.n	800151c <_ZN7Display9drawShapeENS_7Shape_tEtPv+0x9dc>
        break;
 8001516:	bf00      	nop
 8001518:	e000      	b.n	800151c <_ZN7Display9drawShapeENS_7Shape_tEtPv+0x9dc>
        break;
 800151a:	bf00      	nop
    }
    }
}
 800151c:	bf00      	nop
 800151e:	3784      	adds	r7, #132	; 0x84
 8001520:	46bd      	mov	sp, r7
 8001522:	bdf0      	pop	{r4, r5, r6, r7, pc}
 8001524:	b60b60b7 	.word	0xb60b60b7
 8001528:	200000a8 	.word	0x200000a8

0800152c <_ZN7Display13getDisplayPtrEt>:
   TODO: Possibly move this to the graphics module.

 */
/**************************************************************************/
uint8_t*  Display::getDisplayPtr(uint16_t index)
{
 800152c:	b580      	push	{r7, lr}
 800152e:	b082      	sub	sp, #8
 8001530:	af00      	add	r7, sp, #0
 8001532:	6078      	str	r0, [r7, #4]
 8001534:	460b      	mov	r3, r1
 8001536:	807b      	strh	r3, [r7, #2]
    if ((index < 0) || (index > BUFFER_SIZE))
 8001538:	887b      	ldrh	r3, [r7, #2]
 800153a:	f242 3282 	movw	r2, #9090	; 0x2382
 800153e:	4293      	cmp	r3, r2
 8001540:	d901      	bls.n	8001546 <_ZN7Display13getDisplayPtrEt+0x1a>
        return NULL;
 8001542:	2300      	movs	r3, #0
 8001544:	e005      	b.n	8001552 <_ZN7Display13getDisplayPtrEt+0x26>

    return g_Graphics.getDisplayPtr(index);
 8001546:	887b      	ldrh	r3, [r7, #2]
 8001548:	4619      	mov	r1, r3
 800154a:	4804      	ldr	r0, [pc, #16]	; (800155c <_ZN7Display13getDisplayPtrEt+0x30>)
 800154c:	f001 fa6d 	bl	8002a2a <_ZN8Graphics13getDisplayPtrEt>
 8001550:	4603      	mov	r3, r0
}
 8001552:	4618      	mov	r0, r3
 8001554:	3708      	adds	r7, #8
 8001556:	46bd      	mov	sp, r7
 8001558:	bd80      	pop	{r7, pc}
 800155a:	bf00      	nop
 800155c:	200000a8 	.word	0x200000a8

08001560 <_Z41__static_initialization_and_destruction_0ii>:
/*!
   @brief    DISPLAY OBJECT
   @param    None
 */
/**************************************************************************/
Display g_Display = Display();
 8001560:	b580      	push	{r7, lr}
 8001562:	b082      	sub	sp, #8
 8001564:	af00      	add	r7, sp, #0
 8001566:	6078      	str	r0, [r7, #4]
 8001568:	6039      	str	r1, [r7, #0]
 800156a:	687b      	ldr	r3, [r7, #4]
 800156c:	2b01      	cmp	r3, #1
 800156e:	d107      	bne.n	8001580 <_Z41__static_initialization_and_destruction_0ii+0x20>
 8001570:	683b      	ldr	r3, [r7, #0]
 8001572:	f64f 72ff 	movw	r2, #65535	; 0xffff
 8001576:	4293      	cmp	r3, r2
 8001578:	d102      	bne.n	8001580 <_Z41__static_initialization_and_destruction_0ii+0x20>
 800157a:	4803      	ldr	r0, [pc, #12]	; (8001588 <_Z41__static_initialization_and_destruction_0ii+0x28>)
 800157c:	f7ff fa56 	bl	8000a2c <_ZN7DisplayC1Ev>
 8001580:	bf00      	nop
 8001582:	3708      	adds	r7, #8
 8001584:	46bd      	mov	sp, r7
 8001586:	bd80      	pop	{r7, pc}
 8001588:	20000038 	.word	0x20000038

0800158c <_GLOBAL__sub_I__ZN7DisplayC2Ev>:
 800158c:	b580      	push	{r7, lr}
 800158e:	af00      	add	r7, sp, #0
 8001590:	f64f 71ff 	movw	r1, #65535	; 0xffff
 8001594:	2001      	movs	r0, #1
 8001596:	f7ff ffe3 	bl	8001560 <_Z41__static_initialization_and_destruction_0ii>
 800159a:	bd80      	pop	{r7, pc}

0800159c <LynqGraphics_initDisplayLibrary>:

//***** API Functions definition *****//
//****Remember "API" is used like "public" in C++*******//

void LynqGraphics_initDisplayLibrary(void)
{
 800159c:	b580      	push	{r7, lr}
 800159e:	af00      	add	r7, sp, #0
	g_Display.initDisplay();
 80015a0:	4802      	ldr	r0, [pc, #8]	; (80015ac <LynqGraphics_initDisplayLibrary+0x10>)
 80015a2:	f7ff fa51 	bl	8000a48 <_ZN7Display11initDisplayEv>
}
 80015a6:	bf00      	nop
 80015a8:	bd80      	pop	{r7, pc}
 80015aa:	bf00      	nop
 80015ac:	20000038 	.word	0x20000038

080015b0 <LynqGraphics_getDisplayPtr>:

uint8_t* LynqGraphics_getDisplayPtr(uint16_t index)
{
 80015b0:	b580      	push	{r7, lr}
 80015b2:	b082      	sub	sp, #8
 80015b4:	af00      	add	r7, sp, #0
 80015b6:	4603      	mov	r3, r0
 80015b8:	80fb      	strh	r3, [r7, #6]
	return g_Display.getDisplayPtr(index);
 80015ba:	88fb      	ldrh	r3, [r7, #6]
 80015bc:	4619      	mov	r1, r3
 80015be:	4804      	ldr	r0, [pc, #16]	; (80015d0 <LynqGraphics_getDisplayPtr+0x20>)
 80015c0:	f7ff ffb4 	bl	800152c <_ZN7Display13getDisplayPtrEt>
 80015c4:	4603      	mov	r3, r0
}
 80015c6:	4618      	mov	r0, r3
 80015c8:	3708      	adds	r7, #8
 80015ca:	46bd      	mov	sp, r7
 80015cc:	bd80      	pop	{r7, pc}
 80015ce:	bf00      	nop
 80015d0:	20000038 	.word	0x20000038

080015d4 <LynqGraphics_drawShapeCircle>:

	g_Display.drawShape(Display::Shape_t::SHAPE_Point, color, (void*)&pointCoord);
}

void LynqGraphics_drawShapeCircle(uint16_t color, int16_t x, int16_t y, uint16_t radius)
{
 80015d4:	b590      	push	{r4, r7, lr}
 80015d6:	b085      	sub	sp, #20
 80015d8:	af00      	add	r7, sp, #0
 80015da:	4604      	mov	r4, r0
 80015dc:	4608      	mov	r0, r1
 80015de:	4611      	mov	r1, r2
 80015e0:	461a      	mov	r2, r3
 80015e2:	4623      	mov	r3, r4
 80015e4:	80fb      	strh	r3, [r7, #6]
 80015e6:	4603      	mov	r3, r0
 80015e8:	80bb      	strh	r3, [r7, #4]
 80015ea:	460b      	mov	r3, r1
 80015ec:	807b      	strh	r3, [r7, #2]
 80015ee:	4613      	mov	r3, r2
 80015f0:	803b      	strh	r3, [r7, #0]
		uint16_t y;
		uint16_t radius;

	}circleCoord;

	circleCoord.x = x;
 80015f2:	88bb      	ldrh	r3, [r7, #4]
 80015f4:	813b      	strh	r3, [r7, #8]
	circleCoord.y = y;
 80015f6:	887b      	ldrh	r3, [r7, #2]
 80015f8:	817b      	strh	r3, [r7, #10]
	circleCoord.radius = radius;
 80015fa:	883b      	ldrh	r3, [r7, #0]
 80015fc:	81bb      	strh	r3, [r7, #12]

	g_Display.drawShape(Display::Shape_t::SHAPE_Circle, color, (void*)&circleCoord);
 80015fe:	f107 0308 	add.w	r3, r7, #8
 8001602:	88fa      	ldrh	r2, [r7, #6]
 8001604:	2102      	movs	r1, #2
 8001606:	4803      	ldr	r0, [pc, #12]	; (8001614 <LynqGraphics_drawShapeCircle+0x40>)
 8001608:	f7ff fa9a 	bl	8000b40 <_ZN7Display9drawShapeENS_7Shape_tEtPv>
}
 800160c:	bf00      	nop
 800160e:	3714      	adds	r7, #20
 8001610:	46bd      	mov	sp, r7
 8001612:	bd90      	pop	{r4, r7, pc}
 8001614:	20000038 	.word	0x20000038

08001618 <LynqGraphics_drawShapeTriangle>:

void LynqGraphics_drawShapeTriangle(uint16_t color, int16_t firstX, int16_t firstY,
									   int16_t secondX, int16_t secondY,
									   int16_t thirdX, int16_t thirdY)
{
 8001618:	b590      	push	{r4, r7, lr}
 800161a:	b087      	sub	sp, #28
 800161c:	af00      	add	r7, sp, #0
 800161e:	4604      	mov	r4, r0
 8001620:	4608      	mov	r0, r1
 8001622:	4611      	mov	r1, r2
 8001624:	461a      	mov	r2, r3
 8001626:	4623      	mov	r3, r4
 8001628:	80fb      	strh	r3, [r7, #6]
 800162a:	4603      	mov	r3, r0
 800162c:	80bb      	strh	r3, [r7, #4]
 800162e:	460b      	mov	r3, r1
 8001630:	807b      	strh	r3, [r7, #2]
 8001632:	4613      	mov	r3, r2
 8001634:	803b      	strh	r3, [r7, #0]
		uint16_t thirdX;
		uint16_t thirdY;

	}triangleCoord;

	triangleCoord.firstX = firstX;
 8001636:	88bb      	ldrh	r3, [r7, #4]
 8001638:	81bb      	strh	r3, [r7, #12]
	triangleCoord.firstY = firstY;
 800163a:	887b      	ldrh	r3, [r7, #2]
 800163c:	81fb      	strh	r3, [r7, #14]
	triangleCoord.secondX = secondX;
 800163e:	883b      	ldrh	r3, [r7, #0]
 8001640:	823b      	strh	r3, [r7, #16]
	triangleCoord.secondY = secondY;
 8001642:	8d3b      	ldrh	r3, [r7, #40]	; 0x28
 8001644:	827b      	strh	r3, [r7, #18]
	triangleCoord.thirdX = thirdX;
 8001646:	8dbb      	ldrh	r3, [r7, #44]	; 0x2c
 8001648:	82bb      	strh	r3, [r7, #20]
	triangleCoord.thirdY = thirdY;
 800164a:	8e3b      	ldrh	r3, [r7, #48]	; 0x30
 800164c:	82fb      	strh	r3, [r7, #22]

	g_Display.drawShape(Display::Shape_t::SHAPE_Triangle, color, (void*)&triangleCoord);
 800164e:	f107 030c 	add.w	r3, r7, #12
 8001652:	88fa      	ldrh	r2, [r7, #6]
 8001654:	2103      	movs	r1, #3
 8001656:	4803      	ldr	r0, [pc, #12]	; (8001664 <LynqGraphics_drawShapeTriangle+0x4c>)
 8001658:	f7ff fa72 	bl	8000b40 <_ZN7Display9drawShapeENS_7Shape_tEtPv>
}
 800165c:	bf00      	nop
 800165e:	371c      	adds	r7, #28
 8001660:	46bd      	mov	sp, r7
 8001662:	bd90      	pop	{r4, r7, pc}
 8001664:	20000038 	.word	0x20000038

08001668 <LynqGraphics_drawShapeFillRoundRect>:

	g_Display.drawShape(Display::Shape_t::SHAPE_FillRect, color, (void*)&fillRectCoord);
}

void LynqGraphics_drawShapeFillRoundRect(uint16_t color, int16_t x, int16_t y, int16_t width, int16_t height)
{
 8001668:	b590      	push	{r4, r7, lr}
 800166a:	b085      	sub	sp, #20
 800166c:	af00      	add	r7, sp, #0
 800166e:	4604      	mov	r4, r0
 8001670:	4608      	mov	r0, r1
 8001672:	4611      	mov	r1, r2
 8001674:	461a      	mov	r2, r3
 8001676:	4623      	mov	r3, r4
 8001678:	80fb      	strh	r3, [r7, #6]
 800167a:	4603      	mov	r3, r0
 800167c:	80bb      	strh	r3, [r7, #4]
 800167e:	460b      	mov	r3, r1
 8001680:	807b      	strh	r3, [r7, #2]
 8001682:	4613      	mov	r3, r2
 8001684:	803b      	strh	r3, [r7, #0]
		uint16_t width;
		uint16_t height;

	}fillRoundRectCoord;

	fillRoundRectCoord.x = x;
 8001686:	88bb      	ldrh	r3, [r7, #4]
 8001688:	813b      	strh	r3, [r7, #8]
	fillRoundRectCoord.y = y;
 800168a:	887b      	ldrh	r3, [r7, #2]
 800168c:	817b      	strh	r3, [r7, #10]
	fillRoundRectCoord.width = width;
 800168e:	883b      	ldrh	r3, [r7, #0]
 8001690:	81bb      	strh	r3, [r7, #12]
	fillRoundRectCoord.height = height;
 8001692:	8c3b      	ldrh	r3, [r7, #32]
 8001694:	81fb      	strh	r3, [r7, #14]

	g_Display.drawShape(Display::Shape_t::SHAPE_FillRoundRect, color, (void*)&fillRoundRectCoord);
 8001696:	f107 0308 	add.w	r3, r7, #8
 800169a:	88fa      	ldrh	r2, [r7, #6]
 800169c:	2106      	movs	r1, #6
 800169e:	4803      	ldr	r0, [pc, #12]	; (80016ac <LynqGraphics_drawShapeFillRoundRect+0x44>)
 80016a0:	f7ff fa4e 	bl	8000b40 <_ZN7Display9drawShapeENS_7Shape_tEtPv>
}
 80016a4:	bf00      	nop
 80016a6:	3714      	adds	r7, #20
 80016a8:	46bd      	mov	sp, r7
 80016aa:	bd90      	pop	{r4, r7, pc}
 80016ac:	20000038 	.word	0x20000038

080016b0 <LynqGraphics_drawShapeBoldArc>:

	g_Display.drawShape(Display::Shape_t::SHAPE_Arrow, color, (void*)&arrowCoord);
}

void LynqGraphics_drawShapeBoldArc(uint16_t color, int16_t x, int16_t y, int16_t radius, int16_t heading, int16_t arcLength)
{
 80016b0:	b590      	push	{r4, r7, lr}
 80016b2:	b087      	sub	sp, #28
 80016b4:	af00      	add	r7, sp, #0
 80016b6:	4604      	mov	r4, r0
 80016b8:	4608      	mov	r0, r1
 80016ba:	4611      	mov	r1, r2
 80016bc:	461a      	mov	r2, r3
 80016be:	4623      	mov	r3, r4
 80016c0:	80fb      	strh	r3, [r7, #6]
 80016c2:	4603      	mov	r3, r0
 80016c4:	80bb      	strh	r3, [r7, #4]
 80016c6:	460b      	mov	r3, r1
 80016c8:	807b      	strh	r3, [r7, #2]
 80016ca:	4613      	mov	r3, r2
 80016cc:	803b      	strh	r3, [r7, #0]
		uint16_t x;
		uint16_t y;

	}boldArcCoord;

	boldArcCoord.radius = radius;
 80016ce:	883b      	ldrh	r3, [r7, #0]
 80016d0:	81bb      	strh	r3, [r7, #12]
    boldArcCoord.heading = heading;
 80016d2:	8d3b      	ldrh	r3, [r7, #40]	; 0x28
 80016d4:	81fb      	strh	r3, [r7, #14]
    boldArcCoord.arcLength = arcLength;
 80016d6:	8dbb      	ldrh	r3, [r7, #44]	; 0x2c
 80016d8:	823b      	strh	r3, [r7, #16]
    boldArcCoord.x = x;
 80016da:	88bb      	ldrh	r3, [r7, #4]
 80016dc:	827b      	strh	r3, [r7, #18]
    boldArcCoord.y = y;
 80016de:	887b      	ldrh	r3, [r7, #2]
 80016e0:	82bb      	strh	r3, [r7, #20]

	g_Display.drawShape(Display::Shape_t::SHAPE_BoldArc, color, (void*)&boldArcCoord);
 80016e2:	f107 030c 	add.w	r3, r7, #12
 80016e6:	88fa      	ldrh	r2, [r7, #6]
 80016e8:	2109      	movs	r1, #9
 80016ea:	4803      	ldr	r0, [pc, #12]	; (80016f8 <LynqGraphics_drawShapeBoldArc+0x48>)
 80016ec:	f7ff fa28 	bl	8000b40 <_ZN7Display9drawShapeENS_7Shape_tEtPv>
}
 80016f0:	bf00      	nop
 80016f2:	371c      	adds	r7, #28
 80016f4:	46bd      	mov	sp, r7
 80016f6:	bd90      	pop	{r4, r7, pc}
 80016f8:	20000038 	.word	0x20000038

080016fc <LynqGraphics_writeStream>:

size_t  LynqGraphics_writeStream(const uint8_t *buffer, size_t size)
{
 80016fc:	b580      	push	{r7, lr}
 80016fe:	b082      	sub	sp, #8
 8001700:	af00      	add	r7, sp, #0
 8001702:	6078      	str	r0, [r7, #4]
 8001704:	6039      	str	r1, [r7, #0]
	return g_Display.writeStream(buffer, size);
 8001706:	683a      	ldr	r2, [r7, #0]
 8001708:	6879      	ldr	r1, [r7, #4]
 800170a:	4804      	ldr	r0, [pc, #16]	; (800171c <LynqGraphics_writeStream+0x20>)
 800170c:	f7ff f9f2 	bl	8000af4 <_ZN7Display11writeStreamEPKhj>
 8001710:	4603      	mov	r3, r0
}
 8001712:	4618      	mov	r0, r3
 8001714:	3708      	adds	r7, #8
 8001716:	46bd      	mov	sp, r7
 8001718:	bd80      	pop	{r7, pc}
 800171a:	bf00      	nop
 800171c:	20000038 	.word	0x20000038

08001720 <LynqGraphics_setCursorOffset>:
{
	g_Display.customTextposition(text, nameLen, x, y);
}

void LynqGraphics_setCursorOffset(uint16_t x, uint16_t y)
{
 8001720:	b580      	push	{r7, lr}
 8001722:	b082      	sub	sp, #8
 8001724:	af00      	add	r7, sp, #0
 8001726:	4603      	mov	r3, r0
 8001728:	460a      	mov	r2, r1
 800172a:	80fb      	strh	r3, [r7, #6]
 800172c:	4613      	mov	r3, r2
 800172e:	80bb      	strh	r3, [r7, #4]
	g_Display.setCursorOffset(x, y);
 8001730:	88ba      	ldrh	r2, [r7, #4]
 8001732:	88fb      	ldrh	r3, [r7, #6]
 8001734:	4619      	mov	r1, r3
 8001736:	4803      	ldr	r0, [pc, #12]	; (8001744 <LynqGraphics_setCursorOffset+0x24>)
 8001738:	f7ff f9b6 	bl	8000aa8 <_ZN7Display15setCursorOffsetEtt>
}
 800173c:	bf00      	nop
 800173e:	3708      	adds	r7, #8
 8001740:	46bd      	mov	sp, r7
 8001742:	bd80      	pop	{r7, pc}
 8001744:	20000038 	.word	0x20000038

08001748 <LynqGraphics_setLineNum>:

void LynqGraphics_setLineNum(uint8_t lineNum)
{
 8001748:	b580      	push	{r7, lr}
 800174a:	b082      	sub	sp, #8
 800174c:	af00      	add	r7, sp, #0
 800174e:	4603      	mov	r3, r0
 8001750:	71fb      	strb	r3, [r7, #7]
	g_Display.setLineNum(lineNum);
 8001752:	79fb      	ldrb	r3, [r7, #7]
 8001754:	4619      	mov	r1, r3
 8001756:	4803      	ldr	r0, [pc, #12]	; (8001764 <LynqGraphics_setLineNum+0x1c>)
 8001758:	f7ff f9bc 	bl	8000ad4 <_ZN7Display10setLineNumEh>
}
 800175c:	bf00      	nop
 800175e:	3708      	adds	r7, #8
 8001760:	46bd      	mov	sp, r7
 8001762:	bd80      	pop	{r7, pc}
 8001764:	20000038 	.word	0x20000038

08001768 <_ZN13FastMathClass4isinEl>:
#include "fast_math.h"


/* Calcluates sin(Theta) */
float FastMathClass::isin(long x)
{
 8001768:	b590      	push	{r4, r7, lr}
 800176a:	b085      	sub	sp, #20
 800176c:	af00      	add	r7, sp, #0
 800176e:	6078      	str	r0, [r7, #4]
 8001770:	6039      	str	r1, [r7, #0]
  bool pos = true;  /* positive - keeps an eye on the sign. */
 8001772:	2301      	movs	r3, #1
 8001774:	60fb      	str	r3, [r7, #12]

  if (x < 0)
 8001776:	683b      	ldr	r3, [r7, #0]
 8001778:	2b00      	cmp	r3, #0
 800177a:	da09      	bge.n	8001790 <_ZN13FastMathClass4isinEl+0x28>
  {
    x = -x;
 800177c:	683b      	ldr	r3, [r7, #0]
 800177e:	425b      	negs	r3, r3
 8001780:	603b      	str	r3, [r7, #0]
    pos = !pos;
 8001782:	68fb      	ldr	r3, [r7, #12]
 8001784:	2b00      	cmp	r3, #0
 8001786:	bf0c      	ite	eq
 8001788:	2301      	moveq	r3, #1
 800178a:	2300      	movne	r3, #0
 800178c:	b2db      	uxtb	r3, r3
 800178e:	60fb      	str	r3, [r7, #12]
  }

  if (x >= 360) x %= 360;
 8001790:	683b      	ldr	r3, [r7, #0]
 8001792:	f5b3 7fb4 	cmp.w	r3, #360	; 0x168
 8001796:	db0d      	blt.n	80017b4 <_ZN13FastMathClass4isinEl+0x4c>
 8001798:	683b      	ldr	r3, [r7, #0]
 800179a:	4a2d      	ldr	r2, [pc, #180]	; (8001850 <_ZN13FastMathClass4isinEl+0xe8>)
 800179c:	fb82 1203 	smull	r1, r2, r2, r3
 80017a0:	441a      	add	r2, r3
 80017a2:	1211      	asrs	r1, r2, #8
 80017a4:	17da      	asrs	r2, r3, #31
 80017a6:	1a8a      	subs	r2, r1, r2
 80017a8:	f44f 71b4 	mov.w	r1, #360	; 0x168
 80017ac:	fb01 f202 	mul.w	r2, r1, r2
 80017b0:	1a9b      	subs	r3, r3, r2
 80017b2:	603b      	str	r3, [r7, #0]

  if (x > 180)
 80017b4:	683b      	ldr	r3, [r7, #0]
 80017b6:	2bb4      	cmp	r3, #180	; 0xb4
 80017b8:	dd09      	ble.n	80017ce <_ZN13FastMathClass4isinEl+0x66>
  {
    x -= 180;
 80017ba:	683b      	ldr	r3, [r7, #0]
 80017bc:	3bb4      	subs	r3, #180	; 0xb4
 80017be:	603b      	str	r3, [r7, #0]
    pos = !pos;
 80017c0:	68fb      	ldr	r3, [r7, #12]
 80017c2:	2b00      	cmp	r3, #0
 80017c4:	bf0c      	ite	eq
 80017c6:	2301      	moveq	r3, #1
 80017c8:	2300      	movne	r3, #0
 80017ca:	b2db      	uxtb	r3, r3
 80017cc:	60fb      	str	r3, [r7, #12]
  }

  if (x > 90) x = 180 - x;
 80017ce:	683b      	ldr	r3, [r7, #0]
 80017d0:	2b5a      	cmp	r3, #90	; 0x5a
 80017d2:	dd03      	ble.n	80017dc <_ZN13FastMathClass4isinEl+0x74>
 80017d4:	683b      	ldr	r3, [r7, #0]
 80017d6:	f1c3 03b4 	rsb	r3, r3, #180	; 0xb4
 80017da:	603b      	str	r3, [r7, #0]

#ifdef TABLE_PERCISION_16_BIT
  if (pos) return iSinTable16[x] * 0.0000152590219; // = /65535.0
  return isinTable16[x] * -0.0000152590219 ;
#else
  if (pos) return iSinTable8[x] * 0.003921568627; // = /255.0
 80017dc:	68fb      	ldr	r3, [r7, #12]
 80017de:	2b00      	cmp	r3, #0
 80017e0:	d013      	beq.n	800180a <_ZN13FastMathClass4isinEl+0xa2>
 80017e2:	687a      	ldr	r2, [r7, #4]
 80017e4:	683b      	ldr	r3, [r7, #0]
 80017e6:	4413      	add	r3, r2
 80017e8:	781b      	ldrb	r3, [r3, #0]
 80017ea:	4618      	mov	r0, r3
 80017ec:	f7fe fe3e 	bl	800046c <__aeabi_i2d>
 80017f0:	a313      	add	r3, pc, #76	; (adr r3, 8001840 <_ZN13FastMathClass4isinEl+0xd8>)
 80017f2:	e9d3 2300 	ldrd	r2, r3, [r3]
 80017f6:	f7fe fea3 	bl	8000540 <__aeabi_dmul>
 80017fa:	4603      	mov	r3, r0
 80017fc:	460c      	mov	r4, r1
 80017fe:	4618      	mov	r0, r3
 8001800:	4621      	mov	r1, r4
 8001802:	f7ff f8af 	bl	8000964 <__aeabi_d2f>
 8001806:	4603      	mov	r3, r0
 8001808:	e012      	b.n	8001830 <_ZN13FastMathClass4isinEl+0xc8>
  return iSinTable8[x] * -0.003921568627 ;
 800180a:	687a      	ldr	r2, [r7, #4]
 800180c:	683b      	ldr	r3, [r7, #0]
 800180e:	4413      	add	r3, r2
 8001810:	781b      	ldrb	r3, [r3, #0]
 8001812:	4618      	mov	r0, r3
 8001814:	f7fe fe2a 	bl	800046c <__aeabi_i2d>
 8001818:	a30b      	add	r3, pc, #44	; (adr r3, 8001848 <_ZN13FastMathClass4isinEl+0xe0>)
 800181a:	e9d3 2300 	ldrd	r2, r3, [r3]
 800181e:	f7fe fe8f 	bl	8000540 <__aeabi_dmul>
 8001822:	4603      	mov	r3, r0
 8001824:	460c      	mov	r4, r1
 8001826:	4618      	mov	r0, r3
 8001828:	4621      	mov	r1, r4
 800182a:	f7ff f89b 	bl	8000964 <__aeabi_d2f>
 800182e:	4603      	mov	r3, r0
 8001830:	ee07 3a90 	vmov	s15, r3
#endif
}
 8001834:	eeb0 0a67 	vmov.f32	s0, s15
 8001838:	3714      	adds	r7, #20
 800183a:	46bd      	mov	sp, r7
 800183c:	bd90      	pop	{r4, r7, pc}
 800183e:	bf00      	nop
 8001840:	10082107 	.word	0x10082107
 8001844:	3f701010 	.word	0x3f701010
 8001848:	10082107 	.word	0x10082107
 800184c:	bf701010 	.word	0xbf701010
 8001850:	b60b60b7 	.word	0xb60b60b7

08001854 <_ZN13FastMathClass4icosEl>:

/* Calcluates cos(Theta) */
float FastMathClass::icos(long x)
{
 8001854:	b580      	push	{r7, lr}
 8001856:	b082      	sub	sp, #8
 8001858:	af00      	add	r7, sp, #0
 800185a:	6078      	str	r0, [r7, #4]
 800185c:	6039      	str	r1, [r7, #0]
  return isin(x+90);
 800185e:	683b      	ldr	r3, [r7, #0]
 8001860:	335a      	adds	r3, #90	; 0x5a
 8001862:	4619      	mov	r1, r3
 8001864:	6878      	ldr	r0, [r7, #4]
 8001866:	f7ff ff7f 	bl	8001768 <_ZN13FastMathClass4isinEl>
 800186a:	eef0 7a40 	vmov.f32	s15, s0
}
 800186e:	eeb0 0a67 	vmov.f32	s0, s15
 8001872:	3708      	adds	r7, #8
 8001874:	46bd      	mov	sp, r7
 8001876:	bd80      	pop	{r7, pc}

08001878 <_ZN8Graphics12initGraphicsEv>:
    @brief Initializes the graphics dimentions, font and cursors
    @param  None
*/
/**************************************************************************/
void Graphics::initGraphics()
{
 8001878:	b580      	push	{r7, lr}
 800187a:	b082      	sub	sp, #8
 800187c:	af00      	add	r7, sp, #0
 800187e:	6078      	str	r0, [r7, #4]
  /* TODO: add #defines to this */

  m_invertDisplayFlag = true;
 8001880:	687b      	ldr	r3, [r7, #4]
 8001882:	f503 530e 	add.w	r3, r3, #9088	; 0x2380
 8001886:	3314      	adds	r3, #20
 8001888:	2201      	movs	r2, #1
 800188a:	601a      	str	r2, [r3, #0]
  m_widthSize = SCREENDIMENSIONSWIDTH;
 800188c:	687b      	ldr	r3, [r7, #4]
 800188e:	f503 530e 	add.w	r3, r3, #9088	; 0x2380
 8001892:	3302      	adds	r3, #2
 8001894:	22f0      	movs	r2, #240	; 0xf0
 8001896:	801a      	strh	r2, [r3, #0]
  m_heightSize = SCREENDIMENSIONSHEIGHT;
 8001898:	687b      	ldr	r3, [r7, #4]
 800189a:	f503 530e 	add.w	r3, r3, #9088	; 0x2380
 800189e:	3304      	adds	r3, #4
 80018a0:	f240 122f 	movw	r2, #303	; 0x12f
 80018a4:	801a      	strh	r2, [r3, #0]
  setCursor(0, 0);
 80018a6:	2200      	movs	r2, #0
 80018a8:	2100      	movs	r1, #0
 80018aa:	6878      	ldr	r0, [r7, #4]
 80018ac:	f001 f815 	bl	80028da <_ZN8Graphics9setCursorEss>
  setBuffer();
 80018b0:	6878      	ldr	r0, [r7, #4]
 80018b2:	f001 f8ab 	bl	8002a0c <_ZN8Graphics9setBufferEv>

  /* Initialize the basic font structure */
//  setFont(&Ariblk14pt7b);
  setFont(&Silom12pt7b);
 80018b6:	4908      	ldr	r1, [pc, #32]	; (80018d8 <_ZN8Graphics12initGraphicsEv+0x60>)
 80018b8:	6878      	ldr	r0, [r7, #4]
 80018ba:	f000 f80f 	bl	80018dc <_ZN8Graphics7setFontEPKNS_8GFX_FONTE>
  setCursor(20, 50);
 80018be:	2232      	movs	r2, #50	; 0x32
 80018c0:	2114      	movs	r1, #20
 80018c2:	6878      	ldr	r0, [r7, #4]
 80018c4:	f001 f809 	bl	80028da <_ZN8Graphics9setCursorEss>
  setTextSize(1);
 80018c8:	2101      	movs	r1, #1
 80018ca:	6878      	ldr	r0, [r7, #4]
 80018cc:	f001 f81f 	bl	800290e <_ZN8Graphics11setTextSizeEh>
}
 80018d0:	bf00      	nop
 80018d2:	3708      	adds	r7, #8
 80018d4:	46bd      	mov	sp, r7
 80018d6:	bd80      	pop	{r7, pc}
 80018d8:	0800754c 	.word	0x0800754c

080018dc <_ZN8Graphics7setFontEPKNS_8GFX_FONTE>:
    @brief Set the font to display when print()ing, either custom or default
    @param  f  The GFXfont object, if NULL use built in 6x8 font
*/
/**************************************************************************/
void Graphics::setFont(const GFX_FONT *f)
{
 80018dc:	b480      	push	{r7}
 80018de:	b083      	sub	sp, #12
 80018e0:	af00      	add	r7, sp, #0
 80018e2:	6078      	str	r0, [r7, #4]
 80018e4:	6039      	str	r1, [r7, #0]
  if(f)
 80018e6:	683b      	ldr	r3, [r7, #0]
 80018e8:	2b00      	cmp	r3, #0
 80018ea:	d016      	beq.n	800191a <_ZN8Graphics7setFontEPKNS_8GFX_FONTE+0x3e>
  {
    if(!m_gfxFontPtr)
 80018ec:	687b      	ldr	r3, [r7, #4]
 80018ee:	f503 530e 	add.w	r3, r3, #9088	; 0x2380
 80018f2:	3318      	adds	r3, #24
 80018f4:	681b      	ldr	r3, [r3, #0]
 80018f6:	2b00      	cmp	r3, #0
 80018f8:	d125      	bne.n	8001946 <_ZN8Graphics7setFontEPKNS_8GFX_FONTE+0x6a>
    {
      m_cursorY += 6;
 80018fa:	687b      	ldr	r3, [r7, #4]
 80018fc:	f503 530e 	add.w	r3, r3, #9088	; 0x2380
 8001900:	3308      	adds	r3, #8
 8001902:	f9b3 3000 	ldrsh.w	r3, [r3]
 8001906:	b29b      	uxth	r3, r3
 8001908:	3306      	adds	r3, #6
 800190a:	b29b      	uxth	r3, r3
 800190c:	b21a      	sxth	r2, r3
 800190e:	687b      	ldr	r3, [r7, #4]
 8001910:	f503 530e 	add.w	r3, r3, #9088	; 0x2380
 8001914:	3308      	adds	r3, #8
 8001916:	801a      	strh	r2, [r3, #0]
 8001918:	e015      	b.n	8001946 <_ZN8Graphics7setFontEPKNS_8GFX_FONTE+0x6a>
    }
  }
  else if(m_gfxFontPtr)
 800191a:	687b      	ldr	r3, [r7, #4]
 800191c:	f503 530e 	add.w	r3, r3, #9088	; 0x2380
 8001920:	3318      	adds	r3, #24
 8001922:	681b      	ldr	r3, [r3, #0]
 8001924:	2b00      	cmp	r3, #0
 8001926:	d00e      	beq.n	8001946 <_ZN8Graphics7setFontEPKNS_8GFX_FONTE+0x6a>
  {
    // Move cursor pos up 6 pixels so it's at top-left of char.
    m_cursorY -= 6;
 8001928:	687b      	ldr	r3, [r7, #4]
 800192a:	f503 530e 	add.w	r3, r3, #9088	; 0x2380
 800192e:	3308      	adds	r3, #8
 8001930:	f9b3 3000 	ldrsh.w	r3, [r3]
 8001934:	b29b      	uxth	r3, r3
 8001936:	3b06      	subs	r3, #6
 8001938:	b29b      	uxth	r3, r3
 800193a:	b21a      	sxth	r2, r3
 800193c:	687b      	ldr	r3, [r7, #4]
 800193e:	f503 530e 	add.w	r3, r3, #9088	; 0x2380
 8001942:	3308      	adds	r3, #8
 8001944:	801a      	strh	r2, [r3, #0]
  }
  m_gfxFontPtr = (GFX_FONT *)f;
 8001946:	687b      	ldr	r3, [r7, #4]
 8001948:	f503 530e 	add.w	r3, r3, #9088	; 0x2380
 800194c:	3318      	adds	r3, #24
 800194e:	683a      	ldr	r2, [r7, #0]
 8001950:	601a      	str	r2, [r3, #0]
}
 8001952:	bf00      	nop
 8001954:	370c      	adds	r7, #12
 8001956:	46bd      	mov	sp, r7
 8001958:	f85d 7b04 	ldr.w	r7, [sp], #4
 800195c:	4770      	bx	lr
	...

08001960 <_ZN8Graphics9drawPixelEsst>:
    @param   y   y coordinate
   @param    color 0 - white 1 - black
*/
/**************************************************************************/
void Graphics::drawPixel(int16_t x, int16_t y, uint16_t color)
{
 8001960:	b580      	push	{r7, lr}
 8001962:	b086      	sub	sp, #24
 8001964:	af00      	add	r7, sp, #0
 8001966:	60f8      	str	r0, [r7, #12]
 8001968:	4608      	mov	r0, r1
 800196a:	4611      	mov	r1, r2
 800196c:	461a      	mov	r2, r3
 800196e:	4603      	mov	r3, r0
 8001970:	817b      	strh	r3, [r7, #10]
 8001972:	460b      	mov	r3, r1
 8001974:	813b      	strh	r3, [r7, #8]
 8001976:	4613      	mov	r3, r2
 8001978:	80fb      	strh	r3, [r7, #6]

  if((x < 0) || (x >= m_widthSize) || (y < 0) || (y >= m_heightSize)) return;
 800197a:	f9b7 300a 	ldrsh.w	r3, [r7, #10]
 800197e:	2b00      	cmp	r3, #0
 8001980:	db4e      	blt.n	8001a20 <_ZN8Graphics9drawPixelEsst+0xc0>
 8001982:	68fb      	ldr	r3, [r7, #12]
 8001984:	f503 530e 	add.w	r3, r3, #9088	; 0x2380
 8001988:	3302      	adds	r3, #2
 800198a:	f9b3 3000 	ldrsh.w	r3, [r3]
 800198e:	f9b7 200a 	ldrsh.w	r2, [r7, #10]
 8001992:	429a      	cmp	r2, r3
 8001994:	da44      	bge.n	8001a20 <_ZN8Graphics9drawPixelEsst+0xc0>
 8001996:	f9b7 3008 	ldrsh.w	r3, [r7, #8]
 800199a:	2b00      	cmp	r3, #0
 800199c:	db40      	blt.n	8001a20 <_ZN8Graphics9drawPixelEsst+0xc0>
 800199e:	68fb      	ldr	r3, [r7, #12]
 80019a0:	f503 530e 	add.w	r3, r3, #9088	; 0x2380
 80019a4:	3304      	adds	r3, #4
 80019a6:	f9b3 3000 	ldrsh.w	r3, [r3]
 80019aa:	f9b7 2008 	ldrsh.w	r2, [r7, #8]
 80019ae:	429a      	cmp	r2, r3
 80019b0:	da36      	bge.n	8001a20 <_ZN8Graphics9drawPixelEsst+0xc0>

#ifdef DEBUGLOW
  printf("x=%d,y=%d ",x,y);
#endif

  color = getColor(color);
 80019b2:	88fb      	ldrh	r3, [r7, #6]
 80019b4:	4619      	mov	r1, r3
 80019b6:	68f8      	ldr	r0, [r7, #12]
 80019b8:	f000 ffc0 	bl	800293c <_ZN8Graphics8getColorEt>
 80019bc:	4603      	mov	r3, r0
 80019be:	80fb      	strh	r3, [r7, #6]

#ifdef DEBUGLOW
  printf("%x\n",pgm_read_byte(&clr[x & 7]));
#endif

  uint16_t byte = ((y*SCREENDIMENSIONSWIDTH + x) / 8);
 80019c0:	f9b7 2008 	ldrsh.w	r2, [r7, #8]
 80019c4:	4613      	mov	r3, r2
 80019c6:	011b      	lsls	r3, r3, #4
 80019c8:	1a9b      	subs	r3, r3, r2
 80019ca:	011b      	lsls	r3, r3, #4
 80019cc:	461a      	mov	r2, r3
 80019ce:	f9b7 300a 	ldrsh.w	r3, [r7, #10]
 80019d2:	4413      	add	r3, r2
 80019d4:	2b00      	cmp	r3, #0
 80019d6:	da00      	bge.n	80019da <_ZN8Graphics9drawPixelEsst+0x7a>
 80019d8:	3307      	adds	r3, #7
 80019da:	10db      	asrs	r3, r3, #3
 80019dc:	82fb      	strh	r3, [r7, #22]

  if(color)
 80019de:	88fb      	ldrh	r3, [r7, #6]
 80019e0:	2b00      	cmp	r3, #0
 80019e2:	d00e      	beq.n	8001a02 <_ZN8Graphics9drawPixelEsst+0xa2>
  {
    m_displayBuffer[byte] |= pgm_read_byte(&set[x & 7]);
 80019e4:	8afb      	ldrh	r3, [r7, #22]
 80019e6:	68fa      	ldr	r2, [r7, #12]
 80019e8:	5cd1      	ldrb	r1, [r2, r3]
 80019ea:	897b      	ldrh	r3, [r7, #10]
 80019ec:	f003 0307 	and.w	r3, r3, #7
 80019f0:	4a0d      	ldr	r2, [pc, #52]	; (8001a28 <_ZN8Graphics9drawPixelEsst+0xc8>)
 80019f2:	4413      	add	r3, r2
 80019f4:	781a      	ldrb	r2, [r3, #0]
 80019f6:	8afb      	ldrh	r3, [r7, #22]
 80019f8:	430a      	orrs	r2, r1
 80019fa:	b2d1      	uxtb	r1, r2
 80019fc:	68fa      	ldr	r2, [r7, #12]
 80019fe:	54d1      	strb	r1, [r2, r3]
 8001a00:	e00f      	b.n	8001a22 <_ZN8Graphics9drawPixelEsst+0xc2>
  }
  else
  {
    m_displayBuffer[byte] &= pgm_read_byte(&clr[x & 7]);
 8001a02:	8afb      	ldrh	r3, [r7, #22]
 8001a04:	68fa      	ldr	r2, [r7, #12]
 8001a06:	5cd1      	ldrb	r1, [r2, r3]
 8001a08:	897b      	ldrh	r3, [r7, #10]
 8001a0a:	f003 0307 	and.w	r3, r3, #7
 8001a0e:	4a07      	ldr	r2, [pc, #28]	; (8001a2c <_ZN8Graphics9drawPixelEsst+0xcc>)
 8001a10:	4413      	add	r3, r2
 8001a12:	781a      	ldrb	r2, [r3, #0]
 8001a14:	8afb      	ldrh	r3, [r7, #22]
 8001a16:	400a      	ands	r2, r1
 8001a18:	b2d1      	uxtb	r1, r2
 8001a1a:	68fa      	ldr	r2, [r7, #12]
 8001a1c:	54d1      	strb	r1, [r2, r3]
 8001a1e:	e000      	b.n	8001a22 <_ZN8Graphics9drawPixelEsst+0xc2>
  if((x < 0) || (x >= m_widthSize) || (y < 0) || (y >= m_heightSize)) return;
 8001a20:	bf00      	nop
  }
#ifdef DEBUGLOW
  printf("\ndisplayBuffer=%d",m_displayBuffer[(y*SCREENDIMENSIONSWIDTH + x) / 8]);
#endif
}
 8001a22:	3718      	adds	r7, #24
 8001a24:	46bd      	mov	sp, r7
 8001a26:	bd80      	pop	{r7, pc}
 8001a28:	08007558 	.word	0x08007558
 8001a2c:	08007560 	.word	0x08007560

08001a30 <_ZN8Graphics5writeEh>:
    @brief  Print one byte/character of data, used to support print()
    @param  c  The 8-bit ascii character to write
*/
/**************************************************************************/
void Graphics::write(uint8_t c)
{
 8001a30:	b5b0      	push	{r4, r5, r7, lr}
 8001a32:	b08a      	sub	sp, #40	; 0x28
 8001a34:	af04      	add	r7, sp, #16
 8001a36:	6078      	str	r0, [r7, #4]
 8001a38:	460b      	mov	r3, r1
 8001a3a:	70fb      	strb	r3, [r7, #3]

  if(!m_gfxFontPtr)
 8001a3c:	687b      	ldr	r3, [r7, #4]
 8001a3e:	f503 530e 	add.w	r3, r3, #9088	; 0x2380
 8001a42:	3318      	adds	r3, #24
 8001a44:	681b      	ldr	r3, [r3, #0]
 8001a46:	2b00      	cmp	r3, #0
 8001a48:	f000 80f8 	beq.w	8001c3c <_ZN8Graphics5writeEh+0x20c>
  }
  else
  {
    // Custom font

    if(c == '\n')
 8001a4c:	78fb      	ldrb	r3, [r7, #3]
 8001a4e:	2b0a      	cmp	r3, #10
 8001a50:	d126      	bne.n	8001aa0 <_ZN8Graphics5writeEh+0x70>
    {
      m_cursorX  = 0;
 8001a52:	687b      	ldr	r3, [r7, #4]
 8001a54:	f503 530e 	add.w	r3, r3, #9088	; 0x2380
 8001a58:	3306      	adds	r3, #6
 8001a5a:	2200      	movs	r2, #0
 8001a5c:	801a      	strh	r2, [r3, #0]
      m_cursorY += (int16_t)m_textSize *(uint8_t)pgm_read_byte(&m_gfxFontPtr->yAdvance);
 8001a5e:	687b      	ldr	r3, [r7, #4]
 8001a60:	f503 530e 	add.w	r3, r3, #9088	; 0x2380
 8001a64:	3308      	adds	r3, #8
 8001a66:	f9b3 3000 	ldrsh.w	r3, [r3]
 8001a6a:	b29a      	uxth	r2, r3
 8001a6c:	687b      	ldr	r3, [r7, #4]
 8001a6e:	f503 530e 	add.w	r3, r3, #9088	; 0x2380
 8001a72:	330e      	adds	r3, #14
 8001a74:	781b      	ldrb	r3, [r3, #0]
 8001a76:	b299      	uxth	r1, r3
 8001a78:	687b      	ldr	r3, [r7, #4]
 8001a7a:	f503 530e 	add.w	r3, r3, #9088	; 0x2380
 8001a7e:	3318      	adds	r3, #24
 8001a80:	681b      	ldr	r3, [r3, #0]
 8001a82:	330a      	adds	r3, #10
 8001a84:	781b      	ldrb	r3, [r3, #0]
 8001a86:	b29b      	uxth	r3, r3
 8001a88:	fb11 f303 	smulbb	r3, r1, r3
 8001a8c:	b29b      	uxth	r3, r3
 8001a8e:	4413      	add	r3, r2
 8001a90:	b29b      	uxth	r3, r3
 8001a92:	b21a      	sxth	r2, r3
 8001a94:	687b      	ldr	r3, [r7, #4]
 8001a96:	f503 530e 	add.w	r3, r3, #9088	; 0x2380
 8001a9a:	3308      	adds	r3, #8
 8001a9c:	801a      	strh	r2, [r3, #0]
        }
        m_cursorX += pgm_read_byte(&glyph->xAdvance) * (int16_t)m_textSize;
      }
    }
  }
}
 8001a9e:	e0cd      	b.n	8001c3c <_ZN8Graphics5writeEh+0x20c>
    else if(c != '\r')
 8001aa0:	78fb      	ldrb	r3, [r7, #3]
 8001aa2:	2b0d      	cmp	r3, #13
 8001aa4:	f000 80ca 	beq.w	8001c3c <_ZN8Graphics5writeEh+0x20c>
      uint8_t first = pgm_read_byte(&m_gfxFontPtr->first);
 8001aa8:	687b      	ldr	r3, [r7, #4]
 8001aaa:	f503 530e 	add.w	r3, r3, #9088	; 0x2380
 8001aae:	3318      	adds	r3, #24
 8001ab0:	681b      	ldr	r3, [r3, #0]
 8001ab2:	3308      	adds	r3, #8
 8001ab4:	781b      	ldrb	r3, [r3, #0]
 8001ab6:	75fb      	strb	r3, [r7, #23]
      if((c >= first) && (c <= (uint8_t)pgm_read_byte(&m_gfxFontPtr->last)))
 8001ab8:	78fa      	ldrb	r2, [r7, #3]
 8001aba:	7dfb      	ldrb	r3, [r7, #23]
 8001abc:	429a      	cmp	r2, r3
 8001abe:	f0c0 80bd 	bcc.w	8001c3c <_ZN8Graphics5writeEh+0x20c>
 8001ac2:	687b      	ldr	r3, [r7, #4]
 8001ac4:	f503 530e 	add.w	r3, r3, #9088	; 0x2380
 8001ac8:	3318      	adds	r3, #24
 8001aca:	681b      	ldr	r3, [r3, #0]
 8001acc:	3309      	adds	r3, #9
 8001ace:	781b      	ldrb	r3, [r3, #0]
 8001ad0:	78fa      	ldrb	r2, [r7, #3]
 8001ad2:	429a      	cmp	r2, r3
 8001ad4:	f200 80b2 	bhi.w	8001c3c <_ZN8Graphics5writeEh+0x20c>
        uint8_t   c2    = c - pgm_read_byte(&m_gfxFontPtr->first);
 8001ad8:	687b      	ldr	r3, [r7, #4]
 8001ada:	f503 530e 	add.w	r3, r3, #9088	; 0x2380
 8001ade:	3318      	adds	r3, #24
 8001ae0:	681b      	ldr	r3, [r3, #0]
 8001ae2:	3308      	adds	r3, #8
 8001ae4:	781b      	ldrb	r3, [r3, #0]
 8001ae6:	78fa      	ldrb	r2, [r7, #3]
 8001ae8:	1ad3      	subs	r3, r2, r3
 8001aea:	75bb      	strb	r3, [r7, #22]
        GFX_GLYPH *glyph = &(((GFX_GLYPH *)pgm_read_pointer(&m_gfxFontPtr->glyph))[c2]);
 8001aec:	7dbb      	ldrb	r3, [r7, #22]
 8001aee:	00da      	lsls	r2, r3, #3
 8001af0:	687b      	ldr	r3, [r7, #4]
 8001af2:	f503 530e 	add.w	r3, r3, #9088	; 0x2380
 8001af6:	3318      	adds	r3, #24
 8001af8:	681b      	ldr	r3, [r3, #0]
 8001afa:	3304      	adds	r3, #4
 8001afc:	681b      	ldr	r3, [r3, #0]
 8001afe:	4413      	add	r3, r2
 8001b00:	613b      	str	r3, [r7, #16]
        uint8_t   w     = pgm_read_byte(&glyph->width),
 8001b02:	693b      	ldr	r3, [r7, #16]
 8001b04:	3302      	adds	r3, #2
 8001b06:	781b      	ldrb	r3, [r3, #0]
 8001b08:	73fb      	strb	r3, [r7, #15]
                  h     = pgm_read_byte(&glyph->height);
 8001b0a:	693b      	ldr	r3, [r7, #16]
 8001b0c:	3303      	adds	r3, #3
 8001b0e:	781b      	ldrb	r3, [r3, #0]
 8001b10:	73bb      	strb	r3, [r7, #14]
        if((w > 0) && (h > 0))
 8001b12:	7bfb      	ldrb	r3, [r7, #15]
 8001b14:	2b00      	cmp	r3, #0
 8001b16:	d075      	beq.n	8001c04 <_ZN8Graphics5writeEh+0x1d4>
 8001b18:	7bbb      	ldrb	r3, [r7, #14]
 8001b1a:	2b00      	cmp	r3, #0
 8001b1c:	d072      	beq.n	8001c04 <_ZN8Graphics5writeEh+0x1d4>
          int16_t xo = (int8_t)pgm_read_byte(&glyph->xOffset); // sic
 8001b1e:	693b      	ldr	r3, [r7, #16]
 8001b20:	3305      	adds	r3, #5
 8001b22:	781b      	ldrb	r3, [r3, #0]
 8001b24:	b25b      	sxtb	r3, r3
 8001b26:	81bb      	strh	r3, [r7, #12]
          if(m_wrap && ((m_cursorX + m_textSize * (xo + w)) >= m_widthSize))
 8001b28:	687b      	ldr	r3, [r7, #4]
 8001b2a:	f503 530e 	add.w	r3, r3, #9088	; 0x2380
 8001b2e:	3310      	adds	r3, #16
 8001b30:	681b      	ldr	r3, [r3, #0]
 8001b32:	2b00      	cmp	r3, #0
 8001b34:	d041      	beq.n	8001bba <_ZN8Graphics5writeEh+0x18a>
 8001b36:	687b      	ldr	r3, [r7, #4]
 8001b38:	f503 530e 	add.w	r3, r3, #9088	; 0x2380
 8001b3c:	3306      	adds	r3, #6
 8001b3e:	f9b3 3000 	ldrsh.w	r3, [r3]
 8001b42:	4619      	mov	r1, r3
 8001b44:	687b      	ldr	r3, [r7, #4]
 8001b46:	f503 530e 	add.w	r3, r3, #9088	; 0x2380
 8001b4a:	330e      	adds	r3, #14
 8001b4c:	781b      	ldrb	r3, [r3, #0]
 8001b4e:	4618      	mov	r0, r3
 8001b50:	f9b7 200c 	ldrsh.w	r2, [r7, #12]
 8001b54:	7bfb      	ldrb	r3, [r7, #15]
 8001b56:	4413      	add	r3, r2
 8001b58:	fb03 f300 	mul.w	r3, r3, r0
 8001b5c:	18ca      	adds	r2, r1, r3
 8001b5e:	687b      	ldr	r3, [r7, #4]
 8001b60:	f503 530e 	add.w	r3, r3, #9088	; 0x2380
 8001b64:	3302      	adds	r3, #2
 8001b66:	f9b3 3000 	ldrsh.w	r3, [r3]
 8001b6a:	429a      	cmp	r2, r3
 8001b6c:	db25      	blt.n	8001bba <_ZN8Graphics5writeEh+0x18a>
            m_cursorX  = 0;
 8001b6e:	687b      	ldr	r3, [r7, #4]
 8001b70:	f503 530e 	add.w	r3, r3, #9088	; 0x2380
 8001b74:	3306      	adds	r3, #6
 8001b76:	2200      	movs	r2, #0
 8001b78:	801a      	strh	r2, [r3, #0]
            m_cursorY += (int16_t)m_textSize * (uint8_t)pgm_read_byte(&m_gfxFontPtr->yAdvance);
 8001b7a:	687b      	ldr	r3, [r7, #4]
 8001b7c:	f503 530e 	add.w	r3, r3, #9088	; 0x2380
 8001b80:	3308      	adds	r3, #8
 8001b82:	f9b3 3000 	ldrsh.w	r3, [r3]
 8001b86:	b29a      	uxth	r2, r3
 8001b88:	687b      	ldr	r3, [r7, #4]
 8001b8a:	f503 530e 	add.w	r3, r3, #9088	; 0x2380
 8001b8e:	330e      	adds	r3, #14
 8001b90:	781b      	ldrb	r3, [r3, #0]
 8001b92:	b299      	uxth	r1, r3
 8001b94:	687b      	ldr	r3, [r7, #4]
 8001b96:	f503 530e 	add.w	r3, r3, #9088	; 0x2380
 8001b9a:	3318      	adds	r3, #24
 8001b9c:	681b      	ldr	r3, [r3, #0]
 8001b9e:	330a      	adds	r3, #10
 8001ba0:	781b      	ldrb	r3, [r3, #0]
 8001ba2:	b29b      	uxth	r3, r3
 8001ba4:	fb11 f303 	smulbb	r3, r1, r3
 8001ba8:	b29b      	uxth	r3, r3
 8001baa:	4413      	add	r3, r2
 8001bac:	b29b      	uxth	r3, r3
 8001bae:	b21a      	sxth	r2, r3
 8001bb0:	687b      	ldr	r3, [r7, #4]
 8001bb2:	f503 530e 	add.w	r3, r3, #9088	; 0x2380
 8001bb6:	3308      	adds	r3, #8
 8001bb8:	801a      	strh	r2, [r3, #0]
          drawChar(m_cursorX, m_cursorY, c, m_textColor, m_textBgColor, m_textSize);
 8001bba:	687b      	ldr	r3, [r7, #4]
 8001bbc:	f503 530e 	add.w	r3, r3, #9088	; 0x2380
 8001bc0:	3306      	adds	r3, #6
 8001bc2:	f9b3 0000 	ldrsh.w	r0, [r3]
 8001bc6:	687b      	ldr	r3, [r7, #4]
 8001bc8:	f503 530e 	add.w	r3, r3, #9088	; 0x2380
 8001bcc:	3308      	adds	r3, #8
 8001bce:	f9b3 4000 	ldrsh.w	r4, [r3]
 8001bd2:	687b      	ldr	r3, [r7, #4]
 8001bd4:	f503 530e 	add.w	r3, r3, #9088	; 0x2380
 8001bd8:	330a      	adds	r3, #10
 8001bda:	881a      	ldrh	r2, [r3, #0]
 8001bdc:	687b      	ldr	r3, [r7, #4]
 8001bde:	f503 530e 	add.w	r3, r3, #9088	; 0x2380
 8001be2:	330c      	adds	r3, #12
 8001be4:	8819      	ldrh	r1, [r3, #0]
 8001be6:	687b      	ldr	r3, [r7, #4]
 8001be8:	f503 530e 	add.w	r3, r3, #9088	; 0x2380
 8001bec:	330e      	adds	r3, #14
 8001bee:	781b      	ldrb	r3, [r3, #0]
 8001bf0:	78fd      	ldrb	r5, [r7, #3]
 8001bf2:	9302      	str	r3, [sp, #8]
 8001bf4:	9101      	str	r1, [sp, #4]
 8001bf6:	9200      	str	r2, [sp, #0]
 8001bf8:	462b      	mov	r3, r5
 8001bfa:	4622      	mov	r2, r4
 8001bfc:	4601      	mov	r1, r0
 8001bfe:	6878      	ldr	r0, [r7, #4]
 8001c00:	f000 f820 	bl	8001c44 <_ZN8Graphics8drawCharEsshtth>
        m_cursorX += pgm_read_byte(&glyph->xAdvance) * (int16_t)m_textSize;
 8001c04:	687b      	ldr	r3, [r7, #4]
 8001c06:	f503 530e 	add.w	r3, r3, #9088	; 0x2380
 8001c0a:	3306      	adds	r3, #6
 8001c0c:	f9b3 3000 	ldrsh.w	r3, [r3]
 8001c10:	b29a      	uxth	r2, r3
 8001c12:	693b      	ldr	r3, [r7, #16]
 8001c14:	3304      	adds	r3, #4
 8001c16:	781b      	ldrb	r3, [r3, #0]
 8001c18:	b299      	uxth	r1, r3
 8001c1a:	687b      	ldr	r3, [r7, #4]
 8001c1c:	f503 530e 	add.w	r3, r3, #9088	; 0x2380
 8001c20:	330e      	adds	r3, #14
 8001c22:	781b      	ldrb	r3, [r3, #0]
 8001c24:	b29b      	uxth	r3, r3
 8001c26:	fb11 f303 	smulbb	r3, r1, r3
 8001c2a:	b29b      	uxth	r3, r3
 8001c2c:	4413      	add	r3, r2
 8001c2e:	b29b      	uxth	r3, r3
 8001c30:	b21a      	sxth	r2, r3
 8001c32:	687b      	ldr	r3, [r7, #4]
 8001c34:	f503 530e 	add.w	r3, r3, #9088	; 0x2380
 8001c38:	3306      	adds	r3, #6
 8001c3a:	801a      	strh	r2, [r3, #0]
}
 8001c3c:	bf00      	nop
 8001c3e:	3718      	adds	r7, #24
 8001c40:	46bd      	mov	sp, r7
 8001c42:	bdb0      	pop	{r4, r5, r7, pc}

08001c44 <_ZN8Graphics8drawCharEsshtth>:
    @param    bg 16-bit 5-6-5 Color to fill background with (if same as color, no background)
    @param    size  Font magnification level, 1 is 'original' size
*/
/**************************************************************************/
void Graphics::drawChar(int16_t x, int16_t y, unsigned char c, uint16_t color, uint16_t bg, uint8_t size)
{
 8001c44:	b590      	push	{r4, r7, lr}
 8001c46:	b08d      	sub	sp, #52	; 0x34
 8001c48:	af02      	add	r7, sp, #8
 8001c4a:	60f8      	str	r0, [r7, #12]
 8001c4c:	4608      	mov	r0, r1
 8001c4e:	4611      	mov	r1, r2
 8001c50:	461a      	mov	r2, r3
 8001c52:	4603      	mov	r3, r0
 8001c54:	817b      	strh	r3, [r7, #10]
 8001c56:	460b      	mov	r3, r1
 8001c58:	813b      	strh	r3, [r7, #8]
 8001c5a:	4613      	mov	r3, r2
 8001c5c:	71fb      	strb	r3, [r7, #7]
  if(!m_gfxFontPtr)
 8001c5e:	68fb      	ldr	r3, [r7, #12]
 8001c60:	f503 530e 	add.w	r3, r3, #9088	; 0x2380
 8001c64:	3318      	adds	r3, #24
 8001c66:	681b      	ldr	r3, [r3, #0]
 8001c68:	2b00      	cmp	r3, #0
 8001c6a:	f000 80cf 	beq.w	8001e0c <_ZN8Graphics8drawCharEsshtth+0x1c8>

	// Character is assumed previously filtered by write() to eliminate
	// newlines, returns, non-printable characters, etc.  Calling
	// drawChar() directly with 'bad' characters of font may cause mayhem!

    c -= pgm_read_byte(&m_gfxFontPtr->first);
 8001c6e:	68fb      	ldr	r3, [r7, #12]
 8001c70:	f503 530e 	add.w	r3, r3, #9088	; 0x2380
 8001c74:	3318      	adds	r3, #24
 8001c76:	681b      	ldr	r3, [r3, #0]
 8001c78:	3308      	adds	r3, #8
 8001c7a:	781b      	ldrb	r3, [r3, #0]
 8001c7c:	79fa      	ldrb	r2, [r7, #7]
 8001c7e:	1ad3      	subs	r3, r2, r3
 8001c80:	71fb      	strb	r3, [r7, #7]
    GFX_GLYPH *glyph  = &(((GFX_GLYPH *)pgm_read_pointer(&m_gfxFontPtr->glyph))[c]);
 8001c82:	79fb      	ldrb	r3, [r7, #7]
 8001c84:	00da      	lsls	r2, r3, #3
 8001c86:	68fb      	ldr	r3, [r7, #12]
 8001c88:	f503 530e 	add.w	r3, r3, #9088	; 0x2380
 8001c8c:	3318      	adds	r3, #24
 8001c8e:	681b      	ldr	r3, [r3, #0]
 8001c90:	3304      	adds	r3, #4
 8001c92:	681b      	ldr	r3, [r3, #0]
 8001c94:	4413      	add	r3, r2
 8001c96:	61bb      	str	r3, [r7, #24]
    uint8_t  *bitmap = (uint8_t *)pgm_read_pointer(&m_gfxFontPtr->bitmap);
 8001c98:	68fb      	ldr	r3, [r7, #12]
 8001c9a:	f503 530e 	add.w	r3, r3, #9088	; 0x2380
 8001c9e:	3318      	adds	r3, #24
 8001ca0:	681b      	ldr	r3, [r3, #0]
 8001ca2:	681b      	ldr	r3, [r3, #0]
 8001ca4:	617b      	str	r3, [r7, #20]

    uint16_t bo = pgm_read_word(&glyph->bitmapOffset);
 8001ca6:	69bb      	ldr	r3, [r7, #24]
 8001ca8:	881b      	ldrh	r3, [r3, #0]
 8001caa:	84fb      	strh	r3, [r7, #38]	; 0x26
    uint8_t  w  = pgm_read_byte(&glyph->width),
 8001cac:	69bb      	ldr	r3, [r7, #24]
 8001cae:	3302      	adds	r3, #2
 8001cb0:	781b      	ldrb	r3, [r3, #0]
 8001cb2:	74fb      	strb	r3, [r7, #19]
             h  = pgm_read_byte(&glyph->height);
 8001cb4:	69bb      	ldr	r3, [r7, #24]
 8001cb6:	3303      	adds	r3, #3
 8001cb8:	781b      	ldrb	r3, [r3, #0]
 8001cba:	74bb      	strb	r3, [r7, #18]
    int8_t   xo = pgm_read_byte(&glyph->xOffset),
 8001cbc:	69bb      	ldr	r3, [r7, #24]
 8001cbe:	3305      	adds	r3, #5
 8001cc0:	781b      	ldrb	r3, [r3, #0]
 8001cc2:	747b      	strb	r3, [r7, #17]
             yo = pgm_read_byte(&glyph->yOffset);
 8001cc4:	69bb      	ldr	r3, [r7, #24]
 8001cc6:	3306      	adds	r3, #6
 8001cc8:	781b      	ldrb	r3, [r3, #0]
 8001cca:	743b      	strb	r3, [r7, #16]
    uint8_t  xx, yy, bits = 0, bit = 0;
 8001ccc:	2300      	movs	r3, #0
 8001cce:	f887 3023 	strb.w	r3, [r7, #35]	; 0x23
 8001cd2:	2300      	movs	r3, #0
 8001cd4:	f887 3022 	strb.w	r3, [r7, #34]	; 0x22
    int16_t  xo16 = 0, yo16 = 0;
 8001cd8:	2300      	movs	r3, #0
 8001cda:	843b      	strh	r3, [r7, #32]
 8001cdc:	2300      	movs	r3, #0
 8001cde:	83fb      	strh	r3, [r7, #30]

    if(size > 1)
 8001ce0:	f897 3040 	ldrb.w	r3, [r7, #64]	; 0x40
 8001ce4:	2b01      	cmp	r3, #1
 8001ce6:	d905      	bls.n	8001cf4 <_ZN8Graphics8drawCharEsshtth+0xb0>
    {
      xo16 = xo;
 8001ce8:	f997 3011 	ldrsb.w	r3, [r7, #17]
 8001cec:	843b      	strh	r3, [r7, #32]
      yo16 = yo;
 8001cee:	f997 3010 	ldrsb.w	r3, [r7, #16]
 8001cf2:	83fb      	strh	r3, [r7, #30]
    }

    for(yy=0; yy<h; yy++)
 8001cf4:	2300      	movs	r3, #0
 8001cf6:	f887 3024 	strb.w	r3, [r7, #36]	; 0x24
 8001cfa:	f897 2024 	ldrb.w	r2, [r7, #36]	; 0x24
 8001cfe:	7cbb      	ldrb	r3, [r7, #18]
 8001d00:	429a      	cmp	r2, r3
 8001d02:	f080 8083 	bcs.w	8001e0c <_ZN8Graphics8drawCharEsshtth+0x1c8>
    {
      for(xx=0; xx<w; xx++)
 8001d06:	2300      	movs	r3, #0
 8001d08:	f887 3025 	strb.w	r3, [r7, #37]	; 0x25
 8001d0c:	f897 2025 	ldrb.w	r2, [r7, #37]	; 0x25
 8001d10:	7cfb      	ldrb	r3, [r7, #19]
 8001d12:	429a      	cmp	r2, r3
 8001d14:	d274      	bcs.n	8001e00 <_ZN8Graphics8drawCharEsshtth+0x1bc>
      {
        if(!(bit++ & 7))
 8001d16:	f897 3022 	ldrb.w	r3, [r7, #34]	; 0x22
 8001d1a:	1c5a      	adds	r2, r3, #1
 8001d1c:	f887 2022 	strb.w	r2, [r7, #34]	; 0x22
 8001d20:	f003 0307 	and.w	r3, r3, #7
 8001d24:	2b00      	cmp	r3, #0
 8001d26:	bf0c      	ite	eq
 8001d28:	2301      	moveq	r3, #1
 8001d2a:	2300      	movne	r3, #0
 8001d2c:	b2db      	uxtb	r3, r3
 8001d2e:	2b00      	cmp	r3, #0
 8001d30:	d008      	beq.n	8001d44 <_ZN8Graphics8drawCharEsshtth+0x100>
        {
          bits = pgm_read_byte(&bitmap[bo++]);
 8001d32:	8cfb      	ldrh	r3, [r7, #38]	; 0x26
 8001d34:	1c5a      	adds	r2, r3, #1
 8001d36:	84fa      	strh	r2, [r7, #38]	; 0x26
 8001d38:	461a      	mov	r2, r3
 8001d3a:	697b      	ldr	r3, [r7, #20]
 8001d3c:	4413      	add	r3, r2
 8001d3e:	781b      	ldrb	r3, [r3, #0]
 8001d40:	f887 3023 	strb.w	r3, [r7, #35]	; 0x23
        }
        if(bits & 0x80)
 8001d44:	f997 3023 	ldrsb.w	r3, [r7, #35]	; 0x23
 8001d48:	2b00      	cmp	r3, #0
 8001d4a:	da4e      	bge.n	8001dea <_ZN8Graphics8drawCharEsshtth+0x1a6>
        {
          if(size == 1)
 8001d4c:	f897 3040 	ldrb.w	r3, [r7, #64]	; 0x40
 8001d50:	2b01      	cmp	r3, #1
 8001d52:	d11c      	bne.n	8001d8e <_ZN8Graphics8drawCharEsshtth+0x14a>
          {
            drawPixel(x+xo+xx, y+yo+yy, color);
 8001d54:	f997 3011 	ldrsb.w	r3, [r7, #17]
 8001d58:	b29a      	uxth	r2, r3
 8001d5a:	897b      	ldrh	r3, [r7, #10]
 8001d5c:	4413      	add	r3, r2
 8001d5e:	b29a      	uxth	r2, r3
 8001d60:	f897 3025 	ldrb.w	r3, [r7, #37]	; 0x25
 8001d64:	b29b      	uxth	r3, r3
 8001d66:	4413      	add	r3, r2
 8001d68:	b29b      	uxth	r3, r3
 8001d6a:	b219      	sxth	r1, r3
 8001d6c:	f997 3010 	ldrsb.w	r3, [r7, #16]
 8001d70:	b29a      	uxth	r2, r3
 8001d72:	893b      	ldrh	r3, [r7, #8]
 8001d74:	4413      	add	r3, r2
 8001d76:	b29a      	uxth	r2, r3
 8001d78:	f897 3024 	ldrb.w	r3, [r7, #36]	; 0x24
 8001d7c:	b29b      	uxth	r3, r3
 8001d7e:	4413      	add	r3, r2
 8001d80:	b29b      	uxth	r3, r3
 8001d82:	b21a      	sxth	r2, r3
 8001d84:	8f3b      	ldrh	r3, [r7, #56]	; 0x38
 8001d86:	68f8      	ldr	r0, [r7, #12]
 8001d88:	f7ff fdea 	bl	8001960 <_ZN8Graphics9drawPixelEsst>
 8001d8c:	e02d      	b.n	8001dea <_ZN8Graphics8drawCharEsshtth+0x1a6>
          }
          else
          {
            fillRect(x+(xo16+xx)*size, y+(yo16+yy)*size, size, size, color);
 8001d8e:	f9b7 2020 	ldrsh.w	r2, [r7, #32]
 8001d92:	f897 3025 	ldrb.w	r3, [r7, #37]	; 0x25
 8001d96:	4413      	add	r3, r2
 8001d98:	b29a      	uxth	r2, r3
 8001d9a:	f897 3040 	ldrb.w	r3, [r7, #64]	; 0x40
 8001d9e:	b29b      	uxth	r3, r3
 8001da0:	fb12 f303 	smulbb	r3, r2, r3
 8001da4:	b29a      	uxth	r2, r3
 8001da6:	897b      	ldrh	r3, [r7, #10]
 8001da8:	4413      	add	r3, r2
 8001daa:	b29b      	uxth	r3, r3
 8001dac:	b219      	sxth	r1, r3
 8001dae:	f9b7 201e 	ldrsh.w	r2, [r7, #30]
 8001db2:	f897 3024 	ldrb.w	r3, [r7, #36]	; 0x24
 8001db6:	4413      	add	r3, r2
 8001db8:	b29a      	uxth	r2, r3
 8001dba:	f897 3040 	ldrb.w	r3, [r7, #64]	; 0x40
 8001dbe:	b29b      	uxth	r3, r3
 8001dc0:	fb12 f303 	smulbb	r3, r2, r3
 8001dc4:	b29a      	uxth	r2, r3
 8001dc6:	893b      	ldrh	r3, [r7, #8]
 8001dc8:	4413      	add	r3, r2
 8001dca:	b29b      	uxth	r3, r3
 8001dcc:	b218      	sxth	r0, r3
 8001dce:	f897 3040 	ldrb.w	r3, [r7, #64]	; 0x40
 8001dd2:	b21c      	sxth	r4, r3
 8001dd4:	f897 3040 	ldrb.w	r3, [r7, #64]	; 0x40
 8001dd8:	b21b      	sxth	r3, r3
 8001dda:	8f3a      	ldrh	r2, [r7, #56]	; 0x38
 8001ddc:	9201      	str	r2, [sp, #4]
 8001dde:	9300      	str	r3, [sp, #0]
 8001de0:	4623      	mov	r3, r4
 8001de2:	4602      	mov	r2, r0
 8001de4:	68f8      	ldr	r0, [r7, #12]
 8001de6:	f000 fb6e 	bl	80024c6 <_ZN8Graphics8fillRectEsssst>
          }
        }
        bits <<= 1;
 8001dea:	f897 3023 	ldrb.w	r3, [r7, #35]	; 0x23
 8001dee:	005b      	lsls	r3, r3, #1
 8001df0:	f887 3023 	strb.w	r3, [r7, #35]	; 0x23
      for(xx=0; xx<w; xx++)
 8001df4:	f897 3025 	ldrb.w	r3, [r7, #37]	; 0x25
 8001df8:	3301      	adds	r3, #1
 8001dfa:	f887 3025 	strb.w	r3, [r7, #37]	; 0x25
 8001dfe:	e785      	b.n	8001d0c <_ZN8Graphics8drawCharEsshtth+0xc8>
    for(yy=0; yy<h; yy++)
 8001e00:	f897 3024 	ldrb.w	r3, [r7, #36]	; 0x24
 8001e04:	3301      	adds	r3, #1
 8001e06:	f887 3024 	strb.w	r3, [r7, #36]	; 0x24
 8001e0a:	e776      	b.n	8001cfa <_ZN8Graphics8drawCharEsshtth+0xb6>
      }
    }
  }
}
 8001e0c:	bf00      	nop
 8001e0e:	372c      	adds	r7, #44	; 0x2c
 8001e10:	46bd      	mov	sp, r7
 8001e12:	bd90      	pop	{r4, r7, pc}

08001e14 <_ZN8Graphics15getFontXAdvanceEv>:
    @brief Take the widest character attributes
    @param
*/
/**************************************************************************/
uint8_t Graphics::getFontXAdvance()
{
 8001e14:	b480      	push	{r7}
 8001e16:	b085      	sub	sp, #20
 8001e18:	af00      	add	r7, sp, #0
 8001e1a:	6078      	str	r0, [r7, #4]
  uint8_t xa ;
  GFX_GLYPH * glyph;

  if(m_gfxFontPtr)
 8001e1c:	687b      	ldr	r3, [r7, #4]
 8001e1e:	f503 530e 	add.w	r3, r3, #9088	; 0x2380
 8001e22:	3318      	adds	r3, #24
 8001e24:	681b      	ldr	r3, [r3, #0]
 8001e26:	2b00      	cmp	r3, #0
 8001e28:	d00d      	beq.n	8001e46 <_ZN8Graphics15getFontXAdvanceEv+0x32>
  {
    glyph = &(((GFX_GLYPH *)pgm_read_pointer(&m_gfxFontPtr->glyph))[6]);/* Choosing character '%' */
 8001e2a:	687b      	ldr	r3, [r7, #4]
 8001e2c:	f503 530e 	add.w	r3, r3, #9088	; 0x2380
 8001e30:	3318      	adds	r3, #24
 8001e32:	681b      	ldr	r3, [r3, #0]
 8001e34:	3304      	adds	r3, #4
 8001e36:	681b      	ldr	r3, [r3, #0]
 8001e38:	3330      	adds	r3, #48	; 0x30
 8001e3a:	60bb      	str	r3, [r7, #8]
    xa = pgm_read_byte(&glyph->width);
 8001e3c:	68bb      	ldr	r3, [r7, #8]
 8001e3e:	3302      	adds	r3, #2
 8001e40:	781b      	ldrb	r3, [r3, #0]
 8001e42:	73fb      	strb	r3, [r7, #15]
 8001e44:	e001      	b.n	8001e4a <_ZN8Graphics15getFontXAdvanceEv+0x36>
  }
  else
  {
    xa = 6;
 8001e46:	2306      	movs	r3, #6
 8001e48:	73fb      	strb	r3, [r7, #15]
  }
  return xa;
 8001e4a:	7bfb      	ldrb	r3, [r7, #15]
}
 8001e4c:	4618      	mov	r0, r3
 8001e4e:	3714      	adds	r7, #20
 8001e50:	46bd      	mov	sp, r7
 8001e52:	f85d 7b04 	ldr.w	r7, [sp], #4
 8001e56:	4770      	bx	lr

08001e58 <_ZN8Graphics15getFontYAdvanceEv>:
    @brief Take the Tallest character attributes
    @param
*/
/**************************************************************************/
uint8_t Graphics::getFontYAdvance()
{
 8001e58:	b480      	push	{r7}
 8001e5a:	b085      	sub	sp, #20
 8001e5c:	af00      	add	r7, sp, #0
 8001e5e:	6078      	str	r0, [r7, #4]
  uint8_t ya;
  GFX_GLYPH * glyph;

  if(m_gfxFontPtr)
 8001e60:	687b      	ldr	r3, [r7, #4]
 8001e62:	f503 530e 	add.w	r3, r3, #9088	; 0x2380
 8001e66:	3318      	adds	r3, #24
 8001e68:	681b      	ldr	r3, [r3, #0]
 8001e6a:	2b00      	cmp	r3, #0
 8001e6c:	d00f      	beq.n	8001e8e <_ZN8Graphics15getFontYAdvanceEv+0x36>
  {
    glyph = &(((GFX_GLYPH *)pgm_read_pointer(&m_gfxFontPtr->glyph))[45]);/* Choosing character 'L' */
 8001e6e:	687b      	ldr	r3, [r7, #4]
 8001e70:	f503 530e 	add.w	r3, r3, #9088	; 0x2380
 8001e74:	3318      	adds	r3, #24
 8001e76:	681b      	ldr	r3, [r3, #0]
 8001e78:	3304      	adds	r3, #4
 8001e7a:	681b      	ldr	r3, [r3, #0]
 8001e7c:	f503 73b4 	add.w	r3, r3, #360	; 0x168
 8001e80:	60bb      	str	r3, [r7, #8]
    ya = 2 + pgm_read_byte(&glyph->height);
 8001e82:	68bb      	ldr	r3, [r7, #8]
 8001e84:	3303      	adds	r3, #3
 8001e86:	781b      	ldrb	r3, [r3, #0]
 8001e88:	3302      	adds	r3, #2
 8001e8a:	73fb      	strb	r3, [r7, #15]
 8001e8c:	e001      	b.n	8001e92 <_ZN8Graphics15getFontYAdvanceEv+0x3a>
  }
  else
  {
    ya = 8;
 8001e8e:	2308      	movs	r3, #8
 8001e90:	73fb      	strb	r3, [r7, #15]
  }
  return ya;
 8001e92:	7bfb      	ldrb	r3, [r7, #15]
}
 8001e94:	4618      	mov	r0, r3
 8001e96:	3714      	adds	r7, #20
 8001e98:	46bd      	mov	sp, r7
 8001e9a:	f85d 7b04 	ldr.w	r7, [sp], #4
 8001e9e:	4770      	bx	lr

08001ea0 <_ZN8Graphics10drawCircleEssst>:
    @param    r   Radius of circle
    @param    color 0 - white 1 - black
*/
/**************************************************************************/
void Graphics::drawCircle(int16_t x0, int16_t y0, int16_t r, uint16_t color)
{
 8001ea0:	b580      	push	{r7, lr}
 8001ea2:	b088      	sub	sp, #32
 8001ea4:	af00      	add	r7, sp, #0
 8001ea6:	60f8      	str	r0, [r7, #12]
 8001ea8:	4608      	mov	r0, r1
 8001eaa:	4611      	mov	r1, r2
 8001eac:	461a      	mov	r2, r3
 8001eae:	4603      	mov	r3, r0
 8001eb0:	817b      	strh	r3, [r7, #10]
 8001eb2:	460b      	mov	r3, r1
 8001eb4:	813b      	strh	r3, [r7, #8]
 8001eb6:	4613      	mov	r3, r2
 8001eb8:	80fb      	strh	r3, [r7, #6]
  int16_t f = 1 - r;
 8001eba:	88fb      	ldrh	r3, [r7, #6]
 8001ebc:	f1c3 0301 	rsb	r3, r3, #1
 8001ec0:	b29b      	uxth	r3, r3
 8001ec2:	83fb      	strh	r3, [r7, #30]
  int16_t ddF_x = 1;
 8001ec4:	2301      	movs	r3, #1
 8001ec6:	83bb      	strh	r3, [r7, #28]
  int16_t ddF_y = -2 * r;
 8001ec8:	88fb      	ldrh	r3, [r7, #6]
 8001eca:	461a      	mov	r2, r3
 8001ecc:	03d2      	lsls	r2, r2, #15
 8001ece:	1ad3      	subs	r3, r2, r3
 8001ed0:	005b      	lsls	r3, r3, #1
 8001ed2:	b29b      	uxth	r3, r3
 8001ed4:	837b      	strh	r3, [r7, #26]
  int16_t x = 0;
 8001ed6:	2300      	movs	r3, #0
 8001ed8:	833b      	strh	r3, [r7, #24]
  int16_t y = r;
 8001eda:	88fb      	ldrh	r3, [r7, #6]
 8001edc:	82fb      	strh	r3, [r7, #22]

  drawPixel(x0, y0+r, color);
 8001ede:	893a      	ldrh	r2, [r7, #8]
 8001ee0:	88fb      	ldrh	r3, [r7, #6]
 8001ee2:	4413      	add	r3, r2
 8001ee4:	b29b      	uxth	r3, r3
 8001ee6:	b21a      	sxth	r2, r3
 8001ee8:	8d3b      	ldrh	r3, [r7, #40]	; 0x28
 8001eea:	f9b7 100a 	ldrsh.w	r1, [r7, #10]
 8001eee:	68f8      	ldr	r0, [r7, #12]
 8001ef0:	f7ff fd36 	bl	8001960 <_ZN8Graphics9drawPixelEsst>
  drawPixel(x0, y0-r, color);
 8001ef4:	893a      	ldrh	r2, [r7, #8]
 8001ef6:	88fb      	ldrh	r3, [r7, #6]
 8001ef8:	1ad3      	subs	r3, r2, r3
 8001efa:	b29b      	uxth	r3, r3
 8001efc:	b21a      	sxth	r2, r3
 8001efe:	8d3b      	ldrh	r3, [r7, #40]	; 0x28
 8001f00:	f9b7 100a 	ldrsh.w	r1, [r7, #10]
 8001f04:	68f8      	ldr	r0, [r7, #12]
 8001f06:	f7ff fd2b 	bl	8001960 <_ZN8Graphics9drawPixelEsst>
  drawPixel(x0+r, y0, color);
 8001f0a:	897a      	ldrh	r2, [r7, #10]
 8001f0c:	88fb      	ldrh	r3, [r7, #6]
 8001f0e:	4413      	add	r3, r2
 8001f10:	b29b      	uxth	r3, r3
 8001f12:	b219      	sxth	r1, r3
 8001f14:	8d3b      	ldrh	r3, [r7, #40]	; 0x28
 8001f16:	f9b7 2008 	ldrsh.w	r2, [r7, #8]
 8001f1a:	68f8      	ldr	r0, [r7, #12]
 8001f1c:	f7ff fd20 	bl	8001960 <_ZN8Graphics9drawPixelEsst>
  drawPixel(x0-r, y0, color);
 8001f20:	897a      	ldrh	r2, [r7, #10]
 8001f22:	88fb      	ldrh	r3, [r7, #6]
 8001f24:	1ad3      	subs	r3, r2, r3
 8001f26:	b29b      	uxth	r3, r3
 8001f28:	b219      	sxth	r1, r3
 8001f2a:	8d3b      	ldrh	r3, [r7, #40]	; 0x28
 8001f2c:	f9b7 2008 	ldrsh.w	r2, [r7, #8]
 8001f30:	68f8      	ldr	r0, [r7, #12]
 8001f32:	f7ff fd15 	bl	8001960 <_ZN8Graphics9drawPixelEsst>

  while (x<y)
 8001f36:	f9b7 2018 	ldrsh.w	r2, [r7, #24]
 8001f3a:	f9b7 3016 	ldrsh.w	r3, [r7, #22]
 8001f3e:	429a      	cmp	r2, r3
 8001f40:	f280 8093 	bge.w	800206a <_ZN8Graphics10drawCircleEssst+0x1ca>
  {
    if (f >= 0)
 8001f44:	f9b7 301e 	ldrsh.w	r3, [r7, #30]
 8001f48:	2b00      	cmp	r3, #0
 8001f4a:	db0e      	blt.n	8001f6a <_ZN8Graphics10drawCircleEssst+0xca>
    {
      y--;
 8001f4c:	f9b7 3016 	ldrsh.w	r3, [r7, #22]
 8001f50:	b29b      	uxth	r3, r3
 8001f52:	3b01      	subs	r3, #1
 8001f54:	b29b      	uxth	r3, r3
 8001f56:	82fb      	strh	r3, [r7, #22]
      ddF_y += 2;
 8001f58:	8b7b      	ldrh	r3, [r7, #26]
 8001f5a:	3302      	adds	r3, #2
 8001f5c:	b29b      	uxth	r3, r3
 8001f5e:	837b      	strh	r3, [r7, #26]
      f += ddF_y;
 8001f60:	8bfa      	ldrh	r2, [r7, #30]
 8001f62:	8b7b      	ldrh	r3, [r7, #26]
 8001f64:	4413      	add	r3, r2
 8001f66:	b29b      	uxth	r3, r3
 8001f68:	83fb      	strh	r3, [r7, #30]
    }
    x++;
 8001f6a:	f9b7 3018 	ldrsh.w	r3, [r7, #24]
 8001f6e:	b29b      	uxth	r3, r3
 8001f70:	3301      	adds	r3, #1
 8001f72:	b29b      	uxth	r3, r3
 8001f74:	833b      	strh	r3, [r7, #24]
    ddF_x += 2;
 8001f76:	8bbb      	ldrh	r3, [r7, #28]
 8001f78:	3302      	adds	r3, #2
 8001f7a:	b29b      	uxth	r3, r3
 8001f7c:	83bb      	strh	r3, [r7, #28]
    f += ddF_x;
 8001f7e:	8bfa      	ldrh	r2, [r7, #30]
 8001f80:	8bbb      	ldrh	r3, [r7, #28]
 8001f82:	4413      	add	r3, r2
 8001f84:	b29b      	uxth	r3, r3
 8001f86:	83fb      	strh	r3, [r7, #30]

    drawPixel(x0 + x, y0 + y, color);
 8001f88:	897a      	ldrh	r2, [r7, #10]
 8001f8a:	8b3b      	ldrh	r3, [r7, #24]
 8001f8c:	4413      	add	r3, r2
 8001f8e:	b29b      	uxth	r3, r3
 8001f90:	b219      	sxth	r1, r3
 8001f92:	893a      	ldrh	r2, [r7, #8]
 8001f94:	8afb      	ldrh	r3, [r7, #22]
 8001f96:	4413      	add	r3, r2
 8001f98:	b29b      	uxth	r3, r3
 8001f9a:	b21a      	sxth	r2, r3
 8001f9c:	8d3b      	ldrh	r3, [r7, #40]	; 0x28
 8001f9e:	68f8      	ldr	r0, [r7, #12]
 8001fa0:	f7ff fcde 	bl	8001960 <_ZN8Graphics9drawPixelEsst>
    drawPixel(x0 - x, y0 + y, color);
 8001fa4:	897a      	ldrh	r2, [r7, #10]
 8001fa6:	8b3b      	ldrh	r3, [r7, #24]
 8001fa8:	1ad3      	subs	r3, r2, r3
 8001faa:	b29b      	uxth	r3, r3
 8001fac:	b219      	sxth	r1, r3
 8001fae:	893a      	ldrh	r2, [r7, #8]
 8001fb0:	8afb      	ldrh	r3, [r7, #22]
 8001fb2:	4413      	add	r3, r2
 8001fb4:	b29b      	uxth	r3, r3
 8001fb6:	b21a      	sxth	r2, r3
 8001fb8:	8d3b      	ldrh	r3, [r7, #40]	; 0x28
 8001fba:	68f8      	ldr	r0, [r7, #12]
 8001fbc:	f7ff fcd0 	bl	8001960 <_ZN8Graphics9drawPixelEsst>
    drawPixel(x0 + x, y0 - y, color);
 8001fc0:	897a      	ldrh	r2, [r7, #10]
 8001fc2:	8b3b      	ldrh	r3, [r7, #24]
 8001fc4:	4413      	add	r3, r2
 8001fc6:	b29b      	uxth	r3, r3
 8001fc8:	b219      	sxth	r1, r3
 8001fca:	893a      	ldrh	r2, [r7, #8]
 8001fcc:	8afb      	ldrh	r3, [r7, #22]
 8001fce:	1ad3      	subs	r3, r2, r3
 8001fd0:	b29b      	uxth	r3, r3
 8001fd2:	b21a      	sxth	r2, r3
 8001fd4:	8d3b      	ldrh	r3, [r7, #40]	; 0x28
 8001fd6:	68f8      	ldr	r0, [r7, #12]
 8001fd8:	f7ff fcc2 	bl	8001960 <_ZN8Graphics9drawPixelEsst>
    drawPixel(x0 - x, y0 - y, color);
 8001fdc:	897a      	ldrh	r2, [r7, #10]
 8001fde:	8b3b      	ldrh	r3, [r7, #24]
 8001fe0:	1ad3      	subs	r3, r2, r3
 8001fe2:	b29b      	uxth	r3, r3
 8001fe4:	b219      	sxth	r1, r3
 8001fe6:	893a      	ldrh	r2, [r7, #8]
 8001fe8:	8afb      	ldrh	r3, [r7, #22]
 8001fea:	1ad3      	subs	r3, r2, r3
 8001fec:	b29b      	uxth	r3, r3
 8001fee:	b21a      	sxth	r2, r3
 8001ff0:	8d3b      	ldrh	r3, [r7, #40]	; 0x28
 8001ff2:	68f8      	ldr	r0, [r7, #12]
 8001ff4:	f7ff fcb4 	bl	8001960 <_ZN8Graphics9drawPixelEsst>
    drawPixel(x0 + y, y0 + x, color);
 8001ff8:	897a      	ldrh	r2, [r7, #10]
 8001ffa:	8afb      	ldrh	r3, [r7, #22]
 8001ffc:	4413      	add	r3, r2
 8001ffe:	b29b      	uxth	r3, r3
 8002000:	b219      	sxth	r1, r3
 8002002:	893a      	ldrh	r2, [r7, #8]
 8002004:	8b3b      	ldrh	r3, [r7, #24]
 8002006:	4413      	add	r3, r2
 8002008:	b29b      	uxth	r3, r3
 800200a:	b21a      	sxth	r2, r3
 800200c:	8d3b      	ldrh	r3, [r7, #40]	; 0x28
 800200e:	68f8      	ldr	r0, [r7, #12]
 8002010:	f7ff fca6 	bl	8001960 <_ZN8Graphics9drawPixelEsst>
    drawPixel(x0 - y, y0 + x, color);
 8002014:	897a      	ldrh	r2, [r7, #10]
 8002016:	8afb      	ldrh	r3, [r7, #22]
 8002018:	1ad3      	subs	r3, r2, r3
 800201a:	b29b      	uxth	r3, r3
 800201c:	b219      	sxth	r1, r3
 800201e:	893a      	ldrh	r2, [r7, #8]
 8002020:	8b3b      	ldrh	r3, [r7, #24]
 8002022:	4413      	add	r3, r2
 8002024:	b29b      	uxth	r3, r3
 8002026:	b21a      	sxth	r2, r3
 8002028:	8d3b      	ldrh	r3, [r7, #40]	; 0x28
 800202a:	68f8      	ldr	r0, [r7, #12]
 800202c:	f7ff fc98 	bl	8001960 <_ZN8Graphics9drawPixelEsst>
    drawPixel(x0 + y, y0 - x, color);
 8002030:	897a      	ldrh	r2, [r7, #10]
 8002032:	8afb      	ldrh	r3, [r7, #22]
 8002034:	4413      	add	r3, r2
 8002036:	b29b      	uxth	r3, r3
 8002038:	b219      	sxth	r1, r3
 800203a:	893a      	ldrh	r2, [r7, #8]
 800203c:	8b3b      	ldrh	r3, [r7, #24]
 800203e:	1ad3      	subs	r3, r2, r3
 8002040:	b29b      	uxth	r3, r3
 8002042:	b21a      	sxth	r2, r3
 8002044:	8d3b      	ldrh	r3, [r7, #40]	; 0x28
 8002046:	68f8      	ldr	r0, [r7, #12]
 8002048:	f7ff fc8a 	bl	8001960 <_ZN8Graphics9drawPixelEsst>
    drawPixel(x0 - y, y0 - x, color);
 800204c:	897a      	ldrh	r2, [r7, #10]
 800204e:	8afb      	ldrh	r3, [r7, #22]
 8002050:	1ad3      	subs	r3, r2, r3
 8002052:	b29b      	uxth	r3, r3
 8002054:	b219      	sxth	r1, r3
 8002056:	893a      	ldrh	r2, [r7, #8]
 8002058:	8b3b      	ldrh	r3, [r7, #24]
 800205a:	1ad3      	subs	r3, r2, r3
 800205c:	b29b      	uxth	r3, r3
 800205e:	b21a      	sxth	r2, r3
 8002060:	8d3b      	ldrh	r3, [r7, #40]	; 0x28
 8002062:	68f8      	ldr	r0, [r7, #12]
 8002064:	f7ff fc7c 	bl	8001960 <_ZN8Graphics9drawPixelEsst>
  while (x<y)
 8002068:	e765      	b.n	8001f36 <_ZN8Graphics10drawCircleEssst+0x96>
  }
}
 800206a:	bf00      	nop
 800206c:	3720      	adds	r7, #32
 800206e:	46bd      	mov	sp, r7
 8002070:	bd80      	pop	{r7, pc}

08002072 <_ZN8Graphics10fillCircleEssst>:
    @param    r   Radius of circle
    @param    color 0 - white 1 - black
*/
/**************************************************************************/
void Graphics::fillCircle(int16_t x0, int16_t y0, int16_t r, uint16_t color)
{
 8002072:	b580      	push	{r7, lr}
 8002074:	b088      	sub	sp, #32
 8002076:	af04      	add	r7, sp, #16
 8002078:	60f8      	str	r0, [r7, #12]
 800207a:	4608      	mov	r0, r1
 800207c:	4611      	mov	r1, r2
 800207e:	461a      	mov	r2, r3
 8002080:	4603      	mov	r3, r0
 8002082:	817b      	strh	r3, [r7, #10]
 8002084:	460b      	mov	r3, r1
 8002086:	813b      	strh	r3, [r7, #8]
 8002088:	4613      	mov	r3, r2
 800208a:	80fb      	strh	r3, [r7, #6]
  drawFastVLine(x0, y0-r, 2*r+1, color);
 800208c:	893a      	ldrh	r2, [r7, #8]
 800208e:	88fb      	ldrh	r3, [r7, #6]
 8002090:	1ad3      	subs	r3, r2, r3
 8002092:	b29b      	uxth	r3, r3
 8002094:	b21a      	sxth	r2, r3
 8002096:	88fb      	ldrh	r3, [r7, #6]
 8002098:	005b      	lsls	r3, r3, #1
 800209a:	b29b      	uxth	r3, r3
 800209c:	3301      	adds	r3, #1
 800209e:	b29b      	uxth	r3, r3
 80020a0:	b218      	sxth	r0, r3
 80020a2:	f9b7 100a 	ldrsh.w	r1, [r7, #10]
 80020a6:	8b3b      	ldrh	r3, [r7, #24]
 80020a8:	9300      	str	r3, [sp, #0]
 80020aa:	4603      	mov	r3, r0
 80020ac:	68f8      	ldr	r0, [r7, #12]
 80020ae:	f000 f9bf 	bl	8002430 <_ZN8Graphics13drawFastVLineEssst>
  fillCircleHelper(x0, y0, r, 3, 0, color);
 80020b2:	f9b7 0006 	ldrsh.w	r0, [r7, #6]
 80020b6:	f9b7 2008 	ldrsh.w	r2, [r7, #8]
 80020ba:	f9b7 100a 	ldrsh.w	r1, [r7, #10]
 80020be:	8b3b      	ldrh	r3, [r7, #24]
 80020c0:	9302      	str	r3, [sp, #8]
 80020c2:	2300      	movs	r3, #0
 80020c4:	9301      	str	r3, [sp, #4]
 80020c6:	2303      	movs	r3, #3
 80020c8:	9300      	str	r3, [sp, #0]
 80020ca:	4603      	mov	r3, r0
 80020cc:	68f8      	ldr	r0, [r7, #12]
 80020ce:	f000 f804 	bl	80020da <_ZN8Graphics16fillCircleHelperEssshst>
}
 80020d2:	bf00      	nop
 80020d4:	3710      	adds	r7, #16
 80020d6:	46bd      	mov	sp, r7
 80020d8:	bd80      	pop	{r7, pc}

080020da <_ZN8Graphics16fillCircleHelperEssshst>:
    @param    color 0 - white 1 - black
*/
/**************************************************************************/
void Graphics::fillCircleHelper(int16_t x0, int16_t y0, int16_t r,
                                uint8_t cornername, int16_t delta, uint16_t color)
{
 80020da:	b580      	push	{r7, lr}
 80020dc:	b08a      	sub	sp, #40	; 0x28
 80020de:	af02      	add	r7, sp, #8
 80020e0:	60f8      	str	r0, [r7, #12]
 80020e2:	4608      	mov	r0, r1
 80020e4:	4611      	mov	r1, r2
 80020e6:	461a      	mov	r2, r3
 80020e8:	4603      	mov	r3, r0
 80020ea:	817b      	strh	r3, [r7, #10]
 80020ec:	460b      	mov	r3, r1
 80020ee:	813b      	strh	r3, [r7, #8]
 80020f0:	4613      	mov	r3, r2
 80020f2:	80fb      	strh	r3, [r7, #6]

  int16_t f     = 1 - r;
 80020f4:	88fb      	ldrh	r3, [r7, #6]
 80020f6:	f1c3 0301 	rsb	r3, r3, #1
 80020fa:	b29b      	uxth	r3, r3
 80020fc:	83fb      	strh	r3, [r7, #30]
  int16_t ddF_x = 1;
 80020fe:	2301      	movs	r3, #1
 8002100:	83bb      	strh	r3, [r7, #28]
  int16_t ddF_y = -2 * r;
 8002102:	88fb      	ldrh	r3, [r7, #6]
 8002104:	461a      	mov	r2, r3
 8002106:	03d2      	lsls	r2, r2, #15
 8002108:	1ad3      	subs	r3, r2, r3
 800210a:	005b      	lsls	r3, r3, #1
 800210c:	b29b      	uxth	r3, r3
 800210e:	837b      	strh	r3, [r7, #26]
  int16_t x     = 0;
 8002110:	2300      	movs	r3, #0
 8002112:	833b      	strh	r3, [r7, #24]
  int16_t y     = r;
 8002114:	88fb      	ldrh	r3, [r7, #6]
 8002116:	82fb      	strh	r3, [r7, #22]
  while (x<y)
 8002118:	f9b7 2018 	ldrsh.w	r2, [r7, #24]
 800211c:	f9b7 3016 	ldrsh.w	r3, [r7, #22]
 8002120:	429a      	cmp	r2, r3
 8002122:	f280 8097 	bge.w	8002254 <_ZN8Graphics16fillCircleHelperEssshst+0x17a>
  {
    if (f >= 0)
 8002126:	f9b7 301e 	ldrsh.w	r3, [r7, #30]
 800212a:	2b00      	cmp	r3, #0
 800212c:	db0e      	blt.n	800214c <_ZN8Graphics16fillCircleHelperEssshst+0x72>
    {
      y--;
 800212e:	f9b7 3016 	ldrsh.w	r3, [r7, #22]
 8002132:	b29b      	uxth	r3, r3
 8002134:	3b01      	subs	r3, #1
 8002136:	b29b      	uxth	r3, r3
 8002138:	82fb      	strh	r3, [r7, #22]
      ddF_y += 2;
 800213a:	8b7b      	ldrh	r3, [r7, #26]
 800213c:	3302      	adds	r3, #2
 800213e:	b29b      	uxth	r3, r3
 8002140:	837b      	strh	r3, [r7, #26]
      f+= ddF_y;
 8002142:	8bfa      	ldrh	r2, [r7, #30]
 8002144:	8b7b      	ldrh	r3, [r7, #26]
 8002146:	4413      	add	r3, r2
 8002148:	b29b      	uxth	r3, r3
 800214a:	83fb      	strh	r3, [r7, #30]
    }
    x++;
 800214c:	f9b7 3018 	ldrsh.w	r3, [r7, #24]
 8002150:	b29b      	uxth	r3, r3
 8002152:	3301      	adds	r3, #1
 8002154:	b29b      	uxth	r3, r3
 8002156:	833b      	strh	r3, [r7, #24]
    ddF_x += 2;
 8002158:	8bbb      	ldrh	r3, [r7, #28]
 800215a:	3302      	adds	r3, #2
 800215c:	b29b      	uxth	r3, r3
 800215e:	83bb      	strh	r3, [r7, #28]
    f+= ddF_x;
 8002160:	8bfa      	ldrh	r2, [r7, #30]
 8002162:	8bbb      	ldrh	r3, [r7, #28]
 8002164:	4413      	add	r3, r2
 8002166:	b29b      	uxth	r3, r3
 8002168:	83fb      	strh	r3, [r7, #30]

    if (cornername & 0x1)
 800216a:	f897 3028 	ldrb.w	r3, [r7, #40]	; 0x28
 800216e:	f003 0301 	and.w	r3, r3, #1
 8002172:	2b00      	cmp	r3, #0
 8002174:	d033      	beq.n	80021de <_ZN8Graphics16fillCircleHelperEssshst+0x104>
    {
      drawFastVLine(x0+x, y0-y, 2*y+1+delta, color);
 8002176:	897a      	ldrh	r2, [r7, #10]
 8002178:	8b3b      	ldrh	r3, [r7, #24]
 800217a:	4413      	add	r3, r2
 800217c:	b29b      	uxth	r3, r3
 800217e:	b219      	sxth	r1, r3
 8002180:	893a      	ldrh	r2, [r7, #8]
 8002182:	8afb      	ldrh	r3, [r7, #22]
 8002184:	1ad3      	subs	r3, r2, r3
 8002186:	b29b      	uxth	r3, r3
 8002188:	b218      	sxth	r0, r3
 800218a:	8afb      	ldrh	r3, [r7, #22]
 800218c:	005b      	lsls	r3, r3, #1
 800218e:	b29a      	uxth	r2, r3
 8002190:	8dbb      	ldrh	r3, [r7, #44]	; 0x2c
 8002192:	4413      	add	r3, r2
 8002194:	b29b      	uxth	r3, r3
 8002196:	3301      	adds	r3, #1
 8002198:	b29b      	uxth	r3, r3
 800219a:	b21a      	sxth	r2, r3
 800219c:	8e3b      	ldrh	r3, [r7, #48]	; 0x30
 800219e:	9300      	str	r3, [sp, #0]
 80021a0:	4613      	mov	r3, r2
 80021a2:	4602      	mov	r2, r0
 80021a4:	68f8      	ldr	r0, [r7, #12]
 80021a6:	f000 f943 	bl	8002430 <_ZN8Graphics13drawFastVLineEssst>
      drawFastVLine(x0+y, y0-x, 2*x+1+delta, color);
 80021aa:	897a      	ldrh	r2, [r7, #10]
 80021ac:	8afb      	ldrh	r3, [r7, #22]
 80021ae:	4413      	add	r3, r2
 80021b0:	b29b      	uxth	r3, r3
 80021b2:	b219      	sxth	r1, r3
 80021b4:	893a      	ldrh	r2, [r7, #8]
 80021b6:	8b3b      	ldrh	r3, [r7, #24]
 80021b8:	1ad3      	subs	r3, r2, r3
 80021ba:	b29b      	uxth	r3, r3
 80021bc:	b218      	sxth	r0, r3
 80021be:	8b3b      	ldrh	r3, [r7, #24]
 80021c0:	005b      	lsls	r3, r3, #1
 80021c2:	b29a      	uxth	r2, r3
 80021c4:	8dbb      	ldrh	r3, [r7, #44]	; 0x2c
 80021c6:	4413      	add	r3, r2
 80021c8:	b29b      	uxth	r3, r3
 80021ca:	3301      	adds	r3, #1
 80021cc:	b29b      	uxth	r3, r3
 80021ce:	b21a      	sxth	r2, r3
 80021d0:	8e3b      	ldrh	r3, [r7, #48]	; 0x30
 80021d2:	9300      	str	r3, [sp, #0]
 80021d4:	4613      	mov	r3, r2
 80021d6:	4602      	mov	r2, r0
 80021d8:	68f8      	ldr	r0, [r7, #12]
 80021da:	f000 f929 	bl	8002430 <_ZN8Graphics13drawFastVLineEssst>
    }
    if (cornername & 0x2)
 80021de:	f897 3028 	ldrb.w	r3, [r7, #40]	; 0x28
 80021e2:	f003 0302 	and.w	r3, r3, #2
 80021e6:	2b00      	cmp	r3, #0
 80021e8:	d096      	beq.n	8002118 <_ZN8Graphics16fillCircleHelperEssshst+0x3e>
    {
      drawFastVLine(x0-x, y0-y, 2*y+1+delta, color);
 80021ea:	897a      	ldrh	r2, [r7, #10]
 80021ec:	8b3b      	ldrh	r3, [r7, #24]
 80021ee:	1ad3      	subs	r3, r2, r3
 80021f0:	b29b      	uxth	r3, r3
 80021f2:	b219      	sxth	r1, r3
 80021f4:	893a      	ldrh	r2, [r7, #8]
 80021f6:	8afb      	ldrh	r3, [r7, #22]
 80021f8:	1ad3      	subs	r3, r2, r3
 80021fa:	b29b      	uxth	r3, r3
 80021fc:	b218      	sxth	r0, r3
 80021fe:	8afb      	ldrh	r3, [r7, #22]
 8002200:	005b      	lsls	r3, r3, #1
 8002202:	b29a      	uxth	r2, r3
 8002204:	8dbb      	ldrh	r3, [r7, #44]	; 0x2c
 8002206:	4413      	add	r3, r2
 8002208:	b29b      	uxth	r3, r3
 800220a:	3301      	adds	r3, #1
 800220c:	b29b      	uxth	r3, r3
 800220e:	b21a      	sxth	r2, r3
 8002210:	8e3b      	ldrh	r3, [r7, #48]	; 0x30
 8002212:	9300      	str	r3, [sp, #0]
 8002214:	4613      	mov	r3, r2
 8002216:	4602      	mov	r2, r0
 8002218:	68f8      	ldr	r0, [r7, #12]
 800221a:	f000 f909 	bl	8002430 <_ZN8Graphics13drawFastVLineEssst>
      drawFastVLine(x0-y, y0-x, 2*x+1+delta, color);
 800221e:	897a      	ldrh	r2, [r7, #10]
 8002220:	8afb      	ldrh	r3, [r7, #22]
 8002222:	1ad3      	subs	r3, r2, r3
 8002224:	b29b      	uxth	r3, r3
 8002226:	b219      	sxth	r1, r3
 8002228:	893a      	ldrh	r2, [r7, #8]
 800222a:	8b3b      	ldrh	r3, [r7, #24]
 800222c:	1ad3      	subs	r3, r2, r3
 800222e:	b29b      	uxth	r3, r3
 8002230:	b218      	sxth	r0, r3
 8002232:	8b3b      	ldrh	r3, [r7, #24]
 8002234:	005b      	lsls	r3, r3, #1
 8002236:	b29a      	uxth	r2, r3
 8002238:	8dbb      	ldrh	r3, [r7, #44]	; 0x2c
 800223a:	4413      	add	r3, r2
 800223c:	b29b      	uxth	r3, r3
 800223e:	3301      	adds	r3, #1
 8002240:	b29b      	uxth	r3, r3
 8002242:	b21a      	sxth	r2, r3
 8002244:	8e3b      	ldrh	r3, [r7, #48]	; 0x30
 8002246:	9300      	str	r3, [sp, #0]
 8002248:	4613      	mov	r3, r2
 800224a:	4602      	mov	r2, r0
 800224c:	68f8      	ldr	r0, [r7, #12]
 800224e:	f000 f8ef 	bl	8002430 <_ZN8Graphics13drawFastVLineEssst>
  while (x<y)
 8002252:	e761      	b.n	8002118 <_ZN8Graphics16fillCircleHelperEssshst+0x3e>
    }
  }
}
 8002254:	bf00      	nop
 8002256:	3720      	adds	r7, #32
 8002258:	46bd      	mov	sp, r7
 800225a:	bd80      	pop	{r7, pc}

0800225c <_ZN8Graphics8drawLineEsssst>:
    @param    y1  End point y coordinate
    @param    color 0 - white 1 - black
*/
/**************************************************************************/
void Graphics::drawLine(int16_t x0, int16_t y0, int16_t x1, int16_t y1, uint16_t color)
{
 800225c:	b580      	push	{r7, lr}
 800225e:	b08a      	sub	sp, #40	; 0x28
 8002260:	af00      	add	r7, sp, #0
 8002262:	60f8      	str	r0, [r7, #12]
 8002264:	4608      	mov	r0, r1
 8002266:	4611      	mov	r1, r2
 8002268:	461a      	mov	r2, r3
 800226a:	4603      	mov	r3, r0
 800226c:	817b      	strh	r3, [r7, #10]
 800226e:	460b      	mov	r3, r1
 8002270:	813b      	strh	r3, [r7, #8]
 8002272:	4613      	mov	r3, r2
 8002274:	80fb      	strh	r3, [r7, #6]
#ifdef DEBUGLOW
  printf("x0=%d,y0=%d,x1=%d,y1=%d,color=%d\n",x0,y0,x1,y1,color);
#endif
  int16_t steep = abs(y1 - y0) > abs(x1 - x0);
 8002276:	f9b7 2030 	ldrsh.w	r2, [r7, #48]	; 0x30
 800227a:	f9b7 3008 	ldrsh.w	r3, [r7, #8]
 800227e:	1ad3      	subs	r3, r2, r3
 8002280:	ea83 72e3 	eor.w	r2, r3, r3, asr #31
 8002284:	eba2 72e3 	sub.w	r2, r2, r3, asr #31
 8002288:	f9b7 1006 	ldrsh.w	r1, [r7, #6]
 800228c:	f9b7 300a 	ldrsh.w	r3, [r7, #10]
 8002290:	1acb      	subs	r3, r1, r3
 8002292:	2b00      	cmp	r3, #0
 8002294:	bfb8      	it	lt
 8002296:	425b      	neglt	r3, r3
 8002298:	429a      	cmp	r2, r3
 800229a:	bfcc      	ite	gt
 800229c:	2301      	movgt	r3, #1
 800229e:	2300      	movle	r3, #0
 80022a0:	b2db      	uxtb	r3, r3
 80022a2:	847b      	strh	r3, [r7, #34]	; 0x22
  if (steep)
 80022a4:	f9b7 3022 	ldrsh.w	r3, [r7, #34]	; 0x22
 80022a8:	2b00      	cmp	r3, #0
 80022aa:	d00b      	beq.n	80022c4 <_ZN8Graphics8drawLineEsssst+0x68>
  {
    _swap_int16_t(x0, y0);
 80022ac:	897b      	ldrh	r3, [r7, #10]
 80022ae:	843b      	strh	r3, [r7, #32]
 80022b0:	893b      	ldrh	r3, [r7, #8]
 80022b2:	817b      	strh	r3, [r7, #10]
 80022b4:	8c3b      	ldrh	r3, [r7, #32]
 80022b6:	813b      	strh	r3, [r7, #8]
    _swap_int16_t(x1, y1);
 80022b8:	88fb      	ldrh	r3, [r7, #6]
 80022ba:	83fb      	strh	r3, [r7, #30]
 80022bc:	8e3b      	ldrh	r3, [r7, #48]	; 0x30
 80022be:	80fb      	strh	r3, [r7, #6]
 80022c0:	8bfb      	ldrh	r3, [r7, #30]
 80022c2:	863b      	strh	r3, [r7, #48]	; 0x30
  }

  if (x0 > x1)
 80022c4:	f9b7 200a 	ldrsh.w	r2, [r7, #10]
 80022c8:	f9b7 3006 	ldrsh.w	r3, [r7, #6]
 80022cc:	429a      	cmp	r2, r3
 80022ce:	dd0b      	ble.n	80022e8 <_ZN8Graphics8drawLineEsssst+0x8c>
  {
    _swap_int16_t(x0, x1);
 80022d0:	897b      	ldrh	r3, [r7, #10]
 80022d2:	83bb      	strh	r3, [r7, #28]
 80022d4:	88fb      	ldrh	r3, [r7, #6]
 80022d6:	817b      	strh	r3, [r7, #10]
 80022d8:	8bbb      	ldrh	r3, [r7, #28]
 80022da:	80fb      	strh	r3, [r7, #6]
    _swap_int16_t(y0, y1);
 80022dc:	893b      	ldrh	r3, [r7, #8]
 80022de:	837b      	strh	r3, [r7, #26]
 80022e0:	8e3b      	ldrh	r3, [r7, #48]	; 0x30
 80022e2:	813b      	strh	r3, [r7, #8]
 80022e4:	8b7b      	ldrh	r3, [r7, #26]
 80022e6:	863b      	strh	r3, [r7, #48]	; 0x30
  }

  int16_t dx, dy;
  dx = x1 - x0;
 80022e8:	88fa      	ldrh	r2, [r7, #6]
 80022ea:	897b      	ldrh	r3, [r7, #10]
 80022ec:	1ad3      	subs	r3, r2, r3
 80022ee:	b29b      	uxth	r3, r3
 80022f0:	833b      	strh	r3, [r7, #24]
  dy = abs(y1 - y0);
 80022f2:	f9b7 2030 	ldrsh.w	r2, [r7, #48]	; 0x30
 80022f6:	f9b7 3008 	ldrsh.w	r3, [r7, #8]
 80022fa:	1ad3      	subs	r3, r2, r3
 80022fc:	2b00      	cmp	r3, #0
 80022fe:	bfb8      	it	lt
 8002300:	425b      	neglt	r3, r3
 8002302:	82fb      	strh	r3, [r7, #22]

#ifdef DEBUGLOW
  printf("x0=%d,y0=%d,x1=%d,y1=%d,dx=%d,dy=%d\n",x0,y0,x1,y1,dx,dy);
#endif

  int16_t err = dx / 2;
 8002304:	f9b7 3018 	ldrsh.w	r3, [r7, #24]
 8002308:	0fda      	lsrs	r2, r3, #31
 800230a:	4413      	add	r3, r2
 800230c:	105b      	asrs	r3, r3, #1
 800230e:	84fb      	strh	r3, [r7, #38]	; 0x26
  int16_t ystep;

  if (y0 < y1)
 8002310:	f9b7 2008 	ldrsh.w	r2, [r7, #8]
 8002314:	f9b7 3030 	ldrsh.w	r3, [r7, #48]	; 0x30
 8002318:	429a      	cmp	r2, r3
 800231a:	da02      	bge.n	8002322 <_ZN8Graphics8drawLineEsssst+0xc6>
  {
    ystep = 1;
 800231c:	2301      	movs	r3, #1
 800231e:	84bb      	strh	r3, [r7, #36]	; 0x24
 8002320:	e002      	b.n	8002328 <_ZN8Graphics8drawLineEsssst+0xcc>
  }
  else
  {
    ystep = -1;
 8002322:	f64f 73ff 	movw	r3, #65535	; 0xffff
 8002326:	84bb      	strh	r3, [r7, #36]	; 0x24
  }

  for (; x0<=x1; x0++)
 8002328:	f9b7 200a 	ldrsh.w	r2, [r7, #10]
 800232c:	f9b7 3006 	ldrsh.w	r3, [r7, #6]
 8002330:	429a      	cmp	r2, r3
 8002332:	dc2e      	bgt.n	8002392 <_ZN8Graphics8drawLineEsssst+0x136>
  {
    if (steep)
 8002334:	f9b7 3022 	ldrsh.w	r3, [r7, #34]	; 0x22
 8002338:	2b00      	cmp	r3, #0
 800233a:	d008      	beq.n	800234e <_ZN8Graphics8drawLineEsssst+0xf2>
    {
      drawPixel(y0, x0, color);
 800233c:	8ebb      	ldrh	r3, [r7, #52]	; 0x34
 800233e:	f9b7 200a 	ldrsh.w	r2, [r7, #10]
 8002342:	f9b7 1008 	ldrsh.w	r1, [r7, #8]
 8002346:	68f8      	ldr	r0, [r7, #12]
 8002348:	f7ff fb0a 	bl	8001960 <_ZN8Graphics9drawPixelEsst>
 800234c:	e007      	b.n	800235e <_ZN8Graphics8drawLineEsssst+0x102>
    }
    else
    {
      drawPixel(x0, y0, color);
 800234e:	8ebb      	ldrh	r3, [r7, #52]	; 0x34
 8002350:	f9b7 2008 	ldrsh.w	r2, [r7, #8]
 8002354:	f9b7 100a 	ldrsh.w	r1, [r7, #10]
 8002358:	68f8      	ldr	r0, [r7, #12]
 800235a:	f7ff fb01 	bl	8001960 <_ZN8Graphics9drawPixelEsst>
    }
    err -= dy;
 800235e:	8cfa      	ldrh	r2, [r7, #38]	; 0x26
 8002360:	8afb      	ldrh	r3, [r7, #22]
 8002362:	1ad3      	subs	r3, r2, r3
 8002364:	b29b      	uxth	r3, r3
 8002366:	84fb      	strh	r3, [r7, #38]	; 0x26

    if (err < 0)
 8002368:	f9b7 3026 	ldrsh.w	r3, [r7, #38]	; 0x26
 800236c:	2b00      	cmp	r3, #0
 800236e:	da09      	bge.n	8002384 <_ZN8Graphics8drawLineEsssst+0x128>
    {
      y0 += ystep;
 8002370:	893a      	ldrh	r2, [r7, #8]
 8002372:	8cbb      	ldrh	r3, [r7, #36]	; 0x24
 8002374:	4413      	add	r3, r2
 8002376:	b29b      	uxth	r3, r3
 8002378:	813b      	strh	r3, [r7, #8]
      err += dx;
 800237a:	8cfa      	ldrh	r2, [r7, #38]	; 0x26
 800237c:	8b3b      	ldrh	r3, [r7, #24]
 800237e:	4413      	add	r3, r2
 8002380:	b29b      	uxth	r3, r3
 8002382:	84fb      	strh	r3, [r7, #38]	; 0x26
  for (; x0<=x1; x0++)
 8002384:	f9b7 300a 	ldrsh.w	r3, [r7, #10]
 8002388:	b29b      	uxth	r3, r3
 800238a:	3301      	adds	r3, #1
 800238c:	b29b      	uxth	r3, r3
 800238e:	817b      	strh	r3, [r7, #10]
 8002390:	e7ca      	b.n	8002328 <_ZN8Graphics8drawLineEsssst+0xcc>
    }
  }
}
 8002392:	bf00      	nop
 8002394:	3728      	adds	r7, #40	; 0x28
 8002396:	46bd      	mov	sp, r7
 8002398:	bd80      	pop	{r7, pc}

0800239a <_ZN8Graphics8drawRectEsssst>:
    @param    h   Height in pixels
    @param    color 0 - white 1 - black
*/
/**************************************************************************/
void Graphics::drawRect(int16_t x, int16_t y, int16_t w, int16_t h, uint16_t color)
{
 800239a:	b580      	push	{r7, lr}
 800239c:	b086      	sub	sp, #24
 800239e:	af02      	add	r7, sp, #8
 80023a0:	60f8      	str	r0, [r7, #12]
 80023a2:	4608      	mov	r0, r1
 80023a4:	4611      	mov	r1, r2
 80023a6:	461a      	mov	r2, r3
 80023a8:	4603      	mov	r3, r0
 80023aa:	817b      	strh	r3, [r7, #10]
 80023ac:	460b      	mov	r3, r1
 80023ae:	813b      	strh	r3, [r7, #8]
 80023b0:	4613      	mov	r3, r2
 80023b2:	80fb      	strh	r3, [r7, #6]
  drawFastHLine(x, y, w, color);
 80023b4:	f9b7 0006 	ldrsh.w	r0, [r7, #6]
 80023b8:	f9b7 2008 	ldrsh.w	r2, [r7, #8]
 80023bc:	f9b7 100a 	ldrsh.w	r1, [r7, #10]
 80023c0:	8bbb      	ldrh	r3, [r7, #28]
 80023c2:	9300      	str	r3, [sp, #0]
 80023c4:	4603      	mov	r3, r0
 80023c6:	68f8      	ldr	r0, [r7, #12]
 80023c8:	f000 f858 	bl	800247c <_ZN8Graphics13drawFastHLineEssst>
  drawFastHLine(x, y+h-1, w, color);
 80023cc:	893a      	ldrh	r2, [r7, #8]
 80023ce:	8b3b      	ldrh	r3, [r7, #24]
 80023d0:	4413      	add	r3, r2
 80023d2:	b29b      	uxth	r3, r3
 80023d4:	3b01      	subs	r3, #1
 80023d6:	b29b      	uxth	r3, r3
 80023d8:	b21a      	sxth	r2, r3
 80023da:	f9b7 0006 	ldrsh.w	r0, [r7, #6]
 80023de:	f9b7 100a 	ldrsh.w	r1, [r7, #10]
 80023e2:	8bbb      	ldrh	r3, [r7, #28]
 80023e4:	9300      	str	r3, [sp, #0]
 80023e6:	4603      	mov	r3, r0
 80023e8:	68f8      	ldr	r0, [r7, #12]
 80023ea:	f000 f847 	bl	800247c <_ZN8Graphics13drawFastHLineEssst>
  drawFastVLine(x, y, h, color);
 80023ee:	f9b7 0018 	ldrsh.w	r0, [r7, #24]
 80023f2:	f9b7 2008 	ldrsh.w	r2, [r7, #8]
 80023f6:	f9b7 100a 	ldrsh.w	r1, [r7, #10]
 80023fa:	8bbb      	ldrh	r3, [r7, #28]
 80023fc:	9300      	str	r3, [sp, #0]
 80023fe:	4603      	mov	r3, r0
 8002400:	68f8      	ldr	r0, [r7, #12]
 8002402:	f000 f815 	bl	8002430 <_ZN8Graphics13drawFastVLineEssst>
  drawFastVLine(x+w-1, y, h, color);
 8002406:	897a      	ldrh	r2, [r7, #10]
 8002408:	88fb      	ldrh	r3, [r7, #6]
 800240a:	4413      	add	r3, r2
 800240c:	b29b      	uxth	r3, r3
 800240e:	3b01      	subs	r3, #1
 8002410:	b29b      	uxth	r3, r3
 8002412:	b219      	sxth	r1, r3
 8002414:	f9b7 0018 	ldrsh.w	r0, [r7, #24]
 8002418:	f9b7 2008 	ldrsh.w	r2, [r7, #8]
 800241c:	8bbb      	ldrh	r3, [r7, #28]
 800241e:	9300      	str	r3, [sp, #0]
 8002420:	4603      	mov	r3, r0
 8002422:	68f8      	ldr	r0, [r7, #12]
 8002424:	f000 f804 	bl	8002430 <_ZN8Graphics13drawFastVLineEssst>
}
 8002428:	bf00      	nop
 800242a:	3710      	adds	r7, #16
 800242c:	46bd      	mov	sp, r7
 800242e:	bd80      	pop	{r7, pc}

08002430 <_ZN8Graphics13drawFastVLineEssst>:
    @param    h   Height in pixels
   @param    color 0 - white 1 - black
*/
/**************************************************************************/
void Graphics::drawFastVLine(int16_t x, int16_t y, int16_t h, uint16_t color)
{
 8002430:	b590      	push	{r4, r7, lr}
 8002432:	b087      	sub	sp, #28
 8002434:	af02      	add	r7, sp, #8
 8002436:	60f8      	str	r0, [r7, #12]
 8002438:	4608      	mov	r0, r1
 800243a:	4611      	mov	r1, r2
 800243c:	461a      	mov	r2, r3
 800243e:	4603      	mov	r3, r0
 8002440:	817b      	strh	r3, [r7, #10]
 8002442:	460b      	mov	r3, r1
 8002444:	813b      	strh	r3, [r7, #8]
 8002446:	4613      	mov	r3, r2
 8002448:	80fb      	strh	r3, [r7, #6]
  // Update in subclasses if desired!
  drawLine(x, y, x, y+h-1, color);
 800244a:	893a      	ldrh	r2, [r7, #8]
 800244c:	88fb      	ldrh	r3, [r7, #6]
 800244e:	4413      	add	r3, r2
 8002450:	b29b      	uxth	r3, r3
 8002452:	3b01      	subs	r3, #1
 8002454:	b29b      	uxth	r3, r3
 8002456:	b21b      	sxth	r3, r3
 8002458:	f9b7 400a 	ldrsh.w	r4, [r7, #10]
 800245c:	f9b7 0008 	ldrsh.w	r0, [r7, #8]
 8002460:	f9b7 100a 	ldrsh.w	r1, [r7, #10]
 8002464:	8c3a      	ldrh	r2, [r7, #32]
 8002466:	9201      	str	r2, [sp, #4]
 8002468:	9300      	str	r3, [sp, #0]
 800246a:	4623      	mov	r3, r4
 800246c:	4602      	mov	r2, r0
 800246e:	68f8      	ldr	r0, [r7, #12]
 8002470:	f7ff fef4 	bl	800225c <_ZN8Graphics8drawLineEsssst>
}
 8002474:	bf00      	nop
 8002476:	3714      	adds	r7, #20
 8002478:	46bd      	mov	sp, r7
 800247a:	bd90      	pop	{r4, r7, pc}

0800247c <_ZN8Graphics13drawFastHLineEssst>:
    @param    w   Width in pixels
   @param    color 0 - white 1 - black
*/
/**************************************************************************/
void Graphics::drawFastHLine(int16_t x, int16_t y, int16_t w, uint16_t color)
{
 800247c:	b580      	push	{r7, lr}
 800247e:	b086      	sub	sp, #24
 8002480:	af02      	add	r7, sp, #8
 8002482:	60f8      	str	r0, [r7, #12]
 8002484:	4608      	mov	r0, r1
 8002486:	4611      	mov	r1, r2
 8002488:	461a      	mov	r2, r3
 800248a:	4603      	mov	r3, r0
 800248c:	817b      	strh	r3, [r7, #10]
 800248e:	460b      	mov	r3, r1
 8002490:	813b      	strh	r3, [r7, #8]
 8002492:	4613      	mov	r3, r2
 8002494:	80fb      	strh	r3, [r7, #6]
  // Update in subclasses if desired!
  drawLine(x, y, x+w-1, y, color);
 8002496:	897a      	ldrh	r2, [r7, #10]
 8002498:	88fb      	ldrh	r3, [r7, #6]
 800249a:	4413      	add	r3, r2
 800249c:	b29b      	uxth	r3, r3
 800249e:	3b01      	subs	r3, #1
 80024a0:	b29b      	uxth	r3, r3
 80024a2:	b218      	sxth	r0, r3
 80024a4:	f9b7 2008 	ldrsh.w	r2, [r7, #8]
 80024a8:	f9b7 100a 	ldrsh.w	r1, [r7, #10]
 80024ac:	8b3b      	ldrh	r3, [r7, #24]
 80024ae:	9301      	str	r3, [sp, #4]
 80024b0:	f9b7 3008 	ldrsh.w	r3, [r7, #8]
 80024b4:	9300      	str	r3, [sp, #0]
 80024b6:	4603      	mov	r3, r0
 80024b8:	68f8      	ldr	r0, [r7, #12]
 80024ba:	f7ff fecf 	bl	800225c <_ZN8Graphics8drawLineEsssst>
}
 80024be:	bf00      	nop
 80024c0:	3710      	adds	r7, #16
 80024c2:	46bd      	mov	sp, r7
 80024c4:	bd80      	pop	{r7, pc}

080024c6 <_ZN8Graphics8fillRectEsssst>:
    @param    h   Height in pixels
   @param    color 0 - white 1 - black
*/
/**************************************************************************/
void Graphics::fillRect(int16_t x, int16_t y, int16_t w, int16_t h, uint16_t color)
{
 80024c6:	b580      	push	{r7, lr}
 80024c8:	b088      	sub	sp, #32
 80024ca:	af02      	add	r7, sp, #8
 80024cc:	60f8      	str	r0, [r7, #12]
 80024ce:	4608      	mov	r0, r1
 80024d0:	4611      	mov	r1, r2
 80024d2:	461a      	mov	r2, r3
 80024d4:	4603      	mov	r3, r0
 80024d6:	817b      	strh	r3, [r7, #10]
 80024d8:	460b      	mov	r3, r1
 80024da:	813b      	strh	r3, [r7, #8]
 80024dc:	4613      	mov	r3, r2
 80024de:	80fb      	strh	r3, [r7, #6]
  // Update in subclasses if desired!
  for (int16_t i=x; i<x+w; i++)
 80024e0:	897b      	ldrh	r3, [r7, #10]
 80024e2:	82fb      	strh	r3, [r7, #22]
 80024e4:	f9b7 2016 	ldrsh.w	r2, [r7, #22]
 80024e8:	f9b7 100a 	ldrsh.w	r1, [r7, #10]
 80024ec:	f9b7 3006 	ldrsh.w	r3, [r7, #6]
 80024f0:	440b      	add	r3, r1
 80024f2:	429a      	cmp	r2, r3
 80024f4:	da12      	bge.n	800251c <_ZN8Graphics8fillRectEsssst+0x56>
  {
    drawFastVLine(i, y, h, color);
 80024f6:	f9b7 0020 	ldrsh.w	r0, [r7, #32]
 80024fa:	f9b7 2008 	ldrsh.w	r2, [r7, #8]
 80024fe:	f9b7 1016 	ldrsh.w	r1, [r7, #22]
 8002502:	8cbb      	ldrh	r3, [r7, #36]	; 0x24
 8002504:	9300      	str	r3, [sp, #0]
 8002506:	4603      	mov	r3, r0
 8002508:	68f8      	ldr	r0, [r7, #12]
 800250a:	f7ff ff91 	bl	8002430 <_ZN8Graphics13drawFastVLineEssst>
  for (int16_t i=x; i<x+w; i++)
 800250e:	f9b7 3016 	ldrsh.w	r3, [r7, #22]
 8002512:	b29b      	uxth	r3, r3
 8002514:	3301      	adds	r3, #1
 8002516:	b29b      	uxth	r3, r3
 8002518:	82fb      	strh	r3, [r7, #22]
 800251a:	e7e3      	b.n	80024e4 <_ZN8Graphics8fillRectEsssst+0x1e>
  }
}
 800251c:	bf00      	nop
 800251e:	3718      	adds	r7, #24
 8002520:	46bd      	mov	sp, r7
 8002522:	bd80      	pop	{r7, pc}

08002524 <_ZN8Graphics13fillRoundRectEssssst>:
    @param    r   Radius of corner rounding
    @param    color 0 - white 1 - black
*/
/**************************************************************************/
void Graphics::fillRoundRect(int16_t x, int16_t y, int16_t w, int16_t h, int16_t r, uint16_t color)
{
 8002524:	b590      	push	{r4, r7, lr}
 8002526:	b089      	sub	sp, #36	; 0x24
 8002528:	af04      	add	r7, sp, #16
 800252a:	60f8      	str	r0, [r7, #12]
 800252c:	4608      	mov	r0, r1
 800252e:	4611      	mov	r1, r2
 8002530:	461a      	mov	r2, r3
 8002532:	4603      	mov	r3, r0
 8002534:	817b      	strh	r3, [r7, #10]
 8002536:	460b      	mov	r3, r1
 8002538:	813b      	strh	r3, [r7, #8]
 800253a:	4613      	mov	r3, r2
 800253c:	80fb      	strh	r3, [r7, #6]
  // color = getColor(color);
  // smarter version
  fillRect(x+r, y, w-2*r, h, color);
 800253e:	897a      	ldrh	r2, [r7, #10]
 8002540:	8cbb      	ldrh	r3, [r7, #36]	; 0x24
 8002542:	4413      	add	r3, r2
 8002544:	b29b      	uxth	r3, r3
 8002546:	b219      	sxth	r1, r3
 8002548:	88fa      	ldrh	r2, [r7, #6]
 800254a:	8cbb      	ldrh	r3, [r7, #36]	; 0x24
 800254c:	005b      	lsls	r3, r3, #1
 800254e:	b29b      	uxth	r3, r3
 8002550:	1ad3      	subs	r3, r2, r3
 8002552:	b29b      	uxth	r3, r3
 8002554:	b218      	sxth	r0, r3
 8002556:	f9b7 2008 	ldrsh.w	r2, [r7, #8]
 800255a:	8d3b      	ldrh	r3, [r7, #40]	; 0x28
 800255c:	9301      	str	r3, [sp, #4]
 800255e:	f9b7 3020 	ldrsh.w	r3, [r7, #32]
 8002562:	9300      	str	r3, [sp, #0]
 8002564:	4603      	mov	r3, r0
 8002566:	68f8      	ldr	r0, [r7, #12]
 8002568:	f7ff ffad 	bl	80024c6 <_ZN8Graphics8fillRectEsssst>

  // draw four corners
  fillCircleHelper(x+w-r-1, y+r, r, 1, h-2*r-1, color);
 800256c:	897a      	ldrh	r2, [r7, #10]
 800256e:	88fb      	ldrh	r3, [r7, #6]
 8002570:	4413      	add	r3, r2
 8002572:	b29a      	uxth	r2, r3
 8002574:	8cbb      	ldrh	r3, [r7, #36]	; 0x24
 8002576:	1ad3      	subs	r3, r2, r3
 8002578:	b29b      	uxth	r3, r3
 800257a:	3b01      	subs	r3, #1
 800257c:	b29b      	uxth	r3, r3
 800257e:	b219      	sxth	r1, r3
 8002580:	893a      	ldrh	r2, [r7, #8]
 8002582:	8cbb      	ldrh	r3, [r7, #36]	; 0x24
 8002584:	4413      	add	r3, r2
 8002586:	b29b      	uxth	r3, r3
 8002588:	b218      	sxth	r0, r3
 800258a:	8c3a      	ldrh	r2, [r7, #32]
 800258c:	8cbb      	ldrh	r3, [r7, #36]	; 0x24
 800258e:	005b      	lsls	r3, r3, #1
 8002590:	b29b      	uxth	r3, r3
 8002592:	1ad3      	subs	r3, r2, r3
 8002594:	b29b      	uxth	r3, r3
 8002596:	3b01      	subs	r3, #1
 8002598:	b29b      	uxth	r3, r3
 800259a:	b21b      	sxth	r3, r3
 800259c:	f9b7 4024 	ldrsh.w	r4, [r7, #36]	; 0x24
 80025a0:	8d3a      	ldrh	r2, [r7, #40]	; 0x28
 80025a2:	9202      	str	r2, [sp, #8]
 80025a4:	9301      	str	r3, [sp, #4]
 80025a6:	2301      	movs	r3, #1
 80025a8:	9300      	str	r3, [sp, #0]
 80025aa:	4623      	mov	r3, r4
 80025ac:	4602      	mov	r2, r0
 80025ae:	68f8      	ldr	r0, [r7, #12]
 80025b0:	f7ff fd93 	bl	80020da <_ZN8Graphics16fillCircleHelperEssshst>
  fillCircleHelper(x+r, y+r, r, 2, h-2*r-1, color);
 80025b4:	897a      	ldrh	r2, [r7, #10]
 80025b6:	8cbb      	ldrh	r3, [r7, #36]	; 0x24
 80025b8:	4413      	add	r3, r2
 80025ba:	b29b      	uxth	r3, r3
 80025bc:	b219      	sxth	r1, r3
 80025be:	893a      	ldrh	r2, [r7, #8]
 80025c0:	8cbb      	ldrh	r3, [r7, #36]	; 0x24
 80025c2:	4413      	add	r3, r2
 80025c4:	b29b      	uxth	r3, r3
 80025c6:	b218      	sxth	r0, r3
 80025c8:	8c3a      	ldrh	r2, [r7, #32]
 80025ca:	8cbb      	ldrh	r3, [r7, #36]	; 0x24
 80025cc:	005b      	lsls	r3, r3, #1
 80025ce:	b29b      	uxth	r3, r3
 80025d0:	1ad3      	subs	r3, r2, r3
 80025d2:	b29b      	uxth	r3, r3
 80025d4:	3b01      	subs	r3, #1
 80025d6:	b29b      	uxth	r3, r3
 80025d8:	b21b      	sxth	r3, r3
 80025da:	f9b7 4024 	ldrsh.w	r4, [r7, #36]	; 0x24
 80025de:	8d3a      	ldrh	r2, [r7, #40]	; 0x28
 80025e0:	9202      	str	r2, [sp, #8]
 80025e2:	9301      	str	r3, [sp, #4]
 80025e4:	2302      	movs	r3, #2
 80025e6:	9300      	str	r3, [sp, #0]
 80025e8:	4623      	mov	r3, r4
 80025ea:	4602      	mov	r2, r0
 80025ec:	68f8      	ldr	r0, [r7, #12]
 80025ee:	f7ff fd74 	bl	80020da <_ZN8Graphics16fillCircleHelperEssshst>
}
 80025f2:	bf00      	nop
 80025f4:	3714      	adds	r7, #20
 80025f6:	46bd      	mov	sp, r7
 80025f8:	bd90      	pop	{r4, r7, pc}

080025fa <_ZN8Graphics12fillTriangleEsssssst>:
    @param    y2  Vertex #2 y coordinate
    @param    color 0 - white 1 - black
*/
/**************************************************************************/
void Graphics::fillTriangle(int16_t x0, int16_t y0, int16_t x1, int16_t y1, int16_t x2, int16_t y2, uint16_t color)
{
 80025fa:	b580      	push	{r7, lr}
 80025fc:	b092      	sub	sp, #72	; 0x48
 80025fe:	af02      	add	r7, sp, #8
 8002600:	60f8      	str	r0, [r7, #12]
 8002602:	4608      	mov	r0, r1
 8002604:	4611      	mov	r1, r2
 8002606:	461a      	mov	r2, r3
 8002608:	4603      	mov	r3, r0
 800260a:	817b      	strh	r3, [r7, #10]
 800260c:	460b      	mov	r3, r1
 800260e:	813b      	strh	r3, [r7, #8]
 8002610:	4613      	mov	r3, r2
 8002612:	80fb      	strh	r3, [r7, #6]
  // color = getColor(color);
  int16_t a, b, y, last;

  // Sort coordinates by Y order (y2 >= y1 >= y0)
  if (y0 > y1)
 8002614:	f9b7 2008 	ldrsh.w	r2, [r7, #8]
 8002618:	f9b7 3048 	ldrsh.w	r3, [r7, #72]	; 0x48
 800261c:	429a      	cmp	r2, r3
 800261e:	dd0d      	ble.n	800263c <_ZN8Graphics12fillTriangleEsssssst+0x42>
  {
    _swap_int16_t(y0, y1);
 8002620:	893b      	ldrh	r3, [r7, #8]
 8002622:	85fb      	strh	r3, [r7, #46]	; 0x2e
 8002624:	f8b7 3048 	ldrh.w	r3, [r7, #72]	; 0x48
 8002628:	813b      	strh	r3, [r7, #8]
 800262a:	8dfb      	ldrh	r3, [r7, #46]	; 0x2e
 800262c:	f8a7 3048 	strh.w	r3, [r7, #72]	; 0x48
    _swap_int16_t(x0, x1);
 8002630:	897b      	ldrh	r3, [r7, #10]
 8002632:	85bb      	strh	r3, [r7, #44]	; 0x2c
 8002634:	88fb      	ldrh	r3, [r7, #6]
 8002636:	817b      	strh	r3, [r7, #10]
 8002638:	8dbb      	ldrh	r3, [r7, #44]	; 0x2c
 800263a:	80fb      	strh	r3, [r7, #6]
  }

  if (y1 > y2)
 800263c:	f9b7 2048 	ldrsh.w	r2, [r7, #72]	; 0x48
 8002640:	f9b7 3050 	ldrsh.w	r3, [r7, #80]	; 0x50
 8002644:	429a      	cmp	r2, r3
 8002646:	dd11      	ble.n	800266c <_ZN8Graphics12fillTriangleEsssssst+0x72>
  {
    _swap_int16_t(y2, y1);
 8002648:	f8b7 3050 	ldrh.w	r3, [r7, #80]	; 0x50
 800264c:	857b      	strh	r3, [r7, #42]	; 0x2a
 800264e:	f8b7 3048 	ldrh.w	r3, [r7, #72]	; 0x48
 8002652:	f8a7 3050 	strh.w	r3, [r7, #80]	; 0x50
 8002656:	8d7b      	ldrh	r3, [r7, #42]	; 0x2a
 8002658:	f8a7 3048 	strh.w	r3, [r7, #72]	; 0x48
    _swap_int16_t(x2, x1);
 800265c:	f8b7 304c 	ldrh.w	r3, [r7, #76]	; 0x4c
 8002660:	853b      	strh	r3, [r7, #40]	; 0x28
 8002662:	88fb      	ldrh	r3, [r7, #6]
 8002664:	f8a7 304c 	strh.w	r3, [r7, #76]	; 0x4c
 8002668:	8d3b      	ldrh	r3, [r7, #40]	; 0x28
 800266a:	80fb      	strh	r3, [r7, #6]
  }

  if (y0 > y1)
 800266c:	f9b7 2008 	ldrsh.w	r2, [r7, #8]
 8002670:	f9b7 3048 	ldrsh.w	r3, [r7, #72]	; 0x48
 8002674:	429a      	cmp	r2, r3
 8002676:	dd0d      	ble.n	8002694 <_ZN8Graphics12fillTriangleEsssssst+0x9a>
  {
    _swap_int16_t(y0, y1);
 8002678:	893b      	ldrh	r3, [r7, #8]
 800267a:	84fb      	strh	r3, [r7, #38]	; 0x26
 800267c:	f8b7 3048 	ldrh.w	r3, [r7, #72]	; 0x48
 8002680:	813b      	strh	r3, [r7, #8]
 8002682:	8cfb      	ldrh	r3, [r7, #38]	; 0x26
 8002684:	f8a7 3048 	strh.w	r3, [r7, #72]	; 0x48
    _swap_int16_t(x0, x1);
 8002688:	897b      	ldrh	r3, [r7, #10]
 800268a:	84bb      	strh	r3, [r7, #36]	; 0x24
 800268c:	88fb      	ldrh	r3, [r7, #6]
 800268e:	817b      	strh	r3, [r7, #10]
 8002690:	8cbb      	ldrh	r3, [r7, #36]	; 0x24
 8002692:	80fb      	strh	r3, [r7, #6]
  }

  if(y0 == y2)
 8002694:	f9b7 2008 	ldrsh.w	r2, [r7, #8]
 8002698:	f9b7 3050 	ldrsh.w	r3, [r7, #80]	; 0x50
 800269c:	429a      	cmp	r2, r3
 800269e:	d13a      	bne.n	8002716 <_ZN8Graphics12fillTriangleEsssssst+0x11c>
  {
    // Handle awkward all-on-same-line case as its own thing
    a = b = x0;
 80026a0:	897b      	ldrh	r3, [r7, #10]
 80026a2:	87bb      	strh	r3, [r7, #60]	; 0x3c
 80026a4:	8fbb      	ldrh	r3, [r7, #60]	; 0x3c
 80026a6:	87fb      	strh	r3, [r7, #62]	; 0x3e
    if(x1 < a)      a = x1;
 80026a8:	f9b7 2006 	ldrsh.w	r2, [r7, #6]
 80026ac:	f9b7 303e 	ldrsh.w	r3, [r7, #62]	; 0x3e
 80026b0:	429a      	cmp	r2, r3
 80026b2:	da02      	bge.n	80026ba <_ZN8Graphics12fillTriangleEsssssst+0xc0>
 80026b4:	88fb      	ldrh	r3, [r7, #6]
 80026b6:	87fb      	strh	r3, [r7, #62]	; 0x3e
 80026b8:	e007      	b.n	80026ca <_ZN8Graphics12fillTriangleEsssssst+0xd0>
    else if(x1 > b) b = x1;
 80026ba:	f9b7 2006 	ldrsh.w	r2, [r7, #6]
 80026be:	f9b7 303c 	ldrsh.w	r3, [r7, #60]	; 0x3c
 80026c2:	429a      	cmp	r2, r3
 80026c4:	dd01      	ble.n	80026ca <_ZN8Graphics12fillTriangleEsssssst+0xd0>
 80026c6:	88fb      	ldrh	r3, [r7, #6]
 80026c8:	87bb      	strh	r3, [r7, #60]	; 0x3c
    if(x2 < a)      a = x2;
 80026ca:	f9b7 204c 	ldrsh.w	r2, [r7, #76]	; 0x4c
 80026ce:	f9b7 303e 	ldrsh.w	r3, [r7, #62]	; 0x3e
 80026d2:	429a      	cmp	r2, r3
 80026d4:	da03      	bge.n	80026de <_ZN8Graphics12fillTriangleEsssssst+0xe4>
 80026d6:	f8b7 304c 	ldrh.w	r3, [r7, #76]	; 0x4c
 80026da:	87fb      	strh	r3, [r7, #62]	; 0x3e
 80026dc:	e008      	b.n	80026f0 <_ZN8Graphics12fillTriangleEsssssst+0xf6>
    else if(x2 > b) b = x2;
 80026de:	f9b7 204c 	ldrsh.w	r2, [r7, #76]	; 0x4c
 80026e2:	f9b7 303c 	ldrsh.w	r3, [r7, #60]	; 0x3c
 80026e6:	429a      	cmp	r2, r3
 80026e8:	dd02      	ble.n	80026f0 <_ZN8Graphics12fillTriangleEsssssst+0xf6>
 80026ea:	f8b7 304c 	ldrh.w	r3, [r7, #76]	; 0x4c
 80026ee:	87bb      	strh	r3, [r7, #60]	; 0x3c
    drawFastHLine(a, y0, b-a+1, color);
 80026f0:	8fba      	ldrh	r2, [r7, #60]	; 0x3c
 80026f2:	8ffb      	ldrh	r3, [r7, #62]	; 0x3e
 80026f4:	1ad3      	subs	r3, r2, r3
 80026f6:	b29b      	uxth	r3, r3
 80026f8:	3301      	adds	r3, #1
 80026fa:	b29b      	uxth	r3, r3
 80026fc:	b218      	sxth	r0, r3
 80026fe:	f9b7 2008 	ldrsh.w	r2, [r7, #8]
 8002702:	f9b7 103e 	ldrsh.w	r1, [r7, #62]	; 0x3e
 8002706:	f8b7 3054 	ldrh.w	r3, [r7, #84]	; 0x54
 800270a:	9300      	str	r3, [sp, #0]
 800270c:	4603      	mov	r3, r0
 800270e:	68f8      	ldr	r0, [r7, #12]
 8002710:	f7ff feb4 	bl	800247c <_ZN8Graphics13drawFastHLineEssst>
    return;
 8002714:	e0de      	b.n	80028d4 <_ZN8Graphics12fillTriangleEsssssst+0x2da>
  }

  int16_t
  dx01 = x1 - x0,
 8002716:	88fa      	ldrh	r2, [r7, #6]
 8002718:	897b      	ldrh	r3, [r7, #10]
 800271a:	1ad3      	subs	r3, r2, r3
 800271c:	b29b      	uxth	r3, r3
 800271e:	847b      	strh	r3, [r7, #34]	; 0x22
  dy01 = y1 - y0,
 8002720:	f8b7 2048 	ldrh.w	r2, [r7, #72]	; 0x48
 8002724:	893b      	ldrh	r3, [r7, #8]
 8002726:	1ad3      	subs	r3, r2, r3
 8002728:	b29b      	uxth	r3, r3
 800272a:	843b      	strh	r3, [r7, #32]
  dx02 = x2 - x0,
 800272c:	f8b7 204c 	ldrh.w	r2, [r7, #76]	; 0x4c
 8002730:	897b      	ldrh	r3, [r7, #10]
 8002732:	1ad3      	subs	r3, r2, r3
 8002734:	b29b      	uxth	r3, r3
 8002736:	83fb      	strh	r3, [r7, #30]
  dy02 = y2 - y0,
 8002738:	f8b7 2050 	ldrh.w	r2, [r7, #80]	; 0x50
 800273c:	893b      	ldrh	r3, [r7, #8]
 800273e:	1ad3      	subs	r3, r2, r3
 8002740:	b29b      	uxth	r3, r3
 8002742:	83bb      	strh	r3, [r7, #28]
  dx12 = x2 - x1,
 8002744:	f8b7 204c 	ldrh.w	r2, [r7, #76]	; 0x4c
 8002748:	88fb      	ldrh	r3, [r7, #6]
 800274a:	1ad3      	subs	r3, r2, r3
 800274c:	b29b      	uxth	r3, r3
 800274e:	837b      	strh	r3, [r7, #26]
  dy12 = y2 - y1;
 8002750:	f8b7 2050 	ldrh.w	r2, [r7, #80]	; 0x50
 8002754:	f8b7 3048 	ldrh.w	r3, [r7, #72]	; 0x48
 8002758:	1ad3      	subs	r3, r2, r3
 800275a:	b29b      	uxth	r3, r3
 800275c:	833b      	strh	r3, [r7, #24]
  int32_t
  sa   = 0,
 800275e:	2300      	movs	r3, #0
 8002760:	637b      	str	r3, [r7, #52]	; 0x34
  sb   = 0;
 8002762:	2300      	movs	r3, #0
 8002764:	633b      	str	r3, [r7, #48]	; 0x30


  if(y1 == y2) last = y1;   // Include y1 scanline
 8002766:	f9b7 2048 	ldrsh.w	r2, [r7, #72]	; 0x48
 800276a:	f9b7 3050 	ldrsh.w	r3, [r7, #80]	; 0x50
 800276e:	429a      	cmp	r2, r3
 8002770:	d103      	bne.n	800277a <_ZN8Graphics12fillTriangleEsssssst+0x180>
 8002772:	f8b7 3048 	ldrh.w	r3, [r7, #72]	; 0x48
 8002776:	873b      	strh	r3, [r7, #56]	; 0x38
 8002778:	e004      	b.n	8002784 <_ZN8Graphics12fillTriangleEsssssst+0x18a>
  else         last = y1-1; // Skip it
 800277a:	f8b7 3048 	ldrh.w	r3, [r7, #72]	; 0x48
 800277e:	3b01      	subs	r3, #1
 8002780:	b29b      	uxth	r3, r3
 8002782:	873b      	strh	r3, [r7, #56]	; 0x38

  for(y=y0; y<=last; y++)
 8002784:	893b      	ldrh	r3, [r7, #8]
 8002786:	877b      	strh	r3, [r7, #58]	; 0x3a
 8002788:	f9b7 203a 	ldrsh.w	r2, [r7, #58]	; 0x3a
 800278c:	f9b7 3038 	ldrsh.w	r3, [r7, #56]	; 0x38
 8002790:	429a      	cmp	r2, r3
 8002792:	dc42      	bgt.n	800281a <_ZN8Graphics12fillTriangleEsssssst+0x220>
  {
    a   = x0 + sa / dy01;
 8002794:	f9b7 3020 	ldrsh.w	r3, [r7, #32]
 8002798:	6b7a      	ldr	r2, [r7, #52]	; 0x34
 800279a:	fb92 f3f3 	sdiv	r3, r2, r3
 800279e:	b29a      	uxth	r2, r3
 80027a0:	897b      	ldrh	r3, [r7, #10]
 80027a2:	4413      	add	r3, r2
 80027a4:	b29b      	uxth	r3, r3
 80027a6:	87fb      	strh	r3, [r7, #62]	; 0x3e
    b   = x0 + sb / dy02;
 80027a8:	f9b7 301c 	ldrsh.w	r3, [r7, #28]
 80027ac:	6b3a      	ldr	r2, [r7, #48]	; 0x30
 80027ae:	fb92 f3f3 	sdiv	r3, r2, r3
 80027b2:	b29a      	uxth	r2, r3
 80027b4:	897b      	ldrh	r3, [r7, #10]
 80027b6:	4413      	add	r3, r2
 80027b8:	b29b      	uxth	r3, r3
 80027ba:	87bb      	strh	r3, [r7, #60]	; 0x3c
    sa += dx01;
 80027bc:	f9b7 3022 	ldrsh.w	r3, [r7, #34]	; 0x22
 80027c0:	6b7a      	ldr	r2, [r7, #52]	; 0x34
 80027c2:	4413      	add	r3, r2
 80027c4:	637b      	str	r3, [r7, #52]	; 0x34
    sb += dx02;
 80027c6:	f9b7 301e 	ldrsh.w	r3, [r7, #30]
 80027ca:	6b3a      	ldr	r2, [r7, #48]	; 0x30
 80027cc:	4413      	add	r3, r2
 80027ce:	633b      	str	r3, [r7, #48]	; 0x30

    if(a > b) _swap_int16_t(a,b);
 80027d0:	f9b7 203e 	ldrsh.w	r2, [r7, #62]	; 0x3e
 80027d4:	f9b7 303c 	ldrsh.w	r3, [r7, #60]	; 0x3c
 80027d8:	429a      	cmp	r2, r3
 80027da:	dd05      	ble.n	80027e8 <_ZN8Graphics12fillTriangleEsssssst+0x1ee>
 80027dc:	8ffb      	ldrh	r3, [r7, #62]	; 0x3e
 80027de:	82fb      	strh	r3, [r7, #22]
 80027e0:	8fbb      	ldrh	r3, [r7, #60]	; 0x3c
 80027e2:	87fb      	strh	r3, [r7, #62]	; 0x3e
 80027e4:	8afb      	ldrh	r3, [r7, #22]
 80027e6:	87bb      	strh	r3, [r7, #60]	; 0x3c
    drawFastHLine(a, y, b-a+1, color);
 80027e8:	8fba      	ldrh	r2, [r7, #60]	; 0x3c
 80027ea:	8ffb      	ldrh	r3, [r7, #62]	; 0x3e
 80027ec:	1ad3      	subs	r3, r2, r3
 80027ee:	b29b      	uxth	r3, r3
 80027f0:	3301      	adds	r3, #1
 80027f2:	b29b      	uxth	r3, r3
 80027f4:	b218      	sxth	r0, r3
 80027f6:	f9b7 203a 	ldrsh.w	r2, [r7, #58]	; 0x3a
 80027fa:	f9b7 103e 	ldrsh.w	r1, [r7, #62]	; 0x3e
 80027fe:	f8b7 3054 	ldrh.w	r3, [r7, #84]	; 0x54
 8002802:	9300      	str	r3, [sp, #0]
 8002804:	4603      	mov	r3, r0
 8002806:	68f8      	ldr	r0, [r7, #12]
 8002808:	f7ff fe38 	bl	800247c <_ZN8Graphics13drawFastHLineEssst>
  for(y=y0; y<=last; y++)
 800280c:	f9b7 303a 	ldrsh.w	r3, [r7, #58]	; 0x3a
 8002810:	b29b      	uxth	r3, r3
 8002812:	3301      	adds	r3, #1
 8002814:	b29b      	uxth	r3, r3
 8002816:	877b      	strh	r3, [r7, #58]	; 0x3a
 8002818:	e7b6      	b.n	8002788 <_ZN8Graphics12fillTriangleEsssssst+0x18e>
  }

  // For lower part of triangle, find scanline crossings for segments
  // 0-2 and 1-2.  This loop is skipped if y1=y2.
  sa = dx12 * (y - y1);
 800281a:	f9b7 301a 	ldrsh.w	r3, [r7, #26]
 800281e:	f9b7 103a 	ldrsh.w	r1, [r7, #58]	; 0x3a
 8002822:	f9b7 2048 	ldrsh.w	r2, [r7, #72]	; 0x48
 8002826:	1a8a      	subs	r2, r1, r2
 8002828:	fb02 f303 	mul.w	r3, r2, r3
 800282c:	637b      	str	r3, [r7, #52]	; 0x34
  sb = dx02 * (y - y0);
 800282e:	f9b7 301e 	ldrsh.w	r3, [r7, #30]
 8002832:	f9b7 103a 	ldrsh.w	r1, [r7, #58]	; 0x3a
 8002836:	f9b7 2008 	ldrsh.w	r2, [r7, #8]
 800283a:	1a8a      	subs	r2, r1, r2
 800283c:	fb02 f303 	mul.w	r3, r2, r3
 8002840:	633b      	str	r3, [r7, #48]	; 0x30

  for(; y<=y2; y++)
 8002842:	f9b7 203a 	ldrsh.w	r2, [r7, #58]	; 0x3a
 8002846:	f9b7 3050 	ldrsh.w	r3, [r7, #80]	; 0x50
 800284a:	429a      	cmp	r2, r3
 800284c:	dc42      	bgt.n	80028d4 <_ZN8Graphics12fillTriangleEsssssst+0x2da>
  {
    a   = x1 + sa / dy12;
 800284e:	f9b7 3018 	ldrsh.w	r3, [r7, #24]
 8002852:	6b7a      	ldr	r2, [r7, #52]	; 0x34
 8002854:	fb92 f3f3 	sdiv	r3, r2, r3
 8002858:	b29a      	uxth	r2, r3
 800285a:	88fb      	ldrh	r3, [r7, #6]
 800285c:	4413      	add	r3, r2
 800285e:	b29b      	uxth	r3, r3
 8002860:	87fb      	strh	r3, [r7, #62]	; 0x3e
    b   = x0 + sb / dy02;
 8002862:	f9b7 301c 	ldrsh.w	r3, [r7, #28]
 8002866:	6b3a      	ldr	r2, [r7, #48]	; 0x30
 8002868:	fb92 f3f3 	sdiv	r3, r2, r3
 800286c:	b29a      	uxth	r2, r3
 800286e:	897b      	ldrh	r3, [r7, #10]
 8002870:	4413      	add	r3, r2
 8002872:	b29b      	uxth	r3, r3
 8002874:	87bb      	strh	r3, [r7, #60]	; 0x3c
    sa += dx12;
 8002876:	f9b7 301a 	ldrsh.w	r3, [r7, #26]
 800287a:	6b7a      	ldr	r2, [r7, #52]	; 0x34
 800287c:	4413      	add	r3, r2
 800287e:	637b      	str	r3, [r7, #52]	; 0x34
    sb += dx02;
 8002880:	f9b7 301e 	ldrsh.w	r3, [r7, #30]
 8002884:	6b3a      	ldr	r2, [r7, #48]	; 0x30
 8002886:	4413      	add	r3, r2
 8002888:	633b      	str	r3, [r7, #48]	; 0x30
    /* longhand:
    a = x1 + (x2 - x1) * (y - y1) / (y2 - y1);
    b = x0 + (x2 - x0) * (y - y0) / (y2 - y0);
    */
    if(a > b) _swap_int16_t(a,b);
 800288a:	f9b7 203e 	ldrsh.w	r2, [r7, #62]	; 0x3e
 800288e:	f9b7 303c 	ldrsh.w	r3, [r7, #60]	; 0x3c
 8002892:	429a      	cmp	r2, r3
 8002894:	dd05      	ble.n	80028a2 <_ZN8Graphics12fillTriangleEsssssst+0x2a8>
 8002896:	8ffb      	ldrh	r3, [r7, #62]	; 0x3e
 8002898:	82bb      	strh	r3, [r7, #20]
 800289a:	8fbb      	ldrh	r3, [r7, #60]	; 0x3c
 800289c:	87fb      	strh	r3, [r7, #62]	; 0x3e
 800289e:	8abb      	ldrh	r3, [r7, #20]
 80028a0:	87bb      	strh	r3, [r7, #60]	; 0x3c
    drawFastHLine(a, y, b-a+1, color);
 80028a2:	8fba      	ldrh	r2, [r7, #60]	; 0x3c
 80028a4:	8ffb      	ldrh	r3, [r7, #62]	; 0x3e
 80028a6:	1ad3      	subs	r3, r2, r3
 80028a8:	b29b      	uxth	r3, r3
 80028aa:	3301      	adds	r3, #1
 80028ac:	b29b      	uxth	r3, r3
 80028ae:	b218      	sxth	r0, r3
 80028b0:	f9b7 203a 	ldrsh.w	r2, [r7, #58]	; 0x3a
 80028b4:	f9b7 103e 	ldrsh.w	r1, [r7, #62]	; 0x3e
 80028b8:	f8b7 3054 	ldrh.w	r3, [r7, #84]	; 0x54
 80028bc:	9300      	str	r3, [sp, #0]
 80028be:	4603      	mov	r3, r0
 80028c0:	68f8      	ldr	r0, [r7, #12]
 80028c2:	f7ff fddb 	bl	800247c <_ZN8Graphics13drawFastHLineEssst>
  for(; y<=y2; y++)
 80028c6:	f9b7 303a 	ldrsh.w	r3, [r7, #58]	; 0x3a
 80028ca:	b29b      	uxth	r3, r3
 80028cc:	3301      	adds	r3, #1
 80028ce:	b29b      	uxth	r3, r3
 80028d0:	877b      	strh	r3, [r7, #58]	; 0x3a
 80028d2:	e7b6      	b.n	8002842 <_ZN8Graphics12fillTriangleEsssssst+0x248>
  }
}
 80028d4:	3740      	adds	r7, #64	; 0x40
 80028d6:	46bd      	mov	sp, r7
 80028d8:	bd80      	pop	{r7, pc}

080028da <_ZN8Graphics9setCursorEss>:
    @param  x    X coordinate in pixels
    @param  y    Y coordinate in pixels
*/
/**************************************************************************/
void Graphics::setCursor(int16_t x, int16_t y)
{
 80028da:	b480      	push	{r7}
 80028dc:	b083      	sub	sp, #12
 80028de:	af00      	add	r7, sp, #0
 80028e0:	6078      	str	r0, [r7, #4]
 80028e2:	460b      	mov	r3, r1
 80028e4:	807b      	strh	r3, [r7, #2]
 80028e6:	4613      	mov	r3, r2
 80028e8:	803b      	strh	r3, [r7, #0]
  m_cursorX = x;
 80028ea:	687b      	ldr	r3, [r7, #4]
 80028ec:	f503 530e 	add.w	r3, r3, #9088	; 0x2380
 80028f0:	3306      	adds	r3, #6
 80028f2:	887a      	ldrh	r2, [r7, #2]
 80028f4:	801a      	strh	r2, [r3, #0]
  m_cursorY = y;
 80028f6:	687b      	ldr	r3, [r7, #4]
 80028f8:	f503 530e 	add.w	r3, r3, #9088	; 0x2380
 80028fc:	3308      	adds	r3, #8
 80028fe:	883a      	ldrh	r2, [r7, #0]
 8002900:	801a      	strh	r2, [r3, #0]
}
 8002902:	bf00      	nop
 8002904:	370c      	adds	r7, #12
 8002906:	46bd      	mov	sp, r7
 8002908:	f85d 7b04 	ldr.w	r7, [sp], #4
 800290c:	4770      	bx	lr

0800290e <_ZN8Graphics11setTextSizeEh>:
    @brief   Set text 'magnification' size. Each increase in s makes 1 pixel that much bigger.
    @param  s  Desired text size. 1 is default 6x8, 2 is 12x16, 3 is 18x24, etc
*/
/**************************************************************************/
void Graphics::setTextSize(uint8_t s)
{
 800290e:	b480      	push	{r7}
 8002910:	b083      	sub	sp, #12
 8002912:	af00      	add	r7, sp, #0
 8002914:	6078      	str	r0, [r7, #4]
 8002916:	460b      	mov	r3, r1
 8002918:	70fb      	strb	r3, [r7, #3]
  m_textSize = (s > 0) ? s : 1;
 800291a:	78fb      	ldrb	r3, [r7, #3]
 800291c:	2b00      	cmp	r3, #0
 800291e:	d001      	beq.n	8002924 <_ZN8Graphics11setTextSizeEh+0x16>
 8002920:	78fa      	ldrb	r2, [r7, #3]
 8002922:	e000      	b.n	8002926 <_ZN8Graphics11setTextSizeEh+0x18>
 8002924:	2201      	movs	r2, #1
 8002926:	687b      	ldr	r3, [r7, #4]
 8002928:	f503 530e 	add.w	r3, r3, #9088	; 0x2380
 800292c:	330e      	adds	r3, #14
 800292e:	701a      	strb	r2, [r3, #0]
}
 8002930:	bf00      	nop
 8002932:	370c      	adds	r7, #12
 8002934:	46bd      	mov	sp, r7
 8002936:	f85d 7b04 	ldr.w	r7, [sp], #4
 800293a:	4770      	bx	lr

0800293c <_ZN8Graphics8getColorEt>:
    @brief
    @param
*/
/**************************************************************************/
uint16_t Graphics::getColor(uint16_t color)
{
 800293c:	b480      	push	{r7}
 800293e:	b085      	sub	sp, #20
 8002940:	af00      	add	r7, sp, #0
 8002942:	6078      	str	r0, [r7, #4]
 8002944:	460b      	mov	r3, r1
 8002946:	807b      	strh	r3, [r7, #2]
  uint16_t tempColor;
  if(m_invertDisplayFlag)
 8002948:	687b      	ldr	r3, [r7, #4]
 800294a:	f503 530e 	add.w	r3, r3, #9088	; 0x2380
 800294e:	3314      	adds	r3, #20
 8002950:	681b      	ldr	r3, [r3, #0]
 8002952:	2b00      	cmp	r3, #0
 8002954:	d008      	beq.n	8002968 <_ZN8Graphics8getColorEt+0x2c>
  {
    if(color)
 8002956:	887b      	ldrh	r3, [r7, #2]
 8002958:	2b00      	cmp	r3, #0
 800295a:	d002      	beq.n	8002962 <_ZN8Graphics8getColorEt+0x26>
      tempColor = 0 ;
 800295c:	2300      	movs	r3, #0
 800295e:	81fb      	strh	r3, [r7, #14]
 8002960:	e004      	b.n	800296c <_ZN8Graphics8getColorEt+0x30>
    else
      tempColor = 1 ;
 8002962:	2301      	movs	r3, #1
 8002964:	81fb      	strh	r3, [r7, #14]
 8002966:	e001      	b.n	800296c <_ZN8Graphics8getColorEt+0x30>
  }
  else
  {
    tempColor = color;
 8002968:	887b      	ldrh	r3, [r7, #2]
 800296a:	81fb      	strh	r3, [r7, #14]
  }
  return tempColor;
 800296c:	89fb      	ldrh	r3, [r7, #14]
}
 800296e:	4618      	mov	r0, r3
 8002970:	3714      	adds	r7, #20
 8002972:	46bd      	mov	sp, r7
 8002974:	f85d 7b04 	ldr.w	r7, [sp], #4
 8002978:	4770      	bx	lr

0800297a <_ZN8Graphics16setInvertDisplayEi>:
    @brief      Invert the display (ideally using built-in hardware command)
    @param   i  True if you want to invert, false to make 'normal'
*/
/**************************************************************************/
void Graphics::setInvertDisplay(bool i)
{
 800297a:	b480      	push	{r7}
 800297c:	b083      	sub	sp, #12
 800297e:	af00      	add	r7, sp, #0
 8002980:	6078      	str	r0, [r7, #4]
 8002982:	6039      	str	r1, [r7, #0]
  // Do nothing, must be subclassed if supported by hardware
  m_invertDisplayFlag = i;
 8002984:	687b      	ldr	r3, [r7, #4]
 8002986:	f503 530e 	add.w	r3, r3, #9088	; 0x2380
 800298a:	3314      	adds	r3, #20
 800298c:	683a      	ldr	r2, [r7, #0]
 800298e:	601a      	str	r2, [r3, #0]
}
 8002990:	bf00      	nop
 8002992:	370c      	adds	r7, #12
 8002994:	46bd      	mov	sp, r7
 8002996:	f85d 7b04 	ldr.w	r7, [sp], #4
 800299a:	4770      	bx	lr

0800299c <_ZN8Graphics16getInvertDisplayEv>:
    @brief      returns the Invert resule (ideally using built-in hardware command)
    @param   i  True if you want to invert, false to make 'normal'
*/
/**************************************************************************/
bool Graphics::getInvertDisplay()
{
 800299c:	b480      	push	{r7}
 800299e:	b083      	sub	sp, #12
 80029a0:	af00      	add	r7, sp, #0
 80029a2:	6078      	str	r0, [r7, #4]
  return m_invertDisplayFlag;
 80029a4:	687b      	ldr	r3, [r7, #4]
 80029a6:	f503 530e 	add.w	r3, r3, #9088	; 0x2380
 80029aa:	3314      	adds	r3, #20
 80029ac:	681b      	ldr	r3, [r3, #0]
}
 80029ae:	4618      	mov	r0, r3
 80029b0:	370c      	adds	r7, #12
 80029b2:	46bd      	mov	sp, r7
 80029b4:	f85d 7b04 	ldr.w	r7, [sp], #4
 80029b8:	4770      	bx	lr

080029ba <_ZN8Graphics9clearRectEv>:
    @param      if m_invertDisplayFlag is true it sets the array buffers to 0xFF;
                if false it sets the array buffers to 0x00
*/
/**************************************************************************/
void Graphics::clearRect(void)
{
 80029ba:	b580      	push	{r7, lr}
 80029bc:	b082      	sub	sp, #8
 80029be:	af00      	add	r7, sp, #0
 80029c0:	6078      	str	r0, [r7, #4]
  // m_sharpMem.fillRect(0,0,128,128,WHITE);

  if(getInvertDisplay())
 80029c2:	6878      	ldr	r0, [r7, #4]
 80029c4:	f7ff ffea 	bl	800299c <_ZN8Graphics16getInvertDisplayEv>
 80029c8:	4603      	mov	r3, r0
 80029ca:	2b00      	cmp	r3, #0
 80029cc:	bf14      	ite	ne
 80029ce:	2301      	movne	r3, #1
 80029d0:	2300      	moveq	r3, #0
 80029d2:	b2db      	uxtb	r3, r3
 80029d4:	2b00      	cmp	r3, #0
 80029d6:	d003      	beq.n	80029e0 <_ZN8Graphics9clearRectEv+0x26>
  {
    setBuffer();
 80029d8:	6878      	ldr	r0, [r7, #4]
 80029da:	f000 f817 	bl	8002a0c <_ZN8Graphics9setBufferEv>
  }
  else
  {
    clearBuffer();
  }
}
 80029de:	e002      	b.n	80029e6 <_ZN8Graphics9clearRectEv+0x2c>
    clearBuffer();
 80029e0:	6878      	ldr	r0, [r7, #4]
 80029e2:	f000 f804 	bl	80029ee <_ZN8Graphics11clearBufferEv>
}
 80029e6:	bf00      	nop
 80029e8:	3708      	adds	r7, #8
 80029ea:	46bd      	mov	sp, r7
 80029ec:	bd80      	pop	{r7, pc}

080029ee <_ZN8Graphics11clearBufferEv>:
    @brief      clear the image buffer sets to 0xFF
    @param      None
*/
/**************************************************************************/
void Graphics::clearBuffer()
{
 80029ee:	b580      	push	{r7, lr}
 80029f0:	b082      	sub	sp, #8
 80029f2:	af00      	add	r7, sp, #0
 80029f4:	6078      	str	r0, [r7, #4]
  memset(m_displayBuffer, 0xff, BUFFER_SIZE);
 80029f6:	687b      	ldr	r3, [r7, #4]
 80029f8:	f242 3282 	movw	r2, #9090	; 0x2382
 80029fc:	21ff      	movs	r1, #255	; 0xff
 80029fe:	4618      	mov	r0, r3
 8002a00:	f003 ff95 	bl	800692e <memset>
}
 8002a04:	bf00      	nop
 8002a06:	3708      	adds	r7, #8
 8002a08:	46bd      	mov	sp, r7
 8002a0a:	bd80      	pop	{r7, pc}

08002a0c <_ZN8Graphics9setBufferEv>:
    @brief      sets the image buffer sets to 0x00
    @param      None
*/
/**************************************************************************/
void Graphics::setBuffer()
{
 8002a0c:	b580      	push	{r7, lr}
 8002a0e:	b082      	sub	sp, #8
 8002a10:	af00      	add	r7, sp, #0
 8002a12:	6078      	str	r0, [r7, #4]
  memset(m_displayBuffer, 0x00, BUFFER_SIZE);
 8002a14:	687b      	ldr	r3, [r7, #4]
 8002a16:	f242 3282 	movw	r2, #9090	; 0x2382
 8002a1a:	2100      	movs	r1, #0
 8002a1c:	4618      	mov	r0, r3
 8002a1e:	f003 ff86 	bl	800692e <memset>
}
 8002a22:	bf00      	nop
 8002a24:	3708      	adds	r7, #8
 8002a26:	46bd      	mov	sp, r7
 8002a28:	bd80      	pop	{r7, pc}

08002a2a <_ZN8Graphics13getDisplayPtrEt>:
    @brief      returns the pointer to the image buffer
    @param      index if the location in the image buffer.
*/
/**************************************************************************/
uint8_t*  Graphics::getDisplayPtr(uint16_t index)
{
 8002a2a:	b480      	push	{r7}
 8002a2c:	b083      	sub	sp, #12
 8002a2e:	af00      	add	r7, sp, #0
 8002a30:	6078      	str	r0, [r7, #4]
 8002a32:	460b      	mov	r3, r1
 8002a34:	807b      	strh	r3, [r7, #2]
	if ((index < 0) || (index > BUFFER_SIZE))
 8002a36:	887b      	ldrh	r3, [r7, #2]
 8002a38:	f242 3282 	movw	r2, #9090	; 0x2382
 8002a3c:	4293      	cmp	r3, r2
 8002a3e:	d901      	bls.n	8002a44 <_ZN8Graphics13getDisplayPtrEt+0x1a>
		return NULL;
 8002a40:	2300      	movs	r3, #0
 8002a42:	e002      	b.n	8002a4a <_ZN8Graphics13getDisplayPtrEt+0x20>

	return &m_displayBuffer[index];
 8002a44:	887b      	ldrh	r3, [r7, #2]
 8002a46:	687a      	ldr	r2, [r7, #4]
 8002a48:	4413      	add	r3, r2
}
 8002a4a:	4618      	mov	r0, r3
 8002a4c:	370c      	adds	r7, #12
 8002a4e:	46bd      	mov	sp, r7
 8002a50:	f85d 7b04 	ldr.w	r7, [sp], #4
 8002a54:	4770      	bx	lr
	...

08002a58 <Graphics_setInvertDisplay>:

//***** API Functions definition *****//
//****Remember "API" is used like "public" in C++*******//

void Graphics_setInvertDisplay(bool index)
{
 8002a58:	b580      	push	{r7, lr}
 8002a5a:	b082      	sub	sp, #8
 8002a5c:	af00      	add	r7, sp, #0
 8002a5e:	6078      	str	r0, [r7, #4]
	g_Graphics.setInvertDisplay(index);
 8002a60:	6879      	ldr	r1, [r7, #4]
 8002a62:	4803      	ldr	r0, [pc, #12]	; (8002a70 <Graphics_setInvertDisplay+0x18>)
 8002a64:	f7ff ff89 	bl	800297a <_ZN8Graphics16setInvertDisplayEi>
}
 8002a68:	bf00      	nop
 8002a6a:	3708      	adds	r7, #8
 8002a6c:	46bd      	mov	sp, r7
 8002a6e:	bd80      	pop	{r7, pc}
 8002a70:	200000a8 	.word	0x200000a8

08002a74 <Graphics_clearRect>:

void Graphics_clearRect(void)
{
 8002a74:	b580      	push	{r7, lr}
 8002a76:	af00      	add	r7, sp, #0
	g_Graphics.clearRect();
 8002a78:	4802      	ldr	r0, [pc, #8]	; (8002a84 <Graphics_clearRect+0x10>)
 8002a7a:	f7ff ff9e 	bl	80029ba <_ZN8Graphics9clearRectEv>
}
 8002a7e:	bf00      	nop
 8002a80:	bd80      	pop	{r7, pc}
 8002a82:	bf00      	nop
 8002a84:	200000a8 	.word	0x200000a8

08002a88 <Graphics_fillCircle>:
{
	g_Graphics.drawCircleHelper(x0, y0, r, cornername, color);
}

void Graphics_fillCircle(int16_t x0, int16_t y0, int16_t r,uint16_t color)
{
 8002a88:	b590      	push	{r4, r7, lr}
 8002a8a:	b085      	sub	sp, #20
 8002a8c:	af02      	add	r7, sp, #8
 8002a8e:	4604      	mov	r4, r0
 8002a90:	4608      	mov	r0, r1
 8002a92:	4611      	mov	r1, r2
 8002a94:	461a      	mov	r2, r3
 8002a96:	4623      	mov	r3, r4
 8002a98:	80fb      	strh	r3, [r7, #6]
 8002a9a:	4603      	mov	r3, r0
 8002a9c:	80bb      	strh	r3, [r7, #4]
 8002a9e:	460b      	mov	r3, r1
 8002aa0:	807b      	strh	r3, [r7, #2]
 8002aa2:	4613      	mov	r3, r2
 8002aa4:	803b      	strh	r3, [r7, #0]
	g_Graphics.fillCircle(x0, y0, r, color);
 8002aa6:	f9b7 0002 	ldrsh.w	r0, [r7, #2]
 8002aaa:	f9b7 2004 	ldrsh.w	r2, [r7, #4]
 8002aae:	f9b7 1006 	ldrsh.w	r1, [r7, #6]
 8002ab2:	883b      	ldrh	r3, [r7, #0]
 8002ab4:	9300      	str	r3, [sp, #0]
 8002ab6:	4603      	mov	r3, r0
 8002ab8:	4803      	ldr	r0, [pc, #12]	; (8002ac8 <Graphics_fillCircle+0x40>)
 8002aba:	f7ff fada 	bl	8002072 <_ZN8Graphics10fillCircleEssst>
}
 8002abe:	bf00      	nop
 8002ac0:	370c      	adds	r7, #12
 8002ac2:	46bd      	mov	sp, r7
 8002ac4:	bd90      	pop	{r4, r7, pc}
 8002ac6:	bf00      	nop
 8002ac8:	200000a8 	.word	0x200000a8

08002acc <Graphics_setCursor>:
{
	g_Graphics.drawBitmapImage(x, y, bitmap, w, h, color);
}

void Graphics_setCursor(int16_t x, int16_t y)
{
 8002acc:	b580      	push	{r7, lr}
 8002ace:	b082      	sub	sp, #8
 8002ad0:	af00      	add	r7, sp, #0
 8002ad2:	4603      	mov	r3, r0
 8002ad4:	460a      	mov	r2, r1
 8002ad6:	80fb      	strh	r3, [r7, #6]
 8002ad8:	4613      	mov	r3, r2
 8002ada:	80bb      	strh	r3, [r7, #4]
	g_Graphics.setCursor(x, y);
 8002adc:	f9b7 2004 	ldrsh.w	r2, [r7, #4]
 8002ae0:	f9b7 3006 	ldrsh.w	r3, [r7, #6]
 8002ae4:	4619      	mov	r1, r3
 8002ae6:	4803      	ldr	r0, [pc, #12]	; (8002af4 <Graphics_setCursor+0x28>)
 8002ae8:	f7ff fef7 	bl	80028da <_ZN8Graphics9setCursorEss>
}
 8002aec:	bf00      	nop
 8002aee:	3708      	adds	r7, #8
 8002af0:	46bd      	mov	sp, r7
 8002af2:	bd80      	pop	{r7, pc}
 8002af4:	200000a8 	.word	0x200000a8

08002af8 <Graphics_setTextSize>:
{
	return g_Graphics.getCursorY();
}

void Graphics_setTextSize(uint8_t s)
{
 8002af8:	b580      	push	{r7, lr}
 8002afa:	b082      	sub	sp, #8
 8002afc:	af00      	add	r7, sp, #0
 8002afe:	4603      	mov	r3, r0
 8002b00:	71fb      	strb	r3, [r7, #7]
	g_Graphics.setTextSize(s);
 8002b02:	79fb      	ldrb	r3, [r7, #7]
 8002b04:	4619      	mov	r1, r3
 8002b06:	4803      	ldr	r0, [pc, #12]	; (8002b14 <Graphics_setTextSize+0x1c>)
 8002b08:	f7ff ff01 	bl	800290e <_ZN8Graphics11setTextSizeEh>
}
 8002b0c:	bf00      	nop
 8002b0e:	3708      	adds	r7, #8
 8002b10:	46bd      	mov	sp, r7
 8002b12:	bd80      	pop	{r7, pc}
 8002b14:	200000a8 	.word	0x200000a8

08002b18 <LCD_Sharp_Init>:

//***** API Functions definition *****//
//****Remember "API" is used like "public" in C++*******//

void LCD_Sharp_Init(LCD_SHARP_CONFIG* lcdConfig)
{
 8002b18:	b580      	push	{r7, lr}
 8002b1a:	b082      	sub	sp, #8
 8002b1c:	af00      	add	r7, sp, #0
 8002b1e:	6078      	str	r0, [r7, #4]
	m_sharpConfig.extMode = lcdConfig->extMode;
 8002b20:	687b      	ldr	r3, [r7, #4]
 8002b22:	f893 2084 	ldrb.w	r2, [r3, #132]	; 0x84
 8002b26:	4b3e      	ldr	r3, [pc, #248]	; (8002c20 <LCD_Sharp_Init+0x108>)
 8002b28:	f883 2084 	strb.w	r2, [r3, #132]	; 0x84
	m_sharpConfig.gpioCsPin = lcdConfig->gpioCsPin;
 8002b2c:	687b      	ldr	r3, [r7, #4]
 8002b2e:	889a      	ldrh	r2, [r3, #4]
 8002b30:	4b3b      	ldr	r3, [pc, #236]	; (8002c20 <LCD_Sharp_Init+0x108>)
 8002b32:	809a      	strh	r2, [r3, #4]
	m_sharpConfig.gpioCsPort = lcdConfig->gpioCsPort;
 8002b34:	687b      	ldr	r3, [r7, #4]
 8002b36:	681b      	ldr	r3, [r3, #0]
 8002b38:	4a39      	ldr	r2, [pc, #228]	; (8002c20 <LCD_Sharp_Init+0x108>)
 8002b3a:	6013      	str	r3, [r2, #0]
	m_sharpConfig.gpioDispPin = lcdConfig->gpioDispPin;
 8002b3c:	687b      	ldr	r3, [r7, #4]
 8002b3e:	899a      	ldrh	r2, [r3, #12]
 8002b40:	4b37      	ldr	r3, [pc, #220]	; (8002c20 <LCD_Sharp_Init+0x108>)
 8002b42:	819a      	strh	r2, [r3, #12]
	m_sharpConfig.gpioDispPort = lcdConfig->gpioDispPort;
 8002b44:	687b      	ldr	r3, [r7, #4]
